:020000040800F2
:100000000000011039E107086D2B00085596020821
:10001000D9E10708D9E10708D9E107080000000085
:10002000000000000000000000000000C5460008BD
:10003000C946000800000000CD4600083110010844
:10004000D9E10708D9E10708D9E10708D9E107088C
:10005000D9E10708D9E10708E5D00008E9D0000890
:10006000D9E10708EDD00008F1D000086533000899
:10007000793300088D330008A1330008B533000838
:10008000C9330008DD330008D9E10708D9E10708C2
:10009000D9E10708D9E10708D9E10708F5D0000838
:1000A000113200083932000861320008FD310008C1
:1000B000893200089D320008B1320008D9E10708F2
:1000C000D9E10708D9E10708D9E10708D9E107080C
:1000D000D9E107081D2E0008292E0008D9E10708DC
:1000E000F9D00008D9E10708D1460008ED32000830
:1000F000153300083D330008D9320008F1330008F9
:10010000D9E1070805380008C5320008D9E1070819
:10011000352E0008D9E10708D9E10708D9E1070819
:1001200005340008193400082D3400084134000853
:1001300055340008D9E10708D9E10708D9E10708D3
:10014000D9E10708D9E10708D9E107081D470008E8
:10015000693400087D34000891340008412E0008FD
:10016000D9E10708D9E10708D9E10708D9E107086B
:10017000D9E10708D9E10708D9E10708D9E107085B
:08018000D9E10708D9E10708E5
:10019000D0E907239A423CBFC1685218D01A704771
:1001A000D0E9092300699A4238BF1218D31A0138DE
:1001B000C01A7047D0E90902101AB0FA80F040095D
:1001C000704700BF0246036A4069D168C05C0133D2
:1001D0008B4228BF00231362704700BF436A8269C5
:1001E000D154436A0169426B01338B4228BF00231B
:1001F0004362D36843F08003D3607047436B188831
:1002000010F0100002D01A889B880120704700BFB0
:10021000436B99891A88890610B504460AD592B2AB
:10022000900607D5E26A002A2AD09888216B80B20E
:100230009047636B99891A88090692B210D5100607
:100240000ED5D4E909128A4215D0A1692069895CCA
:100250000132C9B29980B2FBF0F100FB1122A26217
:10026000998A1A88C90592B204D5D20744BF4FF6BD
:10027000F7721A8010BDDA6822F08002DA60EFE7C8
:100280009B88E2696169DBB28B54E269E168636B68
:100290000132B2FBF1F001FB1022E261CAE700BFBC
:1002A000036942681F2B10B40AD95468A3F1200CCB
:1002B000202101FA0CF1214207D15DF8044B70476F
:1002C0001468202199402142F7D081690024C86830
:1002D0000C7480684C68016821F00101016020689D
:1002E00094F805C00C4C818934F81C4089B221EA8D
:1002F00004011F2B818107D9A3F1200120238B400A
:100300005DF8044BD3607047202101FA03F35DF8D8
:10031000044B9360704700BF085308084A1C10B490
:1003200018BF4FF0450C494C08BF4FF0800C4FF4FC
:10033000003300E00BB3626B12EA0C0F03F1FF33E2
:10034000F8D0002924DD626B54071DD403291FD087
:100350003E4B5A6BD2071FD402291BD01A69D2B266
:1003600082421DD101295B691CD0062912D113F4E8
:10037000604F43D1364A13600CE0002904DD636B03
:100380005B0701D40329E3D103205DF8044B7047D8
:10039000002BF9D00020F8E701205DF8044B7047EE
:1003A0001020F2E72B4A1A40002AF3D0002B31DB51
:1003B0005C002DD4980031D4D9002DD41A0131D449
:1003C0005C012DD4D80137D419021DD45A02E7D4C8
:1003D0009C022DD4D80229D4190317D45A0323D44C
:1003E0009C0331D4D8032DD4190429D45A0425D41C
:1003F0009C041FD41807CDD51A20C6E7990405D44C
:100400005A04CDD41B04C5D50F20BEE71320BCE78A
:100410000920BAE71C20B8E70B20B6E70A20B4E7AA
:100420000D20B2E70C20B0E71420AEE71220ACE7B5
:100430001120AAE71920A8E70E20A6E71820A4E7B4
:100440001720A2E71620A0E715209EE7002C014008
:100450001020002008E0FFFDF8B5154DEB6A93B1C0
:10046000696B0129044614D0124BDA6A22F00802A3
:10047000DA6240F2FF5100229963EA62236823F0B6
:1004800001032360F8BD0B4AD36B43F48073D3633D
:10049000F8BD084E40F2FF570023B763B36040F247
:1004A0004C43F3600C20FFF739FFB763DCE700BF74
:1004B00010200020002C0140B14BD3E9011270B58F
:1004C0008C0F83F83840C1F3836483F83940C1F35B
:1004D000016483F83A40100EC1F3074483F83B40AF
:1004E0000001C1F30724C9B283F83C4083F83D10F2
:1004F000D887D98F93F89050C2F3035089B2014343
:10050000C2F30344D987C2F3C03083F84040C2F33A
:100510004031C2F3803483F84100012D83F842401A
:100520004FF0000083F84310C2F3003183F8441009
:10053000C2F3072CD96883F8450040F2D680022D1B
:1005400000F0B0802A204FEA4C0C0CF07E0C83F8AF
:10055000514083F852C093F85240C1F3C012144383
:100560001A6983F8524001F07F01D40F83F85310C9
:1005700083F85440910DC2F3417483F8554001F063
:100580000C01C2F3826483F8564083F8571093F845
:100590005710C2F381542143C2F3405583F85710DA
:1005A00083F85850002583F85950C2F3004583F86A
:1005B0005A50C2F3C03583F85B50C2F3803583F8DC
:1005C0005C50C2F3403583F85D505C69C2F300357E
:1005D00083F85E50C2F3812583F85F50C4F307416E
:1005E000C2F30125C2F3460283F860504FF0010CBC
:1005F00083F861200902220E83F862C083F8642028
:10060000A3F86610B3F86610C4F3072289B2114349
:100610002406A3F8661099699C669A6E0C0E42EA4D
:1006200004429A669C6E0A0A02F47F4222439A664A
:100630009D6EDA69C1F307242C43C9B29C6683F826
:100640006C10110E83F86D10110C090619671C6FE0
:10065000110201F47F0121431967196F120292B24E
:100660000A431A67196F1A6A41EA1261196793F807
:100670007410C2F30354214383F87410110A01F477
:100680007061A3F87610B3F87610C2F3072489B22C
:100690002143C2F34602A3F8761083F8782083F84A
:1006A00079C070BD120402F47C129A649A6C0C0E2C
:1006B00042EA04229A649C6CC1F3074222439A6482
:1006C0009A6C013240F10004A40244EA925492026E
:1006D000C3F880204FF40072C3F88440C1F3072CA4
:1006E000C3F88820C1F380342DE74FEA8C2C0CF43A
:1006F00040649C649C6C920002F47F7222439A6472
:100700009D6CC1F3C26445EA91759D6483F84C40C9
:10071000C1F3026483F84D40CA0BC1F3425483F81D
:100720004E4002F00602C1F3824483F84F4083F842
:10073000502093F85020C1F3C034224383F8502056
:100740009D6C93F8504093F840600234012202FA05
:1007500006F6A2404FEAE27EA2FB062406FB0E4408
:1007600005F1010EA2FB0E2E05FB04447444C3E9FF
:100770002024C1F3072CC3F88860C1F38034E2E67B
:100780001020002038B50D4B0D4C1A6840F2FF5573
:1007900040F24D43A5630121A2600D20E360FFF705
:1007A000BDFDA56340B96069C0F34320A0F104001A
:1007B000B0FA80F0400938BD002038BD102000207C
:1007C000002C01402F4B1A68910102D59A6D5207F7
:1007D0004BD42C4B1A68500202D5DA6E11063CD469
:1007E000284B1A68D20102D59A6D90072DD4254B5B
:1007F0001A68510102D59A6D120717D4214B1A6855
:10080000120112D59A6DD0060FD59A6D510334D4CA
:100810009A6DD20503D49A6D22F010029A65194B95
:1008200019484FF000629A6016E670479A6D5003BF
:1008300007D49A6DD10503D49A6D22F008029A6507
:10084000104B4FF080629A60D8E79A6D4FF080713C
:1008500022F002029A659960C9E7DA6E4FF48001CE
:1008600022F08002DA669960BAE79A6D4FF0007163
:1008700022F004029A659960ABE74FF000629A603B
:10088000704700BF0064024058640240384B5A6809
:10089000110303D5D3F8A02052075BD4344B5A6818
:1008A000D00303D5D3F8B420110649D4304B5A688D
:1008B000520303D5D3F8A020900737D42C4B5A68A5
:1008C000D10203D5D3F8A02012071CD4284B5A68B4
:1008D000920217D5D3F8A020D00613D5D3F8A020C4
:1008E000510341D4D3F8A020D20505D4D3F8A020D9
:1008F00022F01002C3F8A0201D4B1E484FF4001236
:10090000DA60A9E57047D3F8A02050030AD4D3F8E1
:10091000A020D10505D4D3F8A02022F00802C3F806
:10092000A020134B4FF48012DA60CFE7D3F8A02059
:100930004FF4802122F00202C3F8A020D960BDE765
:10094000D3F8B4204FF4803122F08002C3F8B420F1
:10095000D960ABE7D3F8A0204FF4002122F00402C5
:10096000C3F8A020D96099E74FF40012DA6070470D
:1009700000640240A064024082B00922274B8DF837
:100980000720DA68D00319D4DA68D10640D4DA68CF
:10099000D20541D4DA6812F0E00F3BD1DB6813F0E6
:1009A000020F0CBF092308238DF807309DF807308C
:1009B000012B0AD09DF8070002B0704701238DF883
:1009C00007309DF80730012BF4D1144A12E0D368A8
:1009D000DB0519D4D36813F0E00F17D1D36813F0F7
:1009E000020F0CBF092308238DF807309DF807304C
:1009F000012BDFD1D168C8034FF00103F4D4D368D1
:100A0000D906E4D50623EFE70223EDE70723EBE75A
:100A10000623D4E70723D2E70223D0E7003C0240B5
:100A2000704700BF704700BF704700BF012070478C
:100A3000034BD3E92503C01AC0F30A00704700BF77
:100A400010200020064AD2E925139942FDD0D11882
:100A50000133C3F30A0391F89C00C2F89830704741
:100A600010200020064BD3F89C0800B97047D3F83B
:100A70009C08A0F10500B0FA80F04009704700BF63
:100A800010200020012380F849307047044BD3E93F
:100A90002503C01AC0F30A00C0F50060704700BF0C
:100AA0001020002010B5D0F8E83504461B6998479F
:100AB000032384F81231002010BD00BF08B50422C2
:100AC00090F81211D0F8E83580F8131180F812214F
:100AD000DB689847002008BD08B5D0F8E435DB692D
:100AE00003B19847002008BD08B5D0F8E4351B6A6B
:100AF0009847002008BD00BF08B5D0F8E4355B6A10
:100B00009847002008BD00BF70B5037805460E4623
:100B10001446DBB101307CF08BFC431CDBB20133AB
:100B20005B00DAB223800323327073702C7864B1D7
:100B30002846022300215A1CD2B2F454B15410F8B2
:100B4000014F0233DBB2002CF5D170BD02221346F7
:100B5000E8E700BF10B5074C2068FF2808D0064919
:100B6000D1F8A02801F6A40100F082F8FF23236049
:100B7000002010BD00000020102000204323014869
:100B80000B80704704000020122301480B8070473F
:100B900048000020042301480B8070475C000020BF
:100BA00010B5044C04480A462146FFF7ADFF204625
:100BB00010BD00BFBC28002088FA080810B5044CFE
:100BC00004480A462146FFF79FFF204610BD00BF9C
:100BD000BC2800209CFA080810B5044C04480A46BA
:100BE0002146FFF791FF204610BD00BFBC28002022
:100BF000A4FA080810B5044C04480A462146FFF739
:100C000083FF204610BD00BFBC280020B0FA0808B2
:100C100010B5044C04480A462146FFF775FF2046EC
:100C200010BD00BFBC280020BCFA0808704700BFF8
:100C3000704700BF704700BF704700BF704700BFDC
:100C4000704700BF704700BF044B00200522C3F867
:100C50009C28C3F8AC09C3F8B009704710200020E5
:100C6000024B0020C3F89C08704700BF10200020F2
:100C7000212838B50C4625D0222816D0202812D19C
:100C800089B1072A0FD1174DD5F8B03913B10968CA
:100C9000002098472168A288A379C5F8B419A5F85F
:100CA000B82985F8BA39002038BD0029FBD0022ABE
:100CB000F9D10C4BD3F8AC39002BF4D009880020C3
:100CC0009847F0E70029EED0072AECD1054BD3F87E
:100CD000B419B3F8B82993F8BA392160A280A37186
:100CE000E1E700BF1020002010B4114CD4E92532F8
:100CF0009A1AC2F30A020A44B2F5006F14D879B105
:100D000001444A1E013810F801CFE118904203F166
:100D1000010381F89CC0C3F30A03F4D1C4F89430F2
:100D200000205DF8044B704702205DF8044B7047CB
:100D300010200020034B93F8E009003818BF012071
:100D4000704700BF1020002070B5124D124C29686A
:100D500040F2FF5640F24D430022A6630D20A160F1
:100D6000C5F8DC290121E360FFF7D8FAA66320B9B2
:100D70006369C3F34323042B08D0D5F8143AC5F8AC
:100D8000D039092385F8E039002070BD85F8E039B5
:100D9000022070BD10200020002C014070B50E4DC7
:100DA00095F8E039042B04460E460BD0082B07D1EA
:100DB000D5F8D83983420CD0FFF7C6FF022801D0FE
:100DC000012070BD082385F8E039C5F8DC69C5F855
:100DD000D849022070BD00BF10200020034B93F8BB
:100DE000E009032894BF0020012070471020002054
:100DF00000487047F429002030B4184B00209C7B39
:100E000014B11D688D4206D00130082803F110038B
:100E1000F5D130BC7047D2B1114B03EB40218A426F
:100E200011D0104B93F8B42112B9012283F8B421E8
:100E30000D4B01225A7000F5817003EB0013012263
:100E40009A7130BC7047022CEBD1183BF3E7064B8C
:100E500000F5817003EB00139A71DAE7F05C002073
:100E6000F04C0020D85C0020D84C002030B41D4C41
:100E7000002384F8A03004F1180004E00133082BAB
:100E800000F110001ED005688D42F7D190F80EC019
:100E9000BCF1030FF2D1BAB1134901EB43208242F6
:100EA00009D094F8B42112B9012284F8B4210F4971
:100EB00001224A7000E0183903F5817301EB031138
:100EC00001238B7130BC70470849D4F89C2003F58E
:100ED000817301EB0313013204219971C4F89C2042
:100EE000F0E700BFD85C0020F04C0020D84C002078
:100EF000A8B183681BB10E4B07229A7070470C4A49
:100F00001178D36003294FF0040014BF4FF48071AF
:100F10008021C2E901111361137590707047044A72
:100F200002F580510123537081F8B431704700BF3E
:100F3000D84C002010B5812104467BF0C3F8204630
:100F400001217BF0BFF8204682217BF0BBF8FFF740
:100F500087FE002010BD00BF034610B4D9691A698E
:100F6000002040F20114A3F844410860D1699C6D4F
:100F700021F002014FF0010CD161A3F89CC3206065
:100F8000D369044923F4003381F8180A5DF8044B4F
:100F9000D361704710200020202301480B80704748
:100FA00060000020122301480B8070478000002061
:100FB000042301480B807047940000200A4608B5BE
:100FC000054920B90548FFF79FFD034808BD0448BF
:100FD000FFF79AFD004808BD2C2A0020CCFA08082B
:100FE000E4FA080810B5044C04480A462146FFF705
:100FF0008BFD204610BD00BF2C2A0020FCFA0808FB
:101000001C48D0F8E837D0F8EC2710B59B184FF003
:101010001A040C8001D1184810BD174AD0F8EA070D
:1010200002F1100411464FF0000E4FEA137CB3F1A9
:10103000204F34BF0CF1300C0CF1370C81F802C09A
:1010400081F803E002318C424FEA0313EDD102F143
:1010500008040021030FB0F1204F34BF3033373381
:101060009374D174023294424FEA0010F2D10248D4
:1010700010BD00BF00F0FF1F9800002010B5044C09
:1010800004480A462146FFF73FFD204610BD00BF39
:101090002C2A002010FB080810B5044C04480A460E
:1010A0002146FFF731FD204610BD00BF2C2A00204D
:1010B0001CFB080810B50E4C0E4BD4F8F41BB4F80A
:1010C000F80B088303F1B402C4F8682DD3F8B430E8
:1010D0009847D4F8683D002BFBD01B69984700283F
:1010E000F7D0D4F8F43BB4F8F82B5A83002010BDA5
:1010F000102000200000002038B5084BD3F8683DD0
:1011000053B1DB6914460D4698474FF400730268EB
:101110002A600020236038BD1B68FFDE10200020FD
:1011200008B5064BD3F8683D23B11B6998470138D1
:1011300040B208BD4FF0FF3008BD00BF10200020B6
:10114000002070472DE9F041184CD4F8B80B154633
:10115000B4F8BC2B428323B30E4603EB050804E02E
:10116000D4F8683D0BB31B699847D4F8681DE1B10A
:1011700000234F681A4631462846B8470028EFD06A
:10118000D4F8683D002BFBD01B6998470028F7D0A6
:101190000135A84506F50076E7D1D4F8B80BB4F8C8
:1011A000BC2B02830020BDE8F081FEE71020002068
:1011B0002DE9F041184CD4F8B80B1546B4F8BC2B07
:1011C000428323B30E4603EB050801E01B699847F1
:1011D000D4F8681D51B10023CF681A46314628461D
:1011E000B847D4F8683D10B1002BEFD1002313B1FC
:1011F0001B69984710B9D4F8683DF8E701354545B3
:1012000006F50076E4D1D4F8B80BB4F8BC2B028311
:101210000020BDE8F08100BF10200020A14A5368E3
:1012200023F4FD4323F07F032DE9F04143F07603DF
:1012300053605368032123F48073536082B01160BC
:101240000FF042FF04460D460FF03EFF001B61EB1E
:101250000501B0F57A7F71F10001F5D30FF034FF8D
:1012600004460D460FF030FF001B61EB0501B0F5A1
:101270007A7F71F10001F5D38A4C6368002040F257
:10128000FF5543F480734FF4806263604FF0FF3189
:10129000A563A060E260FFF741F8A563074618B1B7
:1012A000012002B0BDE8F0814FF4D5724FF489639C
:1012B000A5630721A2600820E360FFF72FF8A5636C
:1012C00028B9794B012283F890204FF08047754C64
:1012D00040F2FF55002240F27743A5630121A2604E
:1012E0003720E360FFF71AF8A5630028D8D147F04C
:1012F00000470646804647F4801701E09642CFD06B
:1013000040F27743A5630121C4F808803720E360E9
:10131000FFF704F8034640F2694203212920A56340
:10132000002BBDD1A563A760E260FEF7F7FF013691
:101330004FF6FF72A5630028B2D16369002BDDDA96
:101340004FF6FF729642ABD05D0000F1B380236888
:101350009807A5D0544D95F89060042E40F0B280C7
:10136000FFF7AAF800289BD14E4C2B6840F2FF579C
:10137000A763A36040F24743E36001210720FEF723
:10138000CDFFA763636823F4FD4323F07F0363600D
:10139000002885D1022E83D8636913F000737FF48F
:1013A0007FAF009308264FF48A63A7630121A660EC
:1013B0001020E360FEF7B2FFA76300287FF470AF50
:1013C0002B68A763A36040F27743E36001213720D5
:1013D000FEF7A4FFA76300287FF462AF334A62627E
:1013E000A662E26A42F03302E26240F27342A7630D
:1013F0000121A060E2603320FEF790FFA763002880
:101400007FF44EAF6B4640F22A4206E0616B8902E0
:1014100044BFD4F8801043F8041B616B1142F5D02F
:10142000636B1B073FF53CAF636B9F073FF538AF1E
:10143000636B9E063FF534AF636B98023FF530AFA8
:10144000009B1BBA59037FF52BAF2A6840F2774304
:1014500040F2FF55A5630121A2603720E360FEF74B
:101460005DFFA56300287FF41BAF022240F24643D4
:10147000A5630121A2600620E360FEF74FFFA5638C
:1014800000287FF40DAF63681A0509D4054A08499E
:1014900053680B4043F40063536053681B05F7D552
:1014A0000020FEE6002C01401020002000E1F505A0
:1014B0000081FFFF274D022685F8906023689C0776
:1014C0003FF4EEAE244C40F2FF570023A763022105
:1014D000A36040F2C243E3600846FEF71FFFA76324
:1014E00000287FF4DDAE63696B61A369AB61E369DA
:1014F000EB61236A2B62022E1BD9062E19D0164CE3
:101500002B6840F2FF57A763A36040F2C943E36032
:1015100002210920FEF702FFA76300287FF4C0AE76
:1015200063696B60A369AB60E369EB60236A2B615D
:1015300016E7094C40F2FF570023A763A36040F26F
:101540004343E36006210320FEF7E8FEA76300287B
:10155000D5D0A5E610200020002C014010B5104C7D
:10156000D4F80C3A43B119689A880B691A4203D12E
:10157000002384F8E03910BDFFF750FE0028F7D1B2
:1015800094F8D4390133DBB2072B84F8D439EFD87F
:10159000D4F8143AC4F8D039012384F8E03910BDE6
:1015A0001020002070B5A14CD4F8100A002800F0DB
:1015B000138194F8E0596B1E082B0ED8DFE803F076
:1015C000C6057F0D61CA340D1500FFF7DBF8002852
:1015D00040F0058194F8E0596B1EDBB2022B40F21B
:1015E000D380042D47D1012070BD914D226840F277
:1015F000FF5640F24D43AE630121AA600D20EB601F
:10160000FEF78CFEAE6328B96B69C3F34323042B4A
:1016100000F0C780D4F8D039D4F8142AFA339342B2
:10162000D8D2FFF79BFFC4E7814D226840F2FF56F6
:1016300040F24D43AE630121AA600D20EB60FEF73E
:101640006DFEAE630028E5D16B69C3F34323042B21
:10165000E0D1D4F8DC3984F8D409012B40F2DF80E2
:10166000D4F8D8290825013B0132C4F8DC39C4F884
:10167000D82984F8E059A5F10800B0FA80F04009B3
:1016800070BDE66A002E40F09080FFF77BF80028DE
:1016900000F09380D4F8C85984F8D469042384F8FE
:1016A000E039002D9FD0D4F8CC39D4F8BC29D4F837
:1016B000C0193046A84794F8E0596B1E8DE7FEF735
:1016C000FBFE002860D194F86420B4F86630A4F8DA
:1016D000E839A16EA36EC4F8DC09090E04201B0CC6
:1016E00084F8EA2984F8E009A26E84F8EB1984F8FA
:1016F000EC39A16E94F86C0094F86D3084F8EE1912
:10170000120A1B0984F8ED2984F8EF0994F86D207A
:1017100084F8F439216FB4F87600B4F87630C4F860
:10172000F01902F00F02C3F30B1384F8F52943EA12
:101730001023B4F8762003F00F0303F5FA6302F0E8
:101740000F02A4F8F63984F8F82932E7022384F866
:10175000E0392EE7236B002B8DD1D4F8C869D4F87B
:10176000143AC4F8D039072584F8E059002E82D005
:10177000D4F8CC39D4F8BC29D4F8C0190120B0472A
:1017800094F8E0596B1E28E7D4F8143AD4F8D0291D
:101790009B1AC82B7FF66FAFFFF7E0FE94F8E05975
:1017A0001FE7042384F8E0391DE7D4F8D039D4F8D2
:1017B000142A64339342BFF45EAFFFF7CFFED4F830
:1017C000C859002D3FF4F5AE0022D4F8CC39D4F836
:1017D000C0191046A847ECE684F8E00970BDFEF792
:1017E0006BFE00287FF4F6AE94F89030002BA3F146
:1017F0000203B3FA83F308BF01255B0984F8D559C6
:1018000084F8D639FEF758FE00287FF40AAFD4F8E2
:101810008020C4F8E429032384F8E039C9E6C0D164
:10182000FFF792FA94F8E0596B1ED6E610200020DC
:10183000002C01402DE9F0411F4E80460B4696F8E2
:101840006C2D002AFBD19BB343445F1E08F1FF3887
:10185000D6F8703DD6F8742D0133C3F30A039A42CB
:1018600016D10FF031FC04460D460FF02DFC001B85
:1018700061EB0501B0F57A7F71F10001F5D3D6F87F
:10188000703DD6F8742D0133C3F30A039342E8D0B8
:10189000D6F8702DD6F8703D18F8011F3244013388
:1018A000C3F30A03B84582F8781DC6F8703DCFD15E
:1018B0000020BDE8F08100BF1020002090F84820F3
:1018C000531C0244DBB280F8483082F8341090F8A0
:1018D000492052B1132B0CD9002280F8482010B5B2
:1018E0000B4CD4F89C282AB910BD80F84820002B56
:1018F000F5D17047D4F89C28052AF5D11946343023
:10190000D4F8143AFFF796FFD4F8143A10BD00BF8C
:101910001020002010B50A4CD4F89C3803B910BD33
:10192000D4F89C38052BFAD1002A0846D4F8143A8A
:101930001146F4DDFFF77EFFD4F8143A10BD00BF66
:101940001020002090F848100023A0F8483001B97A
:10195000704710B5084CD4F89C381BB1D4F89C38AB
:10196000052B00D010BD3430D4F8143AFFF762FFD5
:10197000D4F8143A10BD00BF102000202DE9F04724
:10198000534E1F4606EB80039C68002C00F09B80A2
:1019900004F13E03A36104F59F73E3614FF4807388
:1019A000C4E904332836236866600546E16094F88C
:1019B0003D00A36391460BF06BFC804694F8440213
:1019C00094F83CA0261D002851D194F8450250BB44
:1019D000D4F840326BBB3A0731D419F0020F49D129
:1019E00019F0010F5AD1D4F8483294F9471294F8FB
:1019F00047221B010029DBB20DDB3649881880F82D
:101A000000335009012302F01F02934041F82030B7
:101A10003046BDE8F087304902F00F0211443046ED
:101A20000B76BDE8F08777F0A1FBD4F84032002BAD
:101A3000D1D02A4A116B0B4313633A07CDD5013538
:101A4000EDB2B8F1000F05D040F2067388F80850E7
:101A5000A8F80630FB0694F846222FD417F0200F82
:101A60000CBF3221122140460BF0D6FBBBE777F0CA
:101A70007DFBAAE76B1CDBB2B8F1000F05D088F83C
:101A8000083040F20653A8F8063094F84622404643
:101A900002210BF0C1FB19F0010FA4D050460BF04E
:101AA000F7FB0135EDB218B140F20663C380057251
:101AB00094F8462202210BF0AFFB94E70221404646
:101AC0000BF0AAFB8FE726463046BDE8F08700BF43
:101AD0000853080800E100E0FCEC00E00038024098
:101AE0002DE9F047038A8489A4B21C4082B047D014
:101AF000814688464FF0004501F14C0701F134065C
:101B0000B4FA84F325FA03F2D24391B2A9F8101083
:101B100014401B3BB8F1000F5FD0042B2ED8DFE838
:101B200003F052483D320300D8F80C30D9F82CA00D
:101B300033B19B6823B11FFA8AF108F1040098477A
:101B4000D8F8243033B19B6823B11FFA8AF108F129
:101B50001C009847D8F83C3033B19B6823B11FFA7A
:101B60008AF108F134009847D8F8543033B19B68B3
:101B700023B11FFA8AF108F14C009847002CBFD11D
:101B800002B0BDE8F087D8F80C30D9F834105B68A3
:101B900008F104009847002CB2D1F1E7D8F82430BE
:101BA000D9F838105B6808F11C009847002CA7D1C1
:101BB000E6E7D8F83C30D9F83C105B6830469847E7
:101BC000002C9DD1DCE7D8F85430D9F840105B6880
:101BD00038469847002C93D1D2E7042B07D8DFE88A
:101BE00003F01903140F0A00D9F83C300193019B4C
:101BF000002C85D1C4E7D9F82C300193019BF7E77D
:101C0000D9F834300193019BF2E7D9F838300193C9
:101C1000019BEDE7D9F840300193019BE8E700BF55
:101C2000F8B5264C94F86C2D012A034603D0022AFD
:101C300009D00020F8BD224ED6F880548DB984F822
:101C40006C5D0020F8BD002540F20112C0E954553A
:101C5000C0E95655A0F8442100F5A2717AF02EFB98
:101C6000EDE7402D20D94027D4F8741D154AC3F85C
:101C700058710A44C3E9542240F20112A3F84421E6
:101C80000022C3F85C2103F5A27118467AF016FB16
:101C9000D4F8743D3B44ED1BC3F30A03C4F8743D10
:101CA000C6F880540020F8BDAAB2402A01D02F46C1
:101CB000DAE7022284F86C2DD5E700BF102000205F
:101CC00008310020882D002001EB810138B500EBA0
:101CD000C1010F4DB1F88C1304462846FFF704F8F4
:101CE000E378C4F8A853012083424FF000024FF07C
:101CF0004001C4E9EC12A4F89C0304F56771204686
:101D000008BFC4F8AC537AF0D9FA002038BD00BF40
:101D10008C350020F8B52A4CD4F8C4340F2B04D0ED
:101D20005A1CC4F8C4240020F8BD264D95F86C3D1B
:101D30000022C4F8C424002BF5D1D5F8742DD5F8B1
:101D4000703D9A42EFD0D5F8742DD5F8703D9A4287
:101D50002DD8D5F8706DD5F8743DF61A402E2BD8D5
:101D6000B3B2402B13BF3746402702230123D5F8D7
:101D7000742D85F86C3D144BC0F858711344C0E9BC
:101D8000543340F20113A0F844310023C0F85C3111
:101D900000F5A2717AF092FAD5F8743D3B44F61B37
:101DA000C3F30A03C5F8743DC4F88064BBE7D5F8F3
:101DB000746DC6F50066D1E701234027D7E700BF61
:101DC0000831002010200020882D002010B5324B53
:101DD00093F8D42493F8E8C4D3F8D034044613B16C
:101DE00052EA0C0231D00123E06984F8463140F216
:101DF0000112A4F8442102682849002AA8BFC2F3AE
:101E000080739B0301EA124143F020030B4363F309
:101E10001F42BCF1020F026000D010BDE278204BDF
:101E2000C4F8A8331F200021C4E9EC01012A4FF0B7
:101E30000101A4F89C1308BFC4F8AC3304F5677122
:101E40002046BDE810407AF039BA01217AF000F955
:101E50000122E06984F8462140F20113A4F84431DC
:101E6000016800290A460CDBC1F380730B4C9B030D
:101E700043F0200304EA11410B4363F31F42026065
:101E800010BD064B03EA114343F4804343F02003A3
:101E900063F31F42026010BD08310020DFBFFFFF67
:101EA000D03500202DE9F041B0F8CC15D0F8CE3572
:101EB000B0F8D255B0F8D085C0F84051012284B0B6
:101EC00080F8112101F01F02012A044600F2CC56CD
:101ED000ADF80810C1F3072ECDF80A30ADF80E505A
:101EE0004FEA134C51D0022A7746C9B29BB210D0A8
:101EF000002A55D1BEF1090F4BD8DFE81EF089004A
:101F0000AD004A00C8004A005C01DF004A0013012E
:101F1000330101F0600120295FFA8CF272D0012FA9
:101F200000F0B881032F00F0A181AFBB90F812310F
:101F3000022B00F0E381032B2BD11CF0800F40F02B
:101F4000E98102EB820200EBC20393F87623003AA8
:101F500018BF0122C24D02234FF48071C4E94E33F1
:101F600084F81131C4F83031A4F81C1105F59F63D1
:101F70000021C4F83411C4E94A3304F58E712046B7
:101F8000C5F8F8247AF038F906E090F81231032BFE
:101F90000ED020467AF024F8002004B0BDE8F0818D
:101FA00001F080017AF054F8002004B0BDE8F0811F
:101FB0005FFA8CFCBCF1010FEBD8D0F8E43502A934
:101FC0009B689847BDF80E30002BE5D1C4E94A3331
:101FD000C4E94C3304214FF4807284F81111A4F841
:101FE0001C2104F58E7120467AF006F9636D9D4A36
:101FF0001A61E278012ACFD15E614FF08022196820
:102000001A60C9E7D0F8E43502A99B689847C3E78E
:1020100090F81231023B012BBBD8914BD0F818211C
:102020000021C3F8F01412B10222C3F8F0248E4A42
:1020300002234FF480700021C4E94C31A4F81C0144
:10204000C4E94E33C4E94A2284F8113104F58E7193
:1020500020467AF0D1F89FE790F81221023A012A3F
:1020600097D8012B98D1D0F8E43500259B68C0F8AB
:10207000185102A9984704224FF48073C4E94A55C5
:10208000C4E94C5584F81121A4F81C31A9E7012BAF
:1020900000F03B81022B7FF47FAF5FFA8CF3002BC3
:1020A0007FF47AAF03694FEA1C22023A5B68032A85
:1020B00000F2BD81DFE802F0B6CED2D01E0A022EB9
:1020C000ADF8065000F08A81032E00F04E81012EFB
:1020D0007FF45FAFD0F8EC3580781B680DF1060116
:1020E0009847BDF80630002B3FF456AFBDF80E20E0
:1020F000002A3FF451AF934228BF13464FF4807239
:102100000221A4F81C210022C4E94A0084F811111C
:10211000C4E94E33C4E94C3204F58E7120467AF09E
:102120006BF839E7012D7FF434AF90F81231022BB0
:1021300000F00881032B7FF42CAF4FF4807200F580
:1021400088730221A0F81C21002280F81111C0E937
:102150004E55C0E94A33C0E94C5200F58E717AF011
:102160004BF819E7DDB23E4F012D87F8E9543FF6F1
:1021700010AF90F81231022B00F0D880032B7FF4BF
:1021800008AF002D00F0358190F81011012910D012
:10219000D0F8E4355B68984797F8E914D4F8E4354B
:1021A00084F810111B6820469847D4F8E8359B68DE
:1021B000984700230AE758EA05027FF4EAAE90F850
:1021C000121103293FF4E5AE03F07F0580F81451A6
:1021D0000069114663F30A1103681943042301607F
:1021E00084F811314FF48073C4E94A22C4E94C22C7
:1021F000A4F81C3104F58E71204679F0FDFF636D63
:10220000184A1A61E278012A06D0002D00F0FC80FD
:10221000022384F81231BFE65E614FF08022196814
:102220001A60F2E702210E4861F306130022C0F89B
:10223000F4340423C4E94A22C4E94C2284F811315D
:1022400001224FF4807304F58E7184F81621A4F8EE
:102250001C31C8E60321E6E70521E4E70421E2E7B3
:102260000831002018000860F835002090F812119D
:10227000022943D003297FF48CAE23B9510602D042
:10228000114679F0E5FED4F8E4359B6802A92046B2
:1022900098478EE790F8121102292FD003297FF476
:1022A00078AE002B7FF478AE12F07F0181D01CF065
:1022B000800F40F0AD8002EB820100EBC10181F89C
:1022C000763381F87533282381F8742303FB0203E6
:1022D00000EB820193F87723496D0B68023A012ADB
:1022E00023F400138CBFC3F30072012262F31C734A
:1022F000D4F8E4250B60936802A9C8E753063FF4BD
:102300004BAE114679F0A4FE46E6D0F8E425C0F8BD
:102310001831F0E702F07F0202EB820200EBC20309
:1023200093F81E21003A18BF012213E6002D3FF456
:10233000A2AE01210322D0F8E43580F8101180F814
:1023400012212FE73B4A80F811314FF480710023AE
:10235000A0F81C11C0E94E55C0E94A22C0E94C530F
:1023600000F58E7179F048FF16E6DBB2052B3FF6DB
:1023700010AEDFE803F02B231B130B03D0F8EC3572
:1023800080789B690DF106019847AAE6D0F8EC35F4
:1023900080785B690DF106019847A2E6D0F8EC352C
:1023A00080781B690DF1060198479AE6D0F8EC3564
:1023B0008078DB680DF10601984792E6D0F8EC359D
:1023C00080789B680DF1060198478AE6D0F8EC35D5
:1023D00080785B680DF10601984782E6D0F8E43515
:1023E00080789B6A0DF1060198474670C4F8F005A5
:1023F00077E60222D0F8E43580F8122180F81051F7
:102400005B682946984736E6012384F81231C3E514
:10241000282202FB010080F81C1104EB810180F8E6
:102420001E3180F81DE190F81F21896955E70121CF
:10243000F9E600BFF435002010B5044629B990F83C
:102440001121032A0DD0002010BDD0F8E4359B697E
:10245000002BF8D090F81221032AF4D198470020DD
:1024600010BDD0F890230B46D0F87C138A4219D9BE
:10247000521AC0F8902394F803C0D0F880038A421F
:1024800028BF0A46BCF1010F92B234D0C4E9E2235E
:1024900004F55D71C4F88003A4F87433204679F024
:1024A000ABFED0E7D0F8E4351B691BB190F81221E0
:1024B000032A1ED000234FF480720421C4E94A335A
:1024C000C4E94C3384F81111A4F81C2104F58E7171
:1024D000204679F091FE636D0D4A1A61E278012A77
:1024E000B1D104F2CC545C614FF0802219681A60BB
:1024F000A9E79847DEE70844C4E9E22304F55D71E3
:10250000C4F88003A4F87433C4F88403C6E700BF9A
:102510001800086038B5044649B990F81131022B0B
:1025200011D094F81631012B39D0002038BDD0F8E5
:10253000E4355B69002BF8D090F81221032AF4D11E
:102540009847002038BDD0F83831D0F82421934284
:102550002FD990F803C09B1ABCF1010F0D46C0F8AB
:102560003831D0F828116ED09BB2C0F830314FF41A
:102570008073C0E94A11C0F8345100F58E71A0F89B
:102580001C3179F039FEC4E9E255C4F8805304F5F2
:102590005D71A4F87453204679F02EFEC1E73F4BDD
:1025A0002269D3F8F4145160002384F81631002016
:1025B00038BDD0F83C31B3FBF2F502FB15350DBB4D
:1025C0009A421FD8D0F8402193421BD24FF4807317
:1025D000A0F81C3100F58E71C0E94A55C0E94C5590
:1025E00079F00AFEE378C4F84051012BC4E9E255C2
:1025F000C4F88053A4F8745308BFC4F8845304F596
:102600005D71C8E7D4F8E435DB681BB194F812219A
:10261000032A15D0E27800230521012A84F811113C
:10262000C4E9E233C4F88033A4F8743304F55D716F
:1026300024D0204679F0E0FD636D194A1A6170E7F5
:1026400020469847E6E79BB21144C0F830314FF47A
:102650008073C0E94A11C0F8345100F58E71A0F8BA
:102660001C3179F0C9FDC4E9E255C4F8805304F582
:102670005D71A4F87453C4F884538CE7C4F88433B0
:10268000204679F0B9FD636D0548186104F2CC521B
:102690005A614FF080211A68196042E70831002022
:1026A0001800086070B50B7813F060020D46044600
:1026B00024D0202A04D0204679F092FC022070BD5C
:1026C000CA8848781AB31B0640D5324E3146FEF709
:1026D000CFFAEB884FF480720221A4F81C2100226B
:1026E00084F81111C4E94E33C4E94A66C4E94C3296
:1026F00004F58E71204679F07FFD06E04B780A2BB9
:1027000010D00B2B08D0062BD5D0002070BD022294
:102710001144FEF7ADFAF8E78B78C3BB1E4AC2F846
:10272000FC34F2E7022180F811114FF48071A0F817
:102730001C111A490123C0E94A11C0E94E33C0E90E
:102740004C3200F58E7179F057FDDEE71449154BD8
:102750000860E078C3F8A028002103F6A40301284C
:102760004FF00305C4F88C13A4F87413C4E9E422F1
:1027700084F81151C4F88823C4F8803304F55D71DE
:1027800008BFC4F88433204679F036FDBDE779F000
:1027900027FCBAE7B42800200831002004360020C6
:1027A0000000002010200020002310B51946044628
:1027B000402279F0B7FC802120460023402279F0A6
:1027C000B1FCD4F8E835A078012284F812215B68C6
:1027D0009847002010BD00BF10B5022304464022D8
:1027E000812179F09FFC204602234022012179F0CB
:1027F00099FC204603230822822179F093FC104B98
:102800000222A3F84C20FEF71FFAE2780D4BC4F821
:10281000A8334021C4F8B013012A4FF000004FF054
:102820000101C4F8B403A4F89C13204604F56771B1
:1028300008BFC4F8AC3379F041FD002010BD00BFE3
:10284000000000208C35002030B5812183B0044683
:1028500079F038FC0121204679F034FC2A49002522
:102860000223402281F8185A2046812179F05AFC2F
:10287000012102234022204679F054FC234BD3F857
:10288000002583F8E8541268284690470095009A7E
:10289000E1681F4B42F010020092009A0A610A6937
:1028A0000092013B02D0009AD006F8D40023019395
:1028B000019B43F020030193019A154B012060F323
:1028C0008A120192019A0A610A690192013B02D0BF
:1028D000019A9206F8D4E2780E4BC4F8A8331F2070
:1028E0000021C4E9EC01012A4FF00101A4F89C1376
:1028F000204604F5677108BFC4F8AC3379F0DEFCFC
:10290000002003B030BD00BF10200020083100209F
:10291000410D0300D03500202DE9F843374F8046A4
:10292000894615461C4697F8E01904290BD008295A
:1029300007D1D7F8D839434505D0FEF705FA022864
:10294000F1D0012057E0012387F8C4393B6397F8A1
:102950009030C7F8CC490622022B294CC7F8C08911
:10296000C7F8C859C7F8BC9987F8E02918BF4FEADB
:1029700048280A2640F2FF554FF48B63A5630121D6
:10298000C4F808801820E360FDF7C8FC03464FF048
:10299000000C40F2774201213720A563D3B1A56333
:1029A000C4F808C0E260FDF7B9FC721EA56388B1E7
:1029B00012F0FF06E0D13E63FEF7D0FDD7F8C8491C
:1029C00034B1D7F8CC39D7F8C01932460120A04726
:1029D000032010E00121484676F040FB084B0949EE
:1029E00059624FF400729A62DA6A002142F0910251
:1029F000DA620846B962BDE8F88300BF1020002003
:102A0000002C014000E1F5052DE9F04F3F4E9946BD
:102A100096F8E03983B0042B01908846924609D09D
:102A2000082B03D0002003B0BDE8F08FFEF78CF92F
:102A30000228F7D196F890300122022BF26262D080
:102A4000019B4FEA432B324C0021404676F006FBB7
:102A50004FF400722F4B6362A262E36A40F2FF57A9
:102A600043F09303E362A763A2604FF48A62E260DB
:102A700001211020FDF752FC0A25A76340F25142C4
:102A8000A7630121C4F808B01120E260FDF746FCFD
:102A900002464FF0000E40F2774301213720A76332
:102AA000DAB1A763C4F808E0E360FDF737FC013D45
:102AB000A76390B115F0FF05E0D1F562B062FEF7B3
:102AC0004DFDD6F8C849002CACD0D6F8CC39D6F894
:102AD000C0192A462846A047A4E7052386F8E0390E
:102AE0000023B362019AD6F8143AC6F8BC890120D3
:102AF000C6F8C029C6F8C8A9C6F8CC99C6F8D03916
:102B000003B0BDE8F08FDDF804B09CE71020002092
:102B1000002C014000E1F5051049114BD1F8882047
:102B200042F4700210B4C1F888201A680D4C0020DD
:102B300042F001021A6098601A6822F0847222F44E
:102B400080321A605C601A68074C22F480221A6096
:102B5000D8608C605DF8044B704700BF00ED00E06A
:102B6000003802401030002400000008704700BF09
:102B700082B00023414A01930093136843F48033E9
:102B8000136003E0019BB3F5A04F09D0136803F471
:102B900000330093019B01330193009B002BF1D084
:102BA000364B1B6813F4003318BF01230093009BBE
:102BB000012B01D000BFFDE7304B31491A6C314881
:102BC00042F080521A640A6842F440420A609A68ED
:102BD0009A609A6842F400429A609A6842F4A0525D
:102BE0009A6058601A6842F080721A601A689201FE
:102BF000FCD5254A40F205711160996821F0030166
:102C00009960996841F00201A2F580629960936829
:102C100003F00C03082BFAD1936803F00C03042B88
:102C200029D0082B0ED0194B1449194A8968194824
:102C3000C1F303110A4492F85C20D340C0F8D430A9
:102C400002B070475368516813F4800F536814BF83
:102C5000114A0E4AC3F3881301F03F01B2FBF1F2AF
:102C600002FB03F3054A5268C2F3014201325200EB
:102C7000B3FBF2F3D8E7084BD6E700BF00380240B9
:102C80000070004008544007003C02400024F4005B
:102C9000085308080000002000127A002DE9F843CC
:102CA00045697DB90768C7F30D0804460E46B8F1BB
:102CB000000F0AD0D6F80080FDF75EFE09283BD051
:102CC0006FF001052846BDE8F883514B9F422AD397
:102CD00003F580439F4224D303F580439F427FD373
:102CE0004C4B9F427FD903F580339F427ED903F539
:102CF00000339F427DD903F500339F427CD903F511
:102D000000339F4269D903F500339F4277D903F519
:102D100080239F4276D9B7F1016F76D305200EF05C
:102D20002FFA4FF00808FDF727FE092821D04FF0B1
:102D3000FF352846BDE8F883374E336923F44073E6
:102D40003361336943F400733361336943F0010342
:102D50003361C7F80080FDF70FFE3369092823F0BF
:102D600001033361ACD12368043323602846BDE8F6
:102D7000F883DFF8A490D9F8103023F44073C9F831
:102D80001030D9F8103043F40073C9F81030D9F876
:102D9000103023F0F803C9F81030D9F8103043EAA6
:102DA000080343F00203C9F81030D9F8103043F497
:102DB0008033C9F81030FDF7DFFDD9F8103023F06B
:102DC0000203C9F81030D9F81030092823F0F803AD
:102DD000C9F810303FF46EAFA9E74FF03808A2E70A
:102DE0004FF010089FE74FF018089CE74FF02008BD
:102DF00099E74FF0280896E74FF0300893E74FF037
:102E0000400890E74FF048088DE74FF058088AE7F0
:102E100000400008FFFF0008003C02400148FDF7A9
:102E2000F7B900BFDC0000200148FDF7F1B900BF91
:102E3000280300200148FDF7EBB900BF740500200E
:102E40000148FDF7E5B900BFC00700202DE9F041BA
:102E50000268214D0746002455F834309A4209D0C3
:102E600001340E2CF8D11D4A0021052005F0DAFBB3
:102E7000002013E01A4B03EB8408D8F804657EB1F8
:102E8000797901EB410306EBC30300221820C3E963
:102E9000032200FB01609F601A750430BDE8F081D9
:102EA00007216C2005F044FC0146C8F8040568B110
:102EB00031466C2281F0FAF8D8F8046505EBC405B8
:102EC000C6E90056F6617663F664D9E7054A05203F
:102ED00005F0A8FBCCE700BF745308082CFB0808DA
:102EE0000831002054FB0808704700BF38B5D0E90E
:102EF000004007EE902A0068324A334B2468D3F82A
:102F0000D4302468013990428DB210D002F580622D
:102F100090420CD002F57052904208D002F58062C7
:102F2000904204D002F58062904218BF5B0807EE21
:102F3000103AF8EE677AB8EE477ADFED246A87EE4A
:102F4000270A30EE260A7CF013F81E492388421E19
:102F50008C4292B29BB21AD01D498C4217D0B4F168
:102F6000804F1FD0A1F580318C421BD001F58061CC
:102F70008C4217D001F580618C4213D015498C42E8
:102F800019D123800123E5622285A38238BD23F471
:102F90005C739BB223800023E56222852386012394
:102FA000A38238BD23F45C739BB223800123E562C6
:102FB0002285A38238BD08498C42E2D023F44073B5
:102FC0009BB2DEE700000140000000200AD7233C4E
:102FD00000040140001000400014004070B5426839
:102FE000937903F0020E13F004033AD175469C4620
:102FF0009E464FF4807001235479032C30D8DFE8CB
:1030000004F08E6202361468704E228C22F48072B4
:103010001204120C2284228C22F4007212042B431C
:10302000120CA58842EA0322A38B23F073031B042E
:103030001B0CB442ADB243F0600300F09B8006F578
:103040008066B44200F09680A580A383E163228469
:10305000A38B23F008031B041B0C43F00803A3837A
:1030600070BD002005464FF0040C0346C4E712680B
:10307000564E148C24F480542404240C1484148C90
:1030800024F4005424042B43240C958844EA03348C
:10309000938B23F4E6431B041B0CB242ADB243F402
:1030A000C04375D006F58066B24271D09580938397
:1030B00011641484938B23F400631B041B0C43F4EE
:1030C0000063938370BD1468404E228C22F010027E
:1030D0001204120C2284228C22F0200212042B43B0
:1030E000120CA58842EA0312238B23F4E6431B0447
:1030F0001B0CB442ADB243F4C04359D006F5806610
:10310000B44255D0A5802383A1632284238B23F46A
:1031100000631B041B0C43F40063238370BD12681F
:10312000148C24F001042404240C1484148C968838
:1031300024F0020424042B43240C1C43138B234D42
:1031400023F073031B041B0CAA42B6B243F06003C6
:1031500023D005F58065AA421FD096801383516362
:103160001484138B23F008031B041B0C43F0080387
:10317000138370BD22F4006242EA0E2222F48062C0
:1031800092B225F4405542EA0C2245EA00155BE76D
:1031900025F4804545EA801588E726F44076064305
:1031A0004FF6F370204040EA0E0040EA0C04D4E7EA
:1031B00022F0800242EA0E1222F0400292B225F47E
:1031C000406542EA0C1245EA80059BE70000014099
:1031D00042685379032B0FD8DFE803F00B08050290
:1031E00010684030704710683C30704710683830C5
:1031F000704710683430704700207047024B034816
:10320000D3F80415FEF76CBC083100200000014023
:1032100010B5064C0648D4F80415FEF761FCD4F846
:1032200024150448BDE81040FEF75ABC08310020C0
:10323000000001400040014010B5064C0648D4F89B
:103240000415FEF74DFCD4F828150448BDE81040DD
:10325000FEF746BC08310020000001400044014058
:1032600010B5064C0648D4F80415FEF739FCD4F81E
:103270002C150448BDE81040FEF732BC0831002090
:103280000000014000480140034B4FF08040D3F85C
:103290000815FEF725BC00BF08310020024B03488B
:1032A000D3F80C15FEF71CBC0831002000040040C8
:1032B000024B0348D3F81015FEF712BC083100206A
:1032C00000080040024B0348D3F81415FEF708BC71
:1032D00008310020000C0040024B0348D3F82015B1
:1032E000FEF7FEBB083100200004014010B5064C7B
:1032F0000648D4F82015FEF7F3FBD4F8301504483F
:10330000BDE81040FEF7ECBB08310020000401408E
:103310000018004010B5064C0648D4F82015FEF7FA
:10332000DFFBD4F834150448BDE81040FEF7D8BBE5
:103330000831002000040140001C004010B5064C7C
:103340000648D4F82015FEF7CBFBD4F8381504480E
:10335000BDE81040FEF7C4BB083100200004014066
:10336000002000400348D0F8143A13B100F60820BA
:1033700018477047000000200348D0F8343A13B1D2
:1033800000F6282018477047000000200348D0F8B6
:10339000543A13B100F64820184770470000002047
:1033A0000348D0F8743A13B100F668201847704704
:1033B000000000200348D0F8943A13B100F68820AA
:1033C00018477047000000200348D0F8B43A13B102
:1033D00000F6A82018477047000000200348D0F8E6
:1033E000D43A13B100F6C8201847704700000020F7
:1033F0000348D0F8F43A13B100F6E82018477047B4
:10340000000000200348D0F8143B13B100F6083048
:1034100018477047000000200348D0F8343B13B130
:1034200000F6283018477047000000200348D0F805
:10343000543B13B100F64830184770470000002095
:103440000348D0F8743B13B100F668301847704752
:10345000000000200348D0F8943B13B100F68830F8
:1034600018477047000000200348D0F8B43B13B160
:1034700000F6A83018477047000000200348D0F835
:10348000D43B13B100F6C830184770470000002045
:103490000348D0F8F43B13B100F6E8301847704702
:1034A0000000002030B44568144CA542144D2C6B2C
:1034B0000CBF44F4001444F480042C6390F914C04D
:1034C000C1601201BCF1000F8361D2B20FDB0D4964
:1034D00001EB0C034FEA5C1083F800230CF01F0C87
:1034E000012303FA0CF330BC41F820307047064B3F
:1034F0000CF00F0C63441A7630BC70470060024039
:103500000038024000E100E0FCEC00E02DE9F84367
:10351000A848002242F2043C510143588CEA0303BC
:1035200013F47C540AD00132102AF5D1A24D0023A5
:10353000C5F8103A85F8E039BDE8F88301449E4D9E
:103540000B7FC5F8101A002BF1D18F689B4B9F425F
:1035500002D048339F42EAD1994A536A43F4006348
:1035600053620DF0B1FD064688460DF0ADFD801B9F
:1035700061EB0801B0F57A7F71F10001F5D3904A53
:10358000536A23F4006353620DF09EFD064688469D
:103590000DF09AFD801B61EB0801B0F57A7F71F1A7
:1035A0000001F5D3DFF818828648D8F8443043F498
:1035B0000063C8F84430D8F8303043F48003C8F8CA
:1035C0003030D8F8303043F00C03C8F830304FF0CA
:1035D0000D0900260C220E21A5F8029D85F8046D28
:1035E00009F01AFE7848A5F80E9D0C220E2185F8E8
:1035F000106D09F011FE7548A5F81A9D0C220E21D8
:1036000085F81C6D09F008FE7148A5F8269D0C226E
:103610000E2185F8286D09F0FFFD6E48A5F8329D52
:103620000C220E2185F8346D09F0F6FD0C226A4853
:10363000A5F8629D0E2185F8646D09F0EDFD674BDC
:10364000302283F831234FF400325A60D8F83030FA
:10365000634A43F48003C8F83030584BC2F83C75D5
:103660009F425BD05F4A6049C2F8A060C2F8A810D0
:103670004FF47411D1605D49C2F8A0100721C2F85F
:10368000B4104C4A5A4F33461046114605E00133F8
:10369000102B01F1200100F089808E68BE42F6D126
:1036A000544901EB43115B01D1F80C6A52498E4237
:1036B0006DD0434E316B41F48001316303440D21E1
:1036C00099834B4993688B4225D00134102C02F129
:1036D0002002F7D10020494900230122FFF7E2FE32
:1036E000D5F80C3A4BB119689A880B691A4204D183
:1036F000002385F8E039BDE8F883FDF78FFD002849
:10370000F6D1D5F8142AC5F8D029012385F8E03977
:1037100085F8D40910E700EB4410DCE73149324862
:103720008E65244A0866334630484FF074668E60D2
:1037300088650720C8661046114604E00133102B47
:1037400001F1200132D08E68BE42F7D1294901EB48
:1037500043115B01D1F80C6A27498E4220D0184EE4
:10376000316B41F48001316303440D219983134986
:1037700093688B4211D00134102C02F12002F7D152
:1037800000201F4900230122FFF78CFEA8E70C4E02
:10379000316B41F40011316390E700EB4410F0E726
:1037A000074E316B41F400113163DDE700235B68A4
:1037B000FFDE00BF080A00201020002058640240ED
:1037C000003802400C2D0020182D0020242D002050
:1037D000302D00203C2D00206C2D002000E100E069
:1037E0000831002000640240802C01406054A3088E
:1037F000A064024000000020006002408D08000824
:10380000C507000870B52D4C636BD9051ED54FF464
:10381000807340F2FF56A363A663E36B284D23F445
:10382000414323F03A03E3636B6B9A071FD40122F1
:1038300000236A62AB62214A40F2FF539363D36B69
:1038400023F4414323F03A03D36370BD636B9807BD
:1038500003D51B4B02229A62EDE7636B190721D453
:10386000636B9A0622D5164B06229A62E3E7154B44
:10387000D3F83C25136823F001031360E36A0022A8
:1038800023F00803E3622A636B6BDB07CFD540F2BA
:103890004C43A6630121A2600C20E360FCF73EFDCF
:1038A000A663C4E7064B04229A62C4E7636BDB0697
:1038B000C1D5034B05229A62BDE700BF002C014031
:1038C000102000200831002002683649002310B47F
:1038D00022F0010221248842026003604360836079
:1038E000C3600361446138D02F4B98422ED02F4BD8
:1038F00098423CD02E4B984240D02E4B984232D02A
:103900002D4B984241D02D4B984246D02C4B98429B
:1039100017D02C4B98423CD02B4B984216D02B4BB7
:10392000984224D02A4B984228D02A4B98421AD049
:10393000294B984229D0294B98422ED0284B9842A7
:1039400008D14FF03D5243F8AC2C03E04FF47462C1
:1039500043F8202C5DF8044B7047224B5DF8044B74
:103960003D229A607047204A43F8642CF2E74FF4F6
:1039700074125DF8044B43F8382C70474FF07462B2
:103980005DF8044B43F8502C7047184A43F87C2CE0
:10399000E0E73D2243F8082CDCE7154A43F8942C75
:1039A000D8E700BF1060024028600240406002403B
:1039B000586002407060024088600240A06002408F
:1039C000B860024010640240286402404064024033
:1039D000586402407064024088640240A06402405F
:1039E000B8640240006002403D000020400F00200B
:1039F00000003D20214A936803F00C03042B10B40F
:103A00003AD0082B1FD01E4B1C4C0360A1681D4AE6
:103A1000C1F30311114491F8DC10CB404360A1685D
:103A2000C1F38221114491F8DC1023FA01F1816085
:103A3000A1685DF8044BC1F342310A4492F8DC20DE
:103A4000D340C36070475368516813F4800F5368C4
:103A500014BF0D4A0A4AC3F3881301F03F01B2FBB9
:103A6000F1F202FB03F3054A5268C2F3014201324C
:103A70005200B3FBF2F3C7E7034BC5E7003802403F
:103A80000024F4000853080800127A0070B5446B53
:103A90008668A38923F400531B041B0CA38185793A
:103AA00090F805C02B0303F40051C5F380000CF01F
:103AB00001032A029B001CF0020F4FEA003002F4BF
:103AC000806218BF43F0080302431A43238A9BB263
:103AD00023F440530B432382A38923F4B05323F0F0
:103AE0000C031B041B0C1343A381A38A23F4407310
:103AF0001B041B0C84B0A3826846FFF77BFF234B9B
:103B00009C4205D003F580639C4201D0029B00E0FB
:103B1000039BA2891E49120403EB83034CBF76006A
:103B2000B60003EB8303B3FBF6F3A1FB0302A0890A
:103B300052096426000406FB12334FEA02121CD419
:103B40001B013233A1FB0313C3F3431313439BB293
:103B500023812A07A38A0AD59BB243F00803A382D4
:103B6000A3899BB243F40053A38104B070BD23F03A
:103B700008031B041B0CA382F2E7DB003233A1FB1A
:103B80000313C3F342131343E1E700BF00100140E6
:103B90001F85EB512DE9F8431D462E4B9DF8206003
:103BA0009DF824909842884617463BD02A4B98426D
:103BB00040D02A4B984245D0294B984221D14B46C0
:103BC000324629460520FDF7D9FE04460023C4E904
:103BD0000B87C4E90733C4E909336671A56084F82B
:103BE00006902046FFF752FFF107626B12D4B3072D
:103BF0000BD493899BB243F4005393812046BDE8D4
:103C0000F88300242046BDE8F883D36843F080039E
:103C1000D360EEE74FF6DF731380D36843F02003E1
:103C2000D360E4E74B46324629460020FDF7A6FE66
:103C30000446CBE74B46324629460120FDF79EFE5F
:103C40000446C3E74B46324629460320FDF796FE5D
:103C50000446BBE70010014000440040004C004017
:103C600000140140816011E741710FE781710DE798
:103C70002DE9F043704F07EBC00985B005464FEAC8
:103C8000C00899F80C0C09F003FB064699F80D0CD6
:103C900009F0FEFA044699F80E0C75F067FA6B1CF1
:103CA000DBB21EB140F60C123372F2801CB12372EB
:103CB00040F60C23E380304604223A2109F0ACFAA6
:103CC000042220463A2109F0A7FA07EB08025B4BD1
:103CD000D2F8084C9C4200F08E80594B9C4200F078
:103CE0009580584B9C4200F09C80474497F80F3CCD
:103CF000022B32D0032B7CD05349544F012B08BFE9
:103D00000F46A6886846FFF775FE26F03F06029B21
:103D10004F4AB3FBF7F13604A2FB0323360C46EA05
:103D20009346A680228822F001021204120C2280FF
:103D30008AB2C1F30B019B0C09B942F001024FF4A6
:103D4000967101FB03F34349A1FB03139B09013364
:103D50009BB242F4004223841FE0A6886846FFF726
:103D600049FE26F03F06029A394B3604A3FB0213A4
:103D7000360C46EA9346A680218821F00101090409
:103D8000090C218034499209A1FB021292099B0C73
:103D90000133042A238438BF0422A28323882F4AB4
:103DA0009BB243F001032380238823F4816323F033
:103DB00002031B041B0C4FF4804143F480632380F7
:103DC0002181238823F080031B041B0C238023887C
:103DD0009BB202EB451243F0010323800121002333
:103DE00082F8405582F8411582F8423505B0BDE8A9
:103DF000F0831B4F85E703F5F2331A6A42F4001291
:103E00001A621A6A22F400121A626EE703F5F0339E
:103E10001A6A42F480021A621A6A22F480021A6252
:103E200063E703F5EE331A6A42F400021A621A6A73
:103E300022F400021A6258E70000002000540040FB
:103E400000580040005C0040009F2400804F12009A
:103E500083DE1B43D34D6210632D3E0508310020E5
:103E6000C02709002DE9F047924E90F900108046D6
:103E7000807806EBC1050138CC0090B0D5F8081C5D
:103E800014282DD8DFE810F04C0120011500550052
:103E90005F009E00A600C301B6017A0084003C02C8
:103EA0000402D701C000D0002F003700A301950104
:103EB0005401888A0C8B81B27F4841EA04418843CF
:103EC00000F02081D8E90201101A42F2107263EB6F
:103ED0000101904271F1000102D3152388F80230EC
:103EE00010B0BDE8F08798F813000882C8E90223F3
:103EF000122088F80200888A0C8B80B240EA0440C5
:103F00006E4C844300F0B28000200E900F90012090
:103F10000F910E900E99002900F017820F9914311D
:103F20000F910F9909684905CCD5142388F8023000
:103F3000D6E798F8110000F0FE000882C8E90223D5
:103F4000052088F80200888A0C8B80B240EA044081
:103F50005B4C844300F0A180002000900190012080
:103F6000019100900099002900F0FB810199143122
:103F70000191019909684F05D7D4A3E798F811007A
:103F800040F001000882C8E902230B2088F80200F3
:103F9000888A0C8B80B240EA04404A4C84436DD03E
:103FA00000200490059001200591049004990029B7
:103FB00000F0D181059914310591059909684D05E5
:103FC000B3D47FE798F813000882C8E902230720DA
:103FD00088F80200888A0C8B80B240EA0440374C93
:103FE00084435ED000200290039001200391029050
:103FF0000299002900F0C1810399143103910399BA
:1040000009684E0591D45DE7088820F480600004BB
:10401000000C088098F8110000F0FE000882C8E942
:104020000223102088F80200888A0C8B80B240EAB4
:104030000440234C844312D000200C900D900120AA
:104040000D910C900C99002900F091810D9914317B
:104050000D910D99096848053FF567AF32E798F86B
:104060001330FF2B06D198F810301BB1132388F8BA
:10407000023035E7112388F8023031E7D8F8140010
:10408000012800F08F81022800F04382098B0E2165
:10409000C8E9022388F8021022E7062388F80230D4
:1040A0001EE7D8F81400002800F06D81082388F876
:1040B000023015E700000020010003008400070023
:1040C0008200070002000300088820F4006000045A
:1040D000000C0880088880B240F48060088008885E
:1040E00080B240F480700880032088F80200888A3B
:1040F0000C8B81B2A94841EA04418843C8E90223F4
:104100007FF4EEAE98F81230002B40F0CE8198F894
:104110001330FF2B00F03F82042388F80230DFE6E3
:10412000098889053FF5CEAE002388F80230D7E62E
:10413000344494F80C0C09F0ABF8064694F80D0CD6
:1041400009F0A6F8964AB2F8A03501339BB2824630
:10415000A2F8A03516B13368B2881A83BAF1000FFD
:1041600004D0DAF80030BAF804201A83112130465E
:1041700009F02EF81121504609F02AF84FF00909EC
:1041800065272EB13368B28819690A4240F023814D
:10419000013F00F01D810CF097FF04460D460CF026
:1041A00093FF001B61EB0501052871F10001F6D3B7
:1041B000E7E7088880B240F4007008804FF6FF30CF
:1041C00088820121C8E9022388F8021088E6D8F81D
:1041D0001400002800F06D81D8F8184014F8016B25
:1041E0000E8201381225C8E90504C8E9022388F8BF
:1041F000025075E6888A0C8B81B2684841EA044116
:1042000088437FF45FAE0A2388F8023068E60888A6
:1042100080B240F480700880092088F80200888A03
:104220000C8B81B25D4841EA04418843C8E902230E
:104230007FF456AEE7E7002401250A940B940B9116
:104240000A950A98002800F047810B9814300B90CB
:104250000B98006846077FF535AED8F814000328A0
:1042600000F06D81022800F24381088820F480600C
:104270000004000C0880088880B240F400700880B8
:10428000098A88F81C40C8E9022388F8025027E60A
:1042900000200124089009900991089408980028AA
:1042A00000F01481099814300990099800684707B4
:1042B0007FF508AEEFF31185102080F3128808888F
:1042C00080B240F400700880D8F818000E8A471CAD
:1042D000C8F81870EDB2067085F311880D8AD8F809
:1042E00018106FF001004E1CC8F818600D70C8E976
:1042F0000223C8F8140088F81C4088F80240EFE553
:10430000002006900790012007910690069C002C43
:1043100000F0E880079C14340794079C2468640626
:104320007FF5D0AD0C8AD8F818104D1CC8F818507D
:104330000C70D8F8141088F81C000139C8E9022361
:10434000C8F8141088F80200CAE50F9918310F91C7
:104350000F990968B6E5059918310591059909681D
:10436000B0E501991831019101990968AAE50D9903
:1043700018310D910D990968A4E50399183103913D
:10438000039909689EE5088880B240F400700880AF
:104390000121C8E9022388F80210A1E50100030009
:1043A00008310020088820F480600004000C088098
:1043B000EFF31184102080F31288088B088880B2F4
:1043C00040F40070E4B2088084F311880C215FE6A9
:1043D00016B13368B2885A830CF076FE04460D4657
:1043E0000CF072FE001B61EB0501052871F1000164
:1043F000F6D316B13368B2881A830CF065FE044612
:104400000D460CF061FE001B61EB0501052871F102
:104410000001F6D3B9F101097FF4B2AE16B13368E9
:10442000B2885A830CF050FE04460D460CF04CFE48
:10443000001B61EB0501052871F10001F6D3BAF10B
:10444000000F04D0DAF80030BAF804205A830CF0D8
:104450003BFE04460D460CF037FE001B61EB0501E8
:10446000052871F10001F6D316B13368B2881A83BA
:104470000CF02AFE04460D460CF026FE001B61EBF4
:104480000501052871F10001F6D3BAF1000F04D03F
:10449000DAF80030BAF804201A8398F90000441CB6
:1044A0003FF442AEFFF7E4FB3EE60F2388F802300C
:1044B00016E5088880B240F4007008800121C8E940
:1044C000022388F81C1088F8021009E509991831B0
:1044D000099109990968F5E40B9918310B910B9929
:1044E0000968EFE407991831079107990968E9E429
:1044F000D8F81800098A441CC8F818400170D8F888
:104500001410C8F808200139C8F81410C8F80C3085
:10451000E6E4088880B240F400600880EFF311847C
:10452000102080F31288088B088820F48060000433
:10453000000CE4B2088084F311880D21A8E50888F6
:1045400020F480600004000C0880EFF31184102038
:1045500080F31288D8F818000D8A461CC8F8186035
:104560000570088880B240F40070E4B2088084F3DB
:104570001188D8F81800098A441CC8F8184001703E
:10458000D8F814100C200239C8E90223C8F8141016
:1045900088F80200A4E498F81030002B3FF4BCAD7A
:1045A00031E600BF38B5184D9DF814E005EB401416
:1045B0004FEA401C94F8410500B938BD490084F821
:1045C0005325C4F8543584F851150023049984F810
:1045D00050E5022205F5A86584F85235C4F858154F
:1045E00084F85C3584F8422565440CF06DFD024684
:1045F0000B462846FFF736FC94F84235002BF4D1E1
:1046000094F85C0538BD00BF0831002038B5184D5E
:104610009DF814E005EB40144FEA401C94F8410566
:1046200000B938BD84F85325C4F85435012200235D
:10463000490005F5A86584F8522584F85C35049A8C
:1046400084F850E5022384F85115C4F8582584F8FD
:10465000423565440CF038FD02460B462846FFF70C
:1046600001FC94F84235002BF4D194F85C0538BD78
:104670000831002082B0064B002201920193019B79
:1046800003EB80030193019B196002B0704700BFE8
:104690005028004010B51C2008F0FAFD11210446F6
:1046A00008F096FD4CB12368A2885A83C8200CF00C
:1046B00039FD2368A2881A8310BDBDE81040C820C8
:1046C0000CF030BD704700BF704700BF704700BF9F
:1046D00010B5104C94F8AE3523B90F4B4FF480222F
:1046E0005A6110BD4FF0E022D2F8103D23F00603CE
:1046F000C2F8103DFEF710FAD4F8B4359B68DB071A
:10470000EBD5D4F8B026136823F0030161F3070357
:104710001360E2E708310020003C01402DE9F04F32
:10472000A34CD4F8B0355A69D5078BB002D50BB07D
:10473000BDE8F08F5A699B6912EA0301F7D0C1F313
:1047400007430803019300F1E180019B5D073FD41B
:104750008807CEB203D5D4F8B03502225A610029B9
:10476000C0F24A820A05C1F3072500F19981370793
:1047700008D5904B9048D3F82C3C9847D4F8B035E6
:1047800008225A61F60600F10F82E80600F1BE81A8
:10479000A80600F11781019BDA0609D5854B8648EA
:1047A000D3F83C3C9847D4F8B0354FF480125A61A6
:1047B000019B9B06BBD57F4B7F48D3F8403C984775
:1047C000D4F8B0354FF400125A610BB0BDE8F08F49
:1047D000D4F8B4359E69DB691E40B6B2002EB7D05E
:1047E000754D4FF0000B05F118080F46F00740F12A
:1047F0008280D4F8B415D8F8002008694B6B23FAEE
:104800000BF3DB01DBB203439068034013F00109B3
:10481000D8B200F00F824B6B012000FA0BF023EAB4
:1048200000034B6301239360624B6348D3F8243C3D
:104830005FFA8BF1984794F8A735012B00F07E8240
:1048400019F0800F57D0D5E94CC1D5F82431D8F8EC
:1048500000E0ACEB01029342DEF8180028BF1346DB
:1048600080B20333B0EB930F45D9D4F8B43594F844
:10487000A795CDE9026BBA4667469C46B94237D246
:10488000D5F82431781A984228BF184600F1030B56
:10489000D5F828314FEA9B0BB9F1000F10D182B245
:1048A00003329210D8F8B8600AD04946013153F863
:1048B000047B37608A42F9D1D5E94C71D5F82831AB
:1048C000014403448F42C5F82831C5F83411DEF89D
:1048D00018300AD195F81C01012202FA00F0DCF828
:1048E000342022EA0002CCF834209BB29B45C5D389
:1048F000DDE9026B574676080BF1010B05F128053F
:1049000008F104087FF472AF394621E7D4F8B435D2
:104910009D69DB691D402D0C3FF417AF04F2A458CC
:10492000DFF890B0029104F5BF6600274FF001094F
:10493000C24608E06D0807F1010706F1040608F118
:10494000280800F09181EA07F4D53068D4F8B4154E
:10495000836849690B40D9B2DB0740F1708194F854
:10496000A735C0F80890012B07D10169D8F87C332E
:10497000C1F312015B1AC8F88C33DBF8203CF9B2A2
:104980005046984794F8A735012BD3D1002FD1D1A9
:1049900094F8B536052BCDD1D4F8F835074919610F
:1049A0000749596119684FF080211960C2E700BFBB
:1049B0000831002000000020AC36002018000860FC
:1049C000783C0020D4F8B455D4F8BC25AB68C3F3C8
:1049D0004103022B136814BF0021032161F30A0372
:1049E00013606B6843F4807306A86B60FFF702F8EE
:1049F000D4F8B025079ED36823F47053D360A86819
:104A000010F0060FC0F3410100F03C819F49A0481F
:104A10003144814240F2AE819E48A6F57401A1F571
:104A20001051814240F2AA819B499C483144814205
:104A3000C0F0A8819A48A6F18C71A1F5434181424A
:104A400040F2A4819749984831448142C0F0A28144
:104A50009649974831448142C0F0A0819548A6F11B
:104A6000B771A1F558518142C0F0A0819249934895
:104A700031448142C0F09681914892493044884245
:104A800034BF062005204025012160F38D23D3602B
:104A90004FF4005384F8A615A4F8A85553617AE69C
:104AA00000238DF8133094F8B6368DF81330864B0A
:104AB0008648D3F8343C9847D4F8B435D4F8B025B8
:104AC000986894F8AE354FF400615161002B3FF4C3
:104AD0004EAEC3077FF54BAE94F8B936012B7FF489
:104AE00046AE9DF81330032B7FF441AED4F8B036B8
:104AF00077491A6842F001021A601A6842F003020C
:104B00001A600B6943F006030B6130E6D4F8B46514
:104B1000D4F8B0157368002723F00103736005977C
:104B2000059B43F020030593059B67F38A130593C8
:104B3000059B0B61674BBC460A690592013B02D09D
:104B4000059A9206F8D494F8A52552B1624B03EB6E
:104B5000820EFF2253F8040F8260D86B7345826087
:104B6000F8D10B2363F3070763F3070C4FF0FF3310
:104B7000B3614FF00113F3617761C6F810C0336879
:104B8000564823F4FE63336094F8A725D4F8F8352B
:104B9000012A18616FD04FF480534B614A4B4B4848
:104BA000D3F8303C9847F3E5D4F8B0359A6922F051
:104BB00010029A611A6AC2F34340022802F00F0100
:104BC00000F09080062812D101EB810104EBC101B5
:104BD000D4F87466D1F83009C2F30A12104432686E
:104BE000C4F8702B3268C4F8742BC1F830099A6984
:104BF00042F010029A61C8E594F8AE353BB1D4F8A2
:104C0000B026136823F0030060F307031360D4F8A1
:104C1000B4252D4B2D48D3F8385C5368029123F00E
:104C200001035360A847D4F8B03502994FF0004211
:104C30005A6197E5010707D5082393605BE68A0769
:104C400007D50223836075E6C3060FD51023936052
:104C500051E60B077FF56EAEDBF8283C50469847CF
:104C600033680821996065E602996EE5410679D5B9
:104C7000402393603FE61A4A5A611A684FF0802237
:104C80001A6088E74FF400750920FEE6401E1BFFFE
:104C90003F420F00DFC810002013FBFE20D6130098
:104CA000FF69180000D3CEFE40771B00C05BB3FE47
:104CB000C091210040AC2700C01D6AFE40E13300D6
:104CC000803C36FEE09C410000000020AC36002015
:104CD00000ED00E0410D0300C03600201800086020
:104CE000783C002047F6F070104280D0C2F30A12E0
:104CF00001EB810004EBC00002F1030C5FEAAC0C95
:104D0000D0F82469D4F874E64FEA810818BF00206F
:104D100006D00130DEF8007046F8047B8445F8D1F7
:104D2000414404EBC101D1F824091044C1F824091D
:104D3000D1F830091044C1F8300958E7BBF1000F31
:104D40007FF47EAD94F8B536042B7FF479ADD4F8BA
:104D5000F835184A1A61184A5A611A684FF08022C9
:104D60001A606DE5830758BF81467FF569AD022360
:104D70009360C0E5012140250E2086E601214025F3
:104D80000D2082E6012140250C207EE601214025F0
:104D90000B207AE6012140250A2076E601214025F4
:104DA000092072E60121402507206EE601214025F9
:104DB00008206AE618000860783C00200278436802
:104DC000022A11D00C490269D1F8180210B4184017
:104DD000D1F81042D1F80C12931E400A04FB0300D4
:104DE00008445DF8044B7047034AD2E9802102EB86
:104DF000410202EB53207047D85C00202DE9F04FB0
:104E000012F0020A884E83B09B4601D000286FD072
:104E1000D6F80852002D58D14FF0FF3C834C844FF8
:104E2000CDF804C0E046E646002300922268A57B48
:104E3000904200F09E80002D40D003F58179012D35
:104E400007EB09190AD199F80750EA0706D415F0BB
:104E50007E0F03D1ED0900F090809E460133082BB0
:104E600004F11004E2D1BCF1000F009A04DABEF1A3
:104E7000000FC0F29280F4466D4CD6F8983004EBE7
:104E80000C1741F2180E013347F80E0041F21C0EC8
:104E90000CF5817547F80E302F01C6F89830E351B4
:104EA00004EB051300275F6004EB05139B79042BCB
:104EB0007AD8DFE803F02940194043009C460133CB
:104EC000082B04F11004B1D1CDE7D6E9833404FBFB
:104ED00005339842A0D396F8B43113B9012386F86C
:104EE000B431534B01225A70002003B0BDE8F08F5B
:104EF00096F8B431A6F58054002B59D00123022036
:104F0000637003B0BDE8F08F12F0010776D104EBB7
:104F10000513D01093F807E0BBF1030F60F3C71E31
:104F200083F807E068D94FF6FF735B4528BF5B46FF
:104F300004EB05108380BAF1000F49D1500705D565
:104F400004EB0510C37943F00103C371D30608D500
:104F500004EB0515EB79C3F34502013262F3460316
:104F6000EB71344B012003EB4C230B6003B0BDE825
:104F7000F08F009A05BB9C467EE7A568019A954292
:104F800038BF984603F1010338BF2A46082B019227
:104F900004F110047FF44AAF65E7B8F1000FA8BF31
:104FA000C446BFF669AF9FE796F8B431002BA5D190
:104FB000012386F8B431A1E7D6F898701C4C03F5AC
:104FC00081759C462B010137E750C6F898706BE756
:104FD000D6F89830D6F89C0001330130C6F89830E6
:104FE000C6F89C0004EB0C1041F21C06835104EB44
:104FF000051304209871A1E73B4699E70E4BD3F8BF
:10500000683D002B3FF470AF0A495E680B4A01EB24
:105010004C210023B04700283FF466AF04EB051590
:105020000223AB7160E700BFD85C0020F05C002079
:10503000D84C0020F04C002010200020F90D000872
:1050400070B5104E3378022B0F4B0BBF020AC0F322
:10505000D412C4B200F07F04D3F8000282B010442E
:105060000D460023032201A9FFF7C8FE012807D13E
:105070003378019A022B0CBF22F8145042F82450C6
:1050800002B070BDD84C0020D85C00202DE9F04F54
:10509000DFF820910D4699F800102B68032985B0A0
:1050A000164640D0022966D14FEA132A5FFA83F8E8
:1050B0004FF4807B421E012A24D801249E421CD931
:1050C00001288CBF00220122394F0192D7F87821A4
:1050D0001AB1D7F89411994250D0D7F800020023A2
:1050E0005044092203A9FFF789FE012824D0022891
:1050F00015D020B12B689E42E8D82E60032005B061
:10510000BDE8F08FB8F1000F14D0294B93F8B4210B
:1051100012B9012283F8B421012389F80130022059
:1051200005B0BDE8F08F4FF0800BC3F3D41A03F045
:105130007F08BFE75C46C1E799F80010022916D046
:105140000329ECD1039B53F8282022F07042019BE5
:10515000D5F800C0B2FA82F252099A4220D0A04497
:105160000CEB0403D8452B601DD20229EAD1039B26
:1051700033F81820EBE74FF4807BD6E7D7F810120E
:10518000013A02EB41224902B2FBF1F21344B3FBB4
:10519000F4F204FB12320AB123449B1A2B60AAE7F3
:1051A0006645ACD8A9E70AF1010A4FF00008A2E76A
:1051B000D85C0020D84C00202DE9F04FDFF850914A
:1051C0000B6899F800C0174609F58052BCF1020F30
:1051D000D2F8005283B08B46824640F08180DEB226
:1051E000A6EB030805EB1325B8444FF480729044F6
:1051F000BB4208F1FF38B8FBF2F843D2A844BCF137
:10520000030F06EB0704A4EB030414BF4FF48072F2
:1052100080229442A8EB050328BF1446B6BB9442F3
:1052200034BF0B220A2201A92846FFF7E7FD012817
:1052300029D199F800C0DBF80000BCF1020F00F1A1
:10524000010325D0A64210D2019906F18042013A0D
:1052500001EB8202043901EB840142F8043F8A42E7
:1052600003F10103F9D1DBF80000A31B0344BAF1F9
:10527000010FCBF8003023D09F4205F101054FF01C
:105280000006BCD8012003B0BDE8F08F0B22CAE7AE
:10529000A642EAD2019906F10042013A01EB42022C
:1052A000023901EB440122F8023F8A4203F1010373
:1052B000F9D1A31B0344BAF1010FCBF80030DBD1C5
:1052C000BB42D9D1BCF1020F019B18D004F180443C
:1052D000013C4FF0FF3243F82420DBF80030CBE7ED
:1052E00003F07F06C3F3D412BCF1030FA6EB03084F
:1052F0001544B84414BF4FF48072802277E704F15C
:105300000044013C4FF6FF7223F814200120BAE755
:10531000D84C002030B50446C06983B010B90120D4
:1053200003B030BD0D460023032201A9FFF766FD3F
:105330000128F5D1B4F92020002A19DB019B012DA9
:105340004FEA421103EB421203D0022D1BD1E5209C
:105350005854A368D3612378032B04D10023137717
:1053600053779377D377636A53831B0C9382D6E783
:10537000064A92F8B41109B982F8B401044B01222B
:105380005A700220CCE7E368E4E700BFD85C002055
:10539000D84C00202DE9F043814683B00E4699F8A1
:1053A0003C30042B00F28980DFE803F02F03704FBC
:1053B0003F00434DDFF810814FF6F77705F5805435
:1053C00018E0BA4260D873F01FFE01284FF00001C8
:1053D00038D1D9F83000FFF733FE012832D1019AD5
:1053E000D4F81412C9F83020531E8B4228BF0B4644
:1053F000C4F814322A78D9F83030032A01A91846A3
:105400009AB2DED14345DED93EE0710001F0FE01E3
:105410004846FFF77FFF012843D1D9F83430002BED
:1054200018BF022089F83C00B9E799F82830042B0E
:1054300004BF002389F82830D9F838300BB148462A
:105440009847012003B0BDE8F0831E48D9F82C200E
:10545000D0F89431C0F894219B1AD0F8102202FBA6
:1054600003F3D0F8782102EB4322C0F87821D0F87A
:105470007C2102EB4322C0F87C21002100F5B870AA
:10548000FFF748FF01280CD10420CBE7D9F83420DE
:1054900009F130010020FFF78FFE012801D1032020
:1054A000C0E70228CED199F82830042B04BF00238E
:1054B00089F8283003B0BDE8F0830220F3E700BF8D
:1054C000D84C0020D85C0020F7FFFF0F38B5044609
:1054D00094F83430052B58D8DFE803F0372B231924
:1054E000100394F82830082B04BF002384F82830D8
:1054F000274B012283F8B521022038BD94F82830CB
:10550000082B04BF002384F82830012038BD002177
:105510002046FFF7FFFE012837D1042084F834002D
:10552000D6E7D4E90B01FFF78BFD01282DD103202D
:10553000F4E7206B4FF0FF31FFF782FD012824D103
:10554000E36A002BF3D00220E8E7114DD5F80822DA
:1055500004F1300101200232FFF798FD012805D047
:105560000238C0B2012810D80520D7E7E368D5F883
:105570001012226BC5F8142203EB4123C4E9033255
:10558000E36A002BCAD16262C8E7002038BD00BFC1
:10559000D85C002070B5044694F83830032B4BD803
:1055A000DFE803F01F170B0200212046FFF7B2FED1
:1055B000431EDBB2012B40D970BD626B04F1300198
:1055C0000120FFF7F9FD0128F2D1032384F83830D8
:1055D000E2E71F480021FFF79DFE0128E8D10223E2
:1055E000F4E71C4AE56802F580531278D3F81012EC
:1055F000D3F89401032A14BF4FF48072802202FB77
:1056000001F105EB4125C4E90350D3F87851A5EB2E
:105610004125C3F87851D3F87C51861AA5EB412176
:105620000244C3F89421C3F87C11E36AC4E90C0274
:105630005BB960620123C9E7022094F82830062B89
:1056400004BF002384F8283070BD2663F2E700BF52
:10565000485E0020D84C00202DE9F0434368C3F396
:1056600008020A44B2F5007F83B005460C4605D215
:1056700023446B60012003B0BDE8F08390F91A2049
:10568000501C0AD0464902F5817201EB0212D17911
:1056900021F00101D171FF22AA7695F91B20511C3E
:1056A00016D03F4E02F5817206EB021106EB021294
:1056B000C979D079C1F34501012986BF01F1FF31D4
:1056C00001F03F010021FF2661F34600D071EE7624
:1056D0002A78022ACCD0324E06F58058D8F810220B
:1056E000B4EB422F4FEA42292BDCD8F818721F4046
:1056F0007A42A24225DCE2194A45286913D32A7E60
:10570000120729D5D8F89421411C8A421BD300D115
:1057100000214B44DB1BA4EB0909686109EB07047A
:1057200029616B6008460028A4D03278032A31D062
:1057300080B24FF6F77290429CD81A4614446C60BF
:1057400098E7002097E798F8B42102BB012388F876
:10575000B43173706B68DCE701A973F055FC012864
:10576000EFD16B68297828696861A4EB0904994432
:10577000A9EB070301986B6002293C4428611A4693
:10578000D1D1D8F82012B3EB412FD7D372E7012241
:105790007270BEE7034A90423FF66CAFCDE700BFA0
:1057A000D84C0020F7FFFF0F2DE9F047044682B0E8
:1057B00094F83830032B00F2AB80DFE803F09A173F
:1057C0000C02236C002084F8280003B198470220C3
:1057D00002B0BDE8F087236C002284F828200BB1CA
:1057E00020469847012002B0BDE8F087237866681C
:1057F000484F022B1CBF474BD3F81832204618BF26
:105800001E40FFF7DBFAC6F34F26361A0546B6B23E
:10581000A7F5805811E0D7F810325A1E914557D29B
:10582000FFF71AFF40B997F8B43113B9012387F88D
:10583000B431012388F80130013506EB050C022252
:1058400001A9002328461FFA8CF9FFF7D7FA01288F
:105850004FF400724FF00001BAD101987EF026FC9F
:10586000E3694FF400712046002BD4D06368002B0D
:10587000D1D1019B4FF020324FF02E0C4FF0100E83
:10588000C3F80120C3F80520A3F8092083F800C05D
:1058900042F62E6AD4F824C0A3F820A083F80BE0C7
:1058A000C3F82220C3F8262083F82A20E26BA3F84D
:1058B0001AC05A872CFA0EFC22FA0EF283F82BE05B
:1058C0009A86A3F814C0D7F810325A1E9145A7D370
:1058D000C3EBC353590201F500712046FFF7BCFE2C
:1058E00028B997F8B4317BB10B4B01225A700220D2
:1058F00007E02046FFF7EAFD012802D0022807D181
:10590000032084F8380053E7012387F8B431EBE72C
:1059100000205DE7D85C0020D84C00202DE9F04144
:10592000B1F904300F2B82B00E460446174632D030
:105930002046FFF743FA94F91B80B8F1FF3F3BD0B4
:105940005C4B41F2180203EB08118A58904211D1C6
:10595000183303EB4825B38801331BB205EB43151D
:10596000B38020463D60FFF729FA3060012002B085
:10597000BDE8F08103F5805292F8B41100295CD0A3
:1059800001225A702378022B4CD02269002A60D160
:1059900000233B60EAE74FF40071FFF75DFE00284B
:1059A00047D04FF6FF73B3802046FFF707FA94F90C
:1059B0001B80B8F1FF3FC3D12378022B41D022696D
:1059C000002AE5D03B4B1B78032B69D093B24FF6EE
:1059D000F7718B4294BF00230123002BD6D138B935
:1059E000354B93F8B421002A4DD0324B01225A7026
:1059F0000023112201A9FFF701FA012810D1019D0E
:105A00002E4BEB1A48BF03F2FF13B3F5805F4FEA4A
:105A100063222DD24FFA82F884F81B80002D9AD190
:105A20002378B0E7244A6368D2F82022B3EB422FF0
:105A3000AED2002002B0BDE8F081012182F8B4119D
:105A40009EE71D4BD3F820226368B3EB422FC6D3E9
:105A50009EE7184B1B78032B19D093B24FF6F772C1
:105A6000934294BF00230123002B91D10020E1E752
:105A7000114B93F8B42112B9012283F8B4210D4BD4
:105A800001225A70C8E7012283F8B421ADE70C4B1C
:105A90009A4294BF00230123002B7FF479AFE5E7FE
:105AA000074B9A4294BF00230123002B7FF46EAF73
:105AB00095E700BFD84C0020D85C0020F04C0020B7
:105AC000F7FFFF0F2DE9F043044689B094F830301A
:105AD000042B11D8DFE803F0501361035A00237E32
:105AE0009A0640F1FA80E0690023112204A9FFF729
:105AF00085F9012800F0F18009B0BDE8F083C64DBA
:105B000003AE04F11C07324639462846FFF706FF6C
:105B1000012800F0FD800228EED1C04901F5805532
:105B200095F9D2315A1C0AD003F5817301EB0313A6
:105B3000DA7922F00102DA71FF2385F8D23195F982
:105B4000D3315F1C16D003F5817301EB031201EB17
:105B50000313D279D979C2F34502012A86BF02F133
:105B6000FF3202F03F02002262F34601FF22D971A8
:105B700085F8D321042306E0A74873F07BFB4FF69A
:105B8000FF720123228484F830309FE70020E36A0B
:105B9000207009B0BDE8F0431847A14D95F8E031F9
:105BA000002BA9D104F11C0703AE05F5DC783246C1
:105BB00039464046FFF7B2FE012840F01A81039BA8
:105BC000002B00F0F4801A78E52A01D0002AEED1EB
:105BD0009449591A48BF01F2FF11B1F5805F4FEAAD
:105BE000612280F050818D4912018F480244907BE0
:105BF00004280CD0D5F898000130C5F89800506002
:105C000004209073D5F89C200132C5F89C2095F9AA
:105C1000D221561C0AD002F5817201EB0212FF203C
:105C200085F8D201D07920F00100D07195F9D32107
:105C3000501C18D002F5817001EB001201EB00112D
:105C4000D279C2F34502012A4FF0FF0088BF02F16A
:105C5000FF3285F8D301C8798CBF02F03F020022E1
:105C600062F34600C8711846202200217EF01EFA19
:105C7000D4F83120D4F8351041600260B4F83920EE
:105C800094F83B1081720281627EC272019005A875
:105C900003F070F8019B002800F0DE809DF81600EC
:105CA0009DF817209DF8191042EA4012BDF8140023
:105CB000A0F2BC7042EA40229DF81A00490141EA74
:105CC00050019DF8180041EAC02192B288B2D981F2
:105CD0001A821A83D882032355E7204673F0CAFA42
:105CE0002369002B00F08A80237E03F0F70213F073
:105CF0000403227640F09A80122A00F0B080E36A12
:105D00000022204684F8282009B0BDE8F043184757
:105D1000DDF80C80B8F1000F00F0C18098F8003079
:105D2000002B00F0BC8098F80B9019F0080F7FF45E
:105D3000EAAE0B2204F1310140467DF011F8002853
:105D40007FF4E1AE637E89EA0303D90640F1E68081
:105D5000324901F5805595F9D2315A1C0AD003F524
:105D6000817301EB0313FF2285F8D221DA7960F306
:105D70000002DA7195F9D321571C3FF4FBAE02F50E
:105D8000817201EB021301EB0212DB79D179C3F3CB
:105D90004503012B86BF03F1FF3303F03F030023CC
:105DA00063F34601FF23D17185F8D331E2E695F81C
:105DB000B831022B4FF009023FF4DCAE95F8E03128
:105DC000002B7FF4D7AEC5E97D3385F8F03185F837
:105DD000EC31D5F8CC31C5F8E4310F48D5F81432A0
:105DE00085F8E021C5F8E831FFF7DEFC01283FF433
:105DF000DEAE02287FF480AE0423C4E6237E1B07B8
:105E00007FF57DAF064B93F89821002A7FF474AE9E
:105E1000072283F8982172E7905E0020D84C00207A
:105E2000D85C0020F04C0020F05C0020A568E66AF9
:105E3000002384F8283029462046FFF70DFC00286F
:105E400066D194F82830002B7FF456AE0223C4E9C3
:105E50000B6584F828304FE644F2817238E7626AB5
:105E6000E16AA163042084F828002046C4E90B22DB
:105E7000C4E9023384F83C306363636209B0BDE86F
:105E8000F04373F0F7B995F8B42112B9012285F8FF
:105E9000B421454901224A706FF00F02A5E642493C
:105EA00001F5805595F9D2315F1C0AD003F5817355
:105EB00001EB0313DA7922F00102DA71FF2385F88E
:105EC000D23195F9D3315E1C16D003F5817301EB05
:105ED000031201EB0313D279D979C2F34502012AE7
:105EE00086BF02F1FF3202F03F02002262F3460158
:105EF000FF22D97185F8D321237ED8067FF53AAEEB
:105F00002A4873F0B7F94FF6FF72022322843AE66B
:105F1000002E3FF4F1AD204633463AE6B8F814209F
:105F2000B8F81A30224D43EA02436362D5F81022D2
:105F3000D8F81C30A3605202B3FBF2F102FB11311E
:105F400009B113445B1AE36084F8199095F9D231D2
:105F500015495E1C0AD003F5817301EB0313DA794E
:105F600022F00102DA71FF2385F8D23195F9D321AD
:105F7000501C3FF4B0AE02F5817201EB021301EB4D
:105F80000212DB79D179C3F34503012B86BF03F1FC
:105F9000FF3303F03F03002363F34601FF23D17176
:105FA00085F8D33197E600BFD84C0020905E0020E2
:105FB000D85C002070B50378017E023B012B0446BB
:105FC00002D911F0060F68D18D0643D494F91A3026
:105FD000581C0AD0374A03F5817302EB0313FF20E4
:105FE000DA7922F00102DA71A07694F91B305A1C9A
:105FF00016D0304803F5817200EB021300EB02105B
:10600000DB79C279C3F34503012B86BF03F1FF336C
:1060100003F03F03002363F34602FF23C271E376DC
:106020000B070ED5244B93F89821072A06D093F836
:10603000B421002A38D01F4A01215170002283F870
:106040009821E26A0023237084F8283022B3BDE847
:106050007040104700231948E5691A01825895429B
:1060600006D00133082BB1D01A0182589542F8D1DD
:10607000104803F5817300EB0312D279C2F3450295
:10608000012A15D9013A02F03F0200EB0313D87937
:1060900062F34600D87199E770BD0121FFF73AF924
:1060A0000128F9D1217E8FE7012283F8B421C2E7CC
:1060B0000022EAE7D84C0020D85C0020F05C0020E9
:1060C00038B5184D05F58054014694F8E00120B923
:1060D00061B191F8283013B138BD002038BD04F506
:1060E000DC7044227CF0C0FE012038BD44220E4802
:1060F0007DF0DCFF2B78D4F81C12C4F8DC110322ED
:106100004FF6FF70022B18BF1346A4F8D20184F893
:10611000D021054884F8B831102284F8D12173F0D9
:10612000A9F8E1E7D84C0020905E00204FF0FF3C3A
:106130002DE9F041344A354D6446002304E0013333
:10614000082B02F1100216D010780428F7D103F5BD
:10615000817005EB0010C179CE07F0D4601C52F8B5
:106160000A1C01D08C45EAD91C460133082B8C4609
:1061700002F11002E8D1002C02DA0120BDE8F08122
:10618000224DDFF8948004F5817705EB0713998899
:10619000D8F8683DF9B92601D8F8683DDFF87C8069
:1061A0002E4441F2180208EB4421B058EBB1DC68F0
:1061B000174A0023A047C0B102280AD108F6E878A0
:1061C00005EB0715D8F89C300122013BC8F89C303C
:1061D000AA710020D2E705EB041041F21802260153
:1061E000805813B19B689847D6E70A4BD3F89C2098
:1061F00005EB07150320013A0121C3F89C20A87183
:1062000083F8A010E5E700BFFE5C0020D84C00201A
:106210006D0E0008D85C002010200020F04C0020FB
:106220002DE9F04390F82830013B83B00446082B59
:106230000BD8DFE803F0393D1F24052A0A2F34006C
:106240000121FFF7A7F8012802D003B0BDE8F083D1
:106250002378216C002284F82820002BF5D0D4E983
:10626000010383424FF0030238BF0346A36084F862
:106270002820E162204603B0BDE8F0439AE6002101
:1062800003B0BDE8F043FFF785B803B0BDE8F043C5
:10629000FFF780B903B0BDE8F043FFF717B903B0CB
:1062A000BDE8F043FFF780BA03B0BDE8F04309E46E
:1062B000534F4368D7F81852026BD7F8101290F872
:1062C00000C01D4005EB020EBEEB412F4FEA4126F8
:1062D000184645D3A7F580594FF6F778BCF1020F61
:1062E00014D02169084600295ED16068A368E26A7B
:1062F000834238BF03460021A36084F82810002A97
:10630000A3D0204603B0BDE8F04310476068D7F83B
:106310002012B0EB412F68D22069217E090735D5C4
:10632000D7F8941100F1010E71452BD297F8B411F2
:1063300000294BD1012387F8B43189F8013094F852
:1063400000C06368226B921B2A4433445B1B964255
:10635000C4E904E06360226318464FF00005BDD92C
:10636000BCF1020F41D021690029BFD0254B1B7819
:10637000032B40D089B24FF6F7739942B6D8104438
:106380006060B3E7DFD14FF0000EDCE701A972F0E7
:106390003BFE01287FF459AF2069DDF804E094F852
:1063A00000C06368226BCEE799F800E0BEF1030FEE
:1063B00012D01FFA81FEC64594BF4FF0000E4FF079
:1063C000010EBEF1000FA8D06068CDE7012189F869
:1063D000011094F800C0B6E7DFF82CE0714594BFD7
:1063E0004FF0000E4FF0010EEBE7D7F82032B0EB84
:1063F000432FC4D37AE7044B99423FF677AFBEE709
:10640000D85C0020D84C0020F7FFFF0F70B5194D65
:10641000194BC5F8983B194B85F8A41B002683F847
:10642000186A05F69833C0E954330D23C0F8583183
:1064300040F201130446C0F85C6100F5A271A0F8B7
:10644000443175F03BFF1F23C4E9EC36E3780122A9
:1064500005F599659342C4F8A853A4F89C2308BF96
:10646000C4F8AC5304F567712046BDE8704075F080
:1064700025BF00BF08310020555342531020002093
:10648000F0B50B7813F0600283B004462BD0202ABD
:1064900030D14A78FE2A39D0FF2A2DD14A88002AE5
:1064A0003BD1CA88002A38D11F0636D46148624BD6
:1064B00080F8182AC4F8B423E278012183F8E8149C
:1064C000A4F89C1303F599631F21012AC4F8B013A3
:1064D000C4F8A83304F5677108BFC4F8AC3320468C
:1064E00075F0ECFE06E04B780A2B1AD00B2B08D087
:1064F000012B2AD0002002E075F072FD022003B0CB
:10650000F0BD4D4B4A8883F8A92BF3E74F8827B994
:10651000CD88012D01D11B0642D4204675F060FDC7
:10652000ECE7022180F811114FF48071A0F81C11E2
:1065300042490123C0E94A11C0E94E33C0E94C3257
:1065400000F58E7175F058FED4E78B88C0681E0682
:10655000DDB244D40192019A394B42F0100201920B
:10656000019A026102690192013B02D0019AD206AE
:10657000F8D4314E2946204675F0A4FD294696F8F8
:10658000E85402234022204675F0CCFD022DB1D103
:106590008121204675F05CFD002386F8E834A9E7E8
:1065A000254ED6F800359B699847C0B286F8A80BEF
:1065B0000028B2D0022306F6A83684F811314FF431
:1065C0008073C4E94E55C4E94A66C4E94C57A4F83F
:1065D0001C3104F58E71204675F00EFE8AE700929C
:1065E000009A174B42F020020092009A65F38A123B
:1065F0000092009A026102690092013B02D0009A67
:106600009106F8D40C4E2946204675F05BFD2946CC
:1066100096F8E85402234022204675F083FD022DAF
:10662000B6D0012D3FF466AF01212046FFF7EEFE04
:1066300060E700BF1020002008310020B13C00209E
:10664000410D030010B50D4B93F8183A022B07D0FB
:10665000033B012B02D80021FFF7D8FE002010BD1C
:10666000074B93F8D514044675F0DCFE0028F5DAE4
:1066700001212046FFF7CAFEF0E700BF10200020EE
:1066800008310020F8B53F4C94F8186A05467EB1F1
:10669000012E01D00020F8BD3B4B93F8D51475F0C6
:1066A000C1FE0028F6DA31462846FFF7AFFEF1E7D3
:1066B000354FB0F8B433D7F8D024C7F8A02B1F2B30
:1066C000D7F8CC24C7F89C2B08D1304BD7F8C82476
:1066D0009A4203D197F8D514012919D997F8AA3B02
:1066E0005A1CD2B207EBC303042A18BF1646052270
:1066F00083F8AC2B4FF400522846C3F8B02B02238A
:1067000087F8AA6B87F8E834FBF760FB0020F8BD38
:1067100097F8D634013B0F2BE0D875F083FE0028A4
:1067200027DB94F8183A013B022BB3D9B7F8CC3BDE
:106730001BB3042284F8182A154AC5F85C61C5E920
:106740005422D7F8D02487F8A46B934228BF13466D
:10675000D7F8A02BC5F8583140F20111A5F8441123
:10676000D21A05F5A2712846C7F8A02B75F0A6FD30
:1067700090E72846FBF72AFB8CE719462846FFF7E7
:1067800045FE87E710200020083100205553424382
:10679000D83C002000207047704700BF704700BF02
:1067A000D0ED007AD0ED036A30EE677AE6EE877AB4
:1067B000B0EE670AC0ED007A704700BF90ED017A35
:1067C000B5EE407AF1EE10FAF0EE407A09D19FED85
:1067D0000D7A60EE870AF7EE006A86EEA07A80ED09
:1067E000017A31EE077A90ED000A80ED021AC1EECF
:1067F000076A77EEC07AC0ED036AA6EEA70A80EDBD
:10680000000A7047DB0FC940D0ED056AD0ED017A70
:1068100090ED066AD0ED025A90ED035AC0ED066A7B
:10682000B0EE407A26EEA70AD0ED007A80ED057A28
:10683000A7EE870AD0ED077AA5EE860A90ED086AE2
:10684000D0ED045AC0ED087AA5EE670AA5EEC60A97
:1068500080ED070A704700BFF0EE406AD0ED007A85
:1068600090ED050A90ED037A90ED016AD0ED025AA1
:10687000A7EEA60AD0ED047A27EE407A67EEC07A3A
:10688000A6EE267AE5EEA67A90ED066AC0ED067AC7
:1068900036EE076A80ED056A704700BF03685A1C30
:1068A00002601970704700BF2DE9F04FD0E9003148
:1068B00085684A1C00EB8104F1EE407A92FBF3F606
:1068C000002D03FB1622426089B084ED200AC4ED3E
:1068D000407A40F346815A189FEDA46A0692591EE9
:1068E0006A1C079200F1800900F5807BF0EE466A91
:1068F00002224FF0010A884606998C1A94FBF3F1A4
:1069000003FB1144611C91FBF3F003FB101101EB3D
:106910000A0009EB840E0BEB840C924590FBF3F418
:106920009EED007ADCED007A03FB1400A3EB020677
:1069300080F2CD80CDE901ECCDE9032637460C4647
:106940000546059031E0A34209EB850C0BEB85066B
:1069500005F1010531DD09EB84000BEB840E2246C5
:10696000013490ED006AD6ED005ADEED006AB4EE17
:10697000C76AF1EE10FA07DD9CED005AB4EEC56A65
:10698000F1EE10FA00F38680F4EEE76AF1EE10FA09
:1069900004DDF4EEE56AF1EE10FA13DC0137474549
:1069A000B0EE467A2EDAF0EE667AAB42CBDCA3424A
:1069B0005E46CC464FF00105CDDCDE46484601245C
:1069C0000022CEE7F4EEE75AF1EE10FA58BFF0EEEF
:1069D000657ABAF1010FCEED007A18BF01200CD014
:1069E0000132934200F10100CEBF0BEB82065E46FE
:1069F00000228245C6ED007AF2D101374745B0EE5C
:106A0000677AD0DBDDE901ECDDE903260598DEEDF0
:106A1000006A9CED006A30E08B4209EB800C0BEBC6
:106A2000800700F1010030DD09EB81050BEB810EE1
:106A30000C46013195ED007AD7ED005ADEED007A73
:106A4000B4EEE67AF1EE10FA06D59CED005AB4EEFB
:106A5000C57AF1EE10FA4DD4F0EE476AF4EEC67A3C
:106A6000F1EE10FA04D5F4EEE57AF1EE10FA5DD409
:106A7000B0EE676A0136B04529DD8342CCDC8B423B
:106A80005F46CC464FF00100CEDCDE464D4601218C
:106A90000024CFE7B4EEC75AF1EE10FA58BFB0EEBB
:106AA000457ABAF1010F80ED007A3FF46DAF1046E0
:106AB00001260130834206F10106CEBF09EB800CAE
:106AC000CC46002056458CED007AF2D15CE7079960
:106AD0000AF1010A8A4502F1020208F1FF387FF447
:106AE0000BAF76EEC66AF6EE007A26EEA70A09B07C
:106AF000BDE8F08FB4EEE65AF1EE10FAD8BFF0EE32
:106B0000456ABAF1010FC5ED006AA7D025460127F5
:106B10000135AB4207F10107CEBF09EB850CCC462E
:106B200000255745CCED006AF2D197E7F4EEC65A3E
:106B3000F1EE10FAD8BFB0EE656ABAF1010F8EED32
:106B4000006A97D001250134A34205F10105CEBFAB
:106B50000BEB84075F460024554587ED006AF2D1B0
:106B600088E79FED020A09B0BDE8F08F0000000041
:106B700003685A1C02601970704700BF024B186806
:106B800003681B68184700BF005F0020007970474A
:106B90000079C0F34010704700794009704700BF8A
:106BA00090F83C20034602F0FF0012B1002283F867
:106BB0003C2070474FF48053838170474FF400634B
:106BC000838170474FF40063838170474FF4006303
:106BD000838170474FF40063838170474FF40063F3
:106BE000838170474FF4006383817047074B10B473
:106BF00003F11001002453F8042B824208BF43F82C
:106C0000044C8B42F7D15DF8044B7047045F0020C1
:106C100070B5374C608CA38AB4F92C50B4F9266057
:106C2000B4F91AC01B1A208C00FB03F3B4F92A0034
:106C300005EBE335C00290FBF5F000EBE330A0F587
:106C40007A6EB4F9243020630EFB0EF52D1305FB8C
:106C500006F605FB03F3B4F91C500EFB0CFC0EFB0F
:106C600005F51B1403EB65334FEAEC2CB4F918500F
:106C70000CEBE62C0CEB850C0233B4F93450A66B0C
:106C8000E48B9B1003F500430CFA05FC04FB03F3B3
:106C90000CF1020C4CF25034A6EBAC0C2C4104FB72
:106CA0000CF4002C4FEAD333ABBF6400B4FBF3F316
:106CB000B4FBF3F35B0089B11C120E4D04FB04F42A
:106CC00040F6DE3606FB04F403FB05F5241404EB62
:106CD000254404F6CF6403EB24130B602AB100EBC8
:106CE00080004000083000111060012070BD00BF1E
:106CF000005F002043E3FFFF012070470120704741
:106D00002DE9F04F734DE86BB5F84030B5F94CE024
:106D1000B5F948C0B5F84680B5F94E6085B0C3EB0B
:106D20002014009204FB04F4B5F94420CDF80CE0E3
:106D3000241302FB04F45B00B5F942200296C3EB76
:106D4000E00302FB03F3A41304EBE324EB6D0193D4
:106D5000A4F5FA30B5F94A30AC6580FB00EA4FEA99
:106D6000E37B03FB0AF98CFB00C20EFB0B99A3FB30
:106D70000E3BCB4412031B0A42EA1C5243EA0B634C
:106D80004FEA0C3C13EB0C0342EB2B22A3FB083C19
:106D900002F5004208FB02CC4FEAEC734FEA6C09A3
:106DA00053EA6C0C0F46B5F9501000F09180029E2A
:106DB000019A86FB0008C2F5801C01FB0AFA4A46CC
:106DC0004FEA48484FEAE17948EAD0380EFB09A972
:106DD0004004A1FB0E1E4118F14449EB08090020B4
:106DE0000CF00048039E411848EA5C084FEACC7C4E
:106DF000BCEB010C09EBC60968EB09081CEB0C0E97
:106E000048EB08011EEB0C0E48EB010188014FEA2C
:106E10008E1940EA9E601EEB090E41EB00018900CD
:106E200041EA9E714FEA8E0E1EEB0C0E48EB0101FB
:106E30004FEA8E00890010EB0C0041EA9E7148EB8E
:106E4000010177F00FF9B5F956304FEA61384FEA92
:106E5000503E4EEAC14EDA1703FB08F984460EFB9A
:106E60000299B5F95400B5F95220A3FB0E35A94497
:106E700003FB08F50EFB0955A3FB0E3E75445B0EA4
:106E800043EAC51313EB0C0341EB65654FEAE07E63
:106E900000FB01F10EFB0C11A0FB0C0C6144C00CBB
:106EA00040EA41301B1845EBE1451B0A43EA056304
:106EB00003EB02130FB11B0A3B60009B23B104EBF1
:106EC0008404803424121C60012005B0BDE8F08FDA
:106ED0000023EFE7005F002001207047012070478A
:106EE0002DE9F04FC54C83B0B4F86400236ECDE9B2
:106EF0000012B4F86620A3EB002394F96800A2FB0B
:106F00000326A3FB0335C71700FB05F5B60446EAC5
:106F1000923603FB07559204A0FB030380182B4411
:106F200043EB0603002B02DA013843F10003009A19
:106F3000DF17C4E92037002A00F00C8103FB07F0BB
:106F4000A3FB032E0EEB400E4FEA921949EA8E691D
:106F50004FEAAE1609FB07F003FB0600A9FB0396F8
:106F60008019D4F8885000F143814FEA192949EA81
:106F700000694FEA202B94F96E004FEAE07C00FB99
:106F80000BF609FB0C66A0FB090C16EB0C0600F1D6
:106F90002B81B4F96980B4F96BC0400940EAC6603E
:106FA0000146A8F5804894F96D004FEA883808EB4F
:106FB00066184FEAE07A00FB0EF602FB0A66A0FBB9
:106FC00002A00644B6004FEA8A00ACF5804C46EABF
:106FD0009A76081848EB06084FEAEC7A0CFB07F69D
:106FE00003FB0A66ACFB03CA5644760546EADC2678
:106FF0004FEA4C5C10EB0C0048EB0606002EC0F28A
:10700000EC8094F974C00CFB0BF84FEAEC7A09FBA6
:107010000A88ACFB09C9000E18EB090840EA0620F3
:107020004FEA266600F1D48094F97390B4F871A009
:1070300009FB0EFE4FEAE97B02FB0BEEA9FB0229DE
:10704000CE444FEA5C1C4FEA0E1E4EEA127E4CEA1A
:10705000C86C12011CEB020CB4F86F204FEAC2326C
:1070600002EB681848EB0E08AAFB03E20AFB0722B2
:10707000920542EA9E224FEA8E5E1CEB0E0C48EB14
:107080000208B8F1000FC0F29E804FEA9C0C94F900
:107090007720B4F975E04CEA887CA0FB05091CEB6D
:1070A000000C05FB069040EBA80002FB07F64FEA38
:1070B000E27803FB0866A2FB032846444FEA0E4829
:1070C00012EB080246EBEE7EA2FB052605FB0E66E0
:1070D000002E71DB520B42EAC642A2FB052E76134C
:1070E00005FB06E6002E60DB520A94F978E042EADE
:1070F000C6521CEB020440EB6620A5FB052C4FEAB0
:10710000EE7602FB06F60EFB0C66A2FB0E2E16EBCD
:107110000E0643D4120C42EA0642A2FB052C36149A
:1071200005FB06C5002D35DBD20942EA456212197E
:1071300040EBE510941840EB0005A41840EB050562
:10714000ED0045EA5475E400A41840EB0500009AF0
:10715000000C1060019A9AB1DA1847EB0701D218B7
:1071600047EB0101C90041EA5271D200D21847EB46
:107170000107002F08DB019B920B42EA87421A604D
:10718000012003B0BDE8F08F43F6FF73D21847F13A
:107190000007F0E77F3245F10005C5E74FF6FF7CB9
:1071A00012EB0C0246F10006B4E740F2FF1E12EBB0
:1071B0000E0246F1000697E741F6FF7E12EB0E0243
:1071C00046F1000686E71CF1030C48F100085CE775
:1071D0001CF11F0C48F1000826E76FF07F4C10EB04
:1071E0000C0046F100060CE71F3046F10006D0E621
:1071F00019F1FF0940F10000B7E600BF005F002071
:1072000031B10A4BD3ED2A7AFDEEE77AC1ED007A6F
:1072100052B1064B9FED067AD3ED2B7A67EE877A53
:10722000FDEEE77AC2ED007A01207047005F002092
:107230000000C8422DE9F04F614DB5F8BE30D5F8D9
:10724000B000B5F8BCE0B5F8BA40B5F8C06085B09C
:107250001B02C01A67EB0707B5F8B8300191AEFB07
:10726000001C0EFB07CCC9091B0441EA4C61C9187C
:107270009346A4FB003EB5F8B62004FB07EE4FEAA8
:1072800013234FEAC23243EA0E634FEAEC1C4CF17F
:10729000000C9B18A6FB002406FB07444FEAD252C1
:1072A00042EA44224FEA2E2E4EF1000EE41512F56A
:1072B000FA6944F10006B9F5FA6F029676F1000614
:1072C00032DAA2FB02A802FB04F6039408EB4604A0
:1072D0004FEA84084FEA8A0616EB0A0648EA9A78CB
:1072E00044EB08084FEA560A4AEAC87AB608B1EBF6
:1072F0000A0A46EA8876334C6CEB680C9E1B3346D0
:10730000029E6EEBA80EA1454FF0FF34A6415146F8
:1073100027DB00FB07F7A0FB000202EB4702C00FD0
:1073200040EA4200B9EB0009019C8CB1D5F8C400D9
:10733000A0FB033200FB0E225B0D43EAC2235B1A63
:107340004FEA625262EB0C02DB0B43EA42432360DA
:10735000BBF1000F01D0CBF80090012005B0BDE8D3
:10736000F08F40F6AC56039C921944F1000402FBE6
:1073700004F4A2FB026202EB44024FEAC208F400EA
:10738000341B48EA567862EB080864184CEB080C8A
:107390002146B41942EB0208A41942EB08084FEA4F
:1073A000880848EA9478A400A41B68EB02086208E5
:1073B00042EAC8729A1A6EEB680E1346A9E700BF3C
:1073C000005F002024FAFFFF0120704710B40F4B2C
:1073D0000F4C1B68D4F8C8001B1AFA2B0BD811B13C
:1073E000D4F8D0300B6012B1D4F8D430136001203F
:1073F0005DF8044B7047074A1368002023F004032C
:1074000084F8CC0013605DF8044B7047242A0020F8
:10741000005F00200000001001207047064B002292
:107420000021C3F8D820C3F8DC20C3F8E020C3F85B
:10743000E4100120704700BF005F0020104B114A8C
:107440001B68D2F8E4105B1AFA2B16D8D2ED366A14
:1074500092ED377AD2ED387AFDEEE66ABDEEC77A64
:1074600016EE903AFDEEE77AC38617EE103A0387E0
:1074700017EE903A4387012070470020704700BF05
:10748000242A0020005F002030B50F4A83B092F814
:10749000E8500191B5B9D2F8EC509DB12B681A684B
:1074A00082B19B6873B104462846984750B12B6857
:1074B000019922461C6828460B46214603B0BDE8C8
:1074C0003040084703B030BD005F00200B4B70B563
:1074D000D3F8F0608EB133681A6872B19B6863B1FB
:1074E000054630460C46984738B133682A46196835
:1074F00030462346BDE87040084770BD005F00205D
:1075000038B51446002944D0344BDFED355AD3ED5D
:107510003D7AB3F9102193ED400AB8EEE77A05EE13
:10752000102AC7EE256AB3F90C210D46D3ED3E7A39
:1075300006EE102AF8EEE77AB3F90E21C7EEA54A57
:1075400005EE902AB3F90A2107EE102AF8EEE55A63
:10755000B3F90821B8EEC77A07EE902AA6EEA57A0D
:10756000B8EEC55AB8EEC66AF8EEE77AA6EE856AB6
:10757000E6EE877A93ED417AB8EEC77AB8EEC00AA4
:10758000A6EE867AA6EE870AA4EEA70A77F0F0FCAC
:1075900028600CB3114B9FED126AD3ED3E7AB3F91C
:1075A000FE20B3F9FC30F8EEE76A07EE102A86EE0B
:1075B000860A07EE903AB8EEC77AF8EEE77A20EE40
:1075C000070AB6EE006AA7EE860ADFED066A20EE2D
:1075D000260A77F0CDFC2060012038BD005F002036
:1075E0000000F04A0000C8422DE9F0410446D0E90D
:1075F0000030134483421DD80D4601EB0208B2B19E
:1076000004F10C07002601E0A84510D023695A1C9C
:107610002261234415F8011B1973042AF4D1394659
:107620002046FBF73BFBA845C4E90460EED1606946
:10763000BDE8F0814FF0FF30FAE700BF034690F954
:1076400010002DE9F04116469A68224C00EB8000AC
:10765000920754F8208009D5404675F05BFC31460E
:10766000404675F057FC0120BDE8F0815D69084691
:1076700015B12B68AA885A83174B184FD3F81441B9
:10768000174B7A684FEAC40CA3FB0C3C4FEA9C1CD6
:107690007B689B1A9C45FBD20146404675F03AFC3C
:1076A0003146404675F036FC0D4B78680B494FF477
:1076B000FA7204FB02F2A3FB023292094B681B1A16
:1076C0009A42FBD2002DCED02B68AA881A830120C3
:1076D000BDE8F081500C0020005F0020001000E0A9
:1076E000D34D621000680379012B0AD0022B01D020
:1076F000002070478368DB074FF0F00218D5FF21A8
:107700009CE700B5826890F910C0417C85B002F01A
:10771000010201920DF10F0200926046FF224FF02C
:10772000F00C8DF80FC0FCF771FF05B05DF804FB9D
:107730007F2183E700680379CA4341EA0211012BE4
:10774000CAB208D0022B01D0002070478368DB0743
:1077500016D5D22172E700B585B090F910C08DF82A
:107760000F208268417C02F001020DF10F00CDE98B
:107770000002D2226046FCF749FF05B05DF804FB29
:1077800052215BE700680379012B0AD0022B01D05C
:10779000002070478368DB074FF0B40218D5FF2143
:1077A0004CE700B5826890F910C0417C85B002F0CA
:1077B000010201920DF10F0200926046FF224FF08C
:1077C000B40C8DF80FC0FCF721FF05B05DF804FB89
:1077D0007F2133E700680379012B09D0022B01D008
:1077E000002070478368DB070A4616D5A52125E7E8
:1077F00000B5826890F910C085B002F001028DF8E2
:107800000F10417C0DF10F00CDE90002A52260466A
:10781000FCF7FCFE05B05DF804FB25210EE700BF78
:1078200000680379012B0AD0022B01D00020704799
:107830008368DB074FF0960218D5FF21FEE600B5FE
:10784000826890F910C0417C85B002F0010201927B
:107850000DF10F0200926046FF224FF0960C8DF85A
:107860000FC0FCF7D3FE05B05DF804FB7F21E5E611
:1078700000680379012B09D0022B01D0002070474A
:107880008368DB070A4616D58721D7E600B58268EC
:1078900090F910C085B002F001028DF80F10417C04
:1078A0000DF10F00CDE9000287226046FCF7AEFE25
:1078B00005B05DF804FB0721C0E600BF006803794E
:1078C000C901012BCAB205D0022B01D0002070479C
:1078D0007821B3E600B585B090F910C08DF80F207F
:1078E0008268417C02F001020DF10F00CDE9000237
:1078F00078226046FCF78AFE05B05DF804FB00BF05
:1079000000680379012B0AD0022B01D000207047B8
:107910008368DB074FF0550218D5A5218EE600B528
:10792000826890F910C0417C85B002F0010201929A
:107930000DF10F0200926046A5224FF0550C8DF814
:107940000FC0FCF763FE05B05DF804FB252175E66A
:1079500000680379012B0AD0022B01D00020704768
:107960008368DB074FF02E0218D5F42166E600B5D8
:10797000826890F910C0417C85B002F0010201924A
:107980000DF10F0200926046F4224FF02E0C8DF89C
:107990000FC0FCF73BFE05B05DF804FB74214DE61B
:1079A000144B00689A8E037992013432012BD2B2C3
:1079B00008D0022B01D0002070478368DB0716D562
:1079C000F4213BE600B585B090F910C08DF80F208A
:1079D0008268417C02F001020DF10F00CDE9000246
:1079E000F4226046FCF712FE05B05DF804FB74213A
:1079F00024E600BF005F002000B500680379012B7A
:107A000085B012D0022B03D0012005B05DF804FB35
:107A10008368DB074FF031024CBFF4217421FFF77C
:107A20000DFE012005B05DF804FB826890F910C0DE
:107A3000417C02F0010201920DF10F0200926046BA
:107A4000F4224FF0310C8DF80FC0FCF7DFFD012060
:107A500005B05DF804FB00BF00680379012B06D078
:107A6000022B01D00020704713221B21E6E500B550
:107A7000826890F910C0417C85B002F00102019249
:107A80000DF10F02009260461B224FF0130C8DF88F
:107A90000FC0FCF7BBFD05B05DF804FB006803797F
:107AA000012B06D0022B01D0002070470122582163
:107AB000C4E500B5826890F910C0417C85B002F041
:107AC000010201920DF10F020092604658228DF8DA
:107AD0000F30FCF79BFD05B05DF804FB00680379EF
:107AE000012B06D0022B01D0002070470122482133
:107AF000A4E500B5826890F910C0417C85B002F021
:107B0000010201920DF10F020092604648228DF8A9
:107B10000F30FCF77BFD05B05DF804FB00680379CE
:107B2000012B06D0022B01D0002070471A460821F5
:107B300084E500B5826890F910C0417C85B002F000
:107B4000010201920DF10F020092604608224FF0EF
:107B5000020C8DF80FC0FCF759FD05B05DF804FB71
:107B600000680379012B06D0022B01D0002070475A
:107B70000122082162E500B5826890F910C0417CBD
:107B800085B002F0010201920DF10F0200926046F1
:107B900008228DF80F30FCF739FD05B05DF804FBC5
:107BA0002DE9F0410C4E356873691D4011D0DFF8A6
:107BB0002C800127B5FA85F4C4F11F0408EB840377
:107BC00007FA04F4D3F8180103689847A5437461D1
:107BD000F0D1BDE8F08100BF003C0140005F002013
:107BE00010B54FEA511E024400EB8E0C624529D9B4
:107BF00001F01F034FF0FF3450F82E1004FA03F386
:107C00000B4093FAA3F3B3FA83F3DBB2202B16D124
:107C10000CF104018A4202D817E08A4212D98C463C
:107C20000431DCF8003093FAA3F3B3FA83F3DBB248
:107C3000202BF2D0ACEB000C03EBCC0010BD03EB1F
:107C40004E1010BD4FF0FF3010BD204610BD00BFDC
:107C50000369416890ED067AF0B4C56A394E8768C9
:107C600053EA010204BF316841606A1C30EE077AB2
:107C70000133012A80ED067A0361C26240D090EDA3
:107C8000075AD0ED096A346807EE902A70EE455A1B
:107C9000B8EEE76A611AC5EE867AB94277EE857A60
:107CA00030EE670AC0ED087AE5EE806AC0ED077A2B
:107CB000C0ED0A6AC0ED096A01D8F0BC7047012A1C
:107CC00029DD07EE905AF8EEE77A86EEA76AB5EE60
:107CD000C06AF1EE10FA1EDBF1EEC67AF4EE677AB6
:107CE000F1EE10FA17D6D0ED056AF4EEE76AF1EE80
:107CF00010FA13D5037BEBB10323F0BC037070477C
:107D0000326880ED080A521ABA424FF0000180ED45
:107D1000070A4162D1D9DFED0C7AE4E707EE903A29
:107D2000F8EE677A0223C7EE276AF0BC0370C0ED55
:107D3000066A704731684160002203618261C36254
:107D4000BBE700BF242A002000000000DFED4F4AFF
:107D500010B5844600F1480E0346B1EC017AD3ED2C
:107D6000067ADA6A77EE877A0132012AC3ED067A5B
:107D7000DA6254D093ED075A93ED096A07EE902A20
:107D800077EE455AF8EEE77AC5EEA76A76EE857A81
:107D9000F0EE466A37EE677AC3ED087AE5EE876A59
:107DA000C3ED0A6AC3ED077AC3ED096A1833734558
:107DB000D3D1374C416822680369521A8168013374
:107DC0008A4203612AD990ED056A00F1300EDCF891
:107DD0002C20DCED0A6A012A02F1FF3126DD07EED4
:107DE000901AF8EEE77A86EEA77AB5EEC07AF1EE51
:107DF00010FA1BDBF1EEC77AF4EE677AF1EE10FAB7
:107E000014D6E645B4EEE76A0CF1180C16D0F1EE84
:107E100010FADCD5037B6BB30323037010BDF0EEC7
:107E2000477AF0EE646A83ED087ABBE7DFED177AF4
:107E3000E645B4EEE76A0CF1180CE8D1F1EE10FA61
:107E4000E8D407EE903AD0ED066A90ED0C7AD0EDCA
:107E5000125AF8EE677A022386EEA76A0370C7EE1D
:107E6000276A85EEA77A80ED066AC0ED0C6A80ED80
:107E7000127A10BD00222168416003618261C362F1
:107E8000026343648264C36510BD00BF000000004C
:107E9000242A0020B0EEC06AF0EEE05AF4EEC65A92
:107EA000F1EE10FAF0EE407A0EDCB5EE400AF1EE9B
:107EB00010FA4BD0F4EEC65AF1EE10FAF0EE466A24
:107EC00050D5B0EE655A03E0F0EE656AB0EE465A62
:107ED00085EE267A9FED252A9FED253A9FED254ACE
:107EE000DFED254ADFED252ADFED253ADFED256AB6
:107EF000A7EE023AE7EE223AA7EE034AB7EE005A9F
:107F0000E7EE044AA7EE235AE7EE246AF4EEC65AD7
:107F1000B1EE667A87EE050AF1EE10FA48BF9FEDE2
:107F20001A7AF5EEC00A48BF37EE400AF1EE10FAB1
:107F300048BF9FED167AF5EEC07A48BF37EE400A8B
:107F4000F1EE10FA48BFB1EE400A7047DFED107A4B
:107F50009FED100AF5EEC00AF1EE10FA58BFB0EE30
:107F6000670A7047B0EE465AB2E700BF39094E3D86
:107F7000E3B59EBE88FA16BE45FE7FBF99FB243F3F
:107F800069A2163EA7DFA8B4DB0FC93FDB0F49404B
:107F9000A7DFA834DA0F494091ED007AD0ED047ADA
:107FA00090ED054AD0ED064A90ED075AD0ED085AFB
:107FB00090ED096AD0ED0A6AE7EE077AF7EE003A2B
:107FC000C0ED047A91ED007AD1ED017AA7EE274A4F
:107FD00090ED0B7A80ED054A91ED024A91ED003A61
:107FE000D0ED0C7AE3EE044AC0ED064AD1ED004A2A
:107FF00035EE245A80ED075AD1ED014A91ED005A31
:10800000E4EE855AC0ED085AD1ED015AA5EEA56AF5
:1080100080ED096AD1ED015A91ED026AE5EE866ABA
:10802000C0ED0A6AD1ED016A37EE267A80ED0B7A4F
:10803000D1ED026A91ED007AE6EE877AC0ED0C7A16
:1080400091ED026AD1ED016AD0ED0D7A90ED0E7AD4
:1080500090ED0F4AD0ED104A90ED115AD0ED135A21
:10806000E6EE267A75EEA35AC0ED0D7AD1ED026ADE
:10807000D0ED127A90ED006AA6EEA67AD0ED016AF4
:1080800080ED0E7A91ED027A34EE074A90ED027A95
:1080900080ED0F4A91ED004A74EE844AC0ED104A1B
:1080A000D1ED014A35EE245A80ED115A91ED025A74
:1080B000C0ED135A77EE857AC0ED127AD1ED017AD0
:1080C000D1ED005A91ED025A67EEA77AE5EEA57A56
:1080D000E5EE057AA5EEA76A80ED006A91ED016AEA
:1080E000E6EE276AC0ED016AD1ED026AA6EEA77A34
:1080F00080ED027A90ED037A77EE277AC0ED037A6D
:10810000704700BF2DE9F04F4FF0000989B0864657
:1081100000F110050646034600F1300807464846C0
:108120002C46CDF80CE08B469C46B24600283CD14C
:108130000CF1040CA445FBD1032800F1010151D03E
:108140009C46AA46029398B1DCED047A0192AAEB10
:108150000903B6467246F3EC016A92ED007AE6EE48
:10816000C77A53450EF1100ECCED047AF2D1019A84
:10817000DCED046A15ED047AC6EE877A0CF1100C7A
:10818000C4450AF1100ACCED007ADCD1029B04361A
:108190001433084608F1040814351034103709F177
:1081A00004099C46B2460028C2D0DCED007A019258
:1081B000D64639467246F1EC016A92ED007AE6EE57
:1081C000C77A99420EF1100ECCED007AF2D10CF183
:1081D000040CA445019A0AF1040AE6D1032800F12F
:1081E0000101ADD1DDF80CE000235946049305935D
:1081F000069307937646774604AD0020F2EC017AA9
:10820000E5EC017AB0B104AC3B46B4EC017AF3EC96
:10821000016AE6EEC77AB34245ED017AF5D1013045
:1082200004280BD0F2EC017A10371436E5EC017A11
:108230000028E8D1103714360120DFE708AD75EDCE
:10824000017A10310EF1400E04287446A1F10402A7
:1082500041ED017A1ED07346F3EC016AB1EC017A6C
:10826000E6EEC77AA342C2ED007AF5D15EED016A6F
:1082700087EEA67A013882ED007A17D0AEF1140E9F
:10828000103C114675ED017A0428A1F1040241ED7C
:10829000017AE0D15EED016A87EEA67A103CAEF17C
:1082A000140E032001ED017A1146EBE709B0BDE899
:1082B000F08F00BFDFED297AB4EEE70AF1EE10FA95
:1082C00028DD9FED277A30EE470AB4EEE70AF1EE9B
:1082D00010FAF8DCDFED237AB4EEE70AF1EE10FADB
:1082E0002FDD30EE670A37EEC00A60EE007A9FEDB0
:1082F0001E7A9FED1E6ADFED1E6AA7EE876A9FED6C
:108300001D7AE7EE866A60EE275AA7EEA67AA5EEFA
:10831000870A7047DFED187AB4EEE70AF1EE10FA3B
:10832000D8D59FED0F7A30EE070AB4EEE70AF1EEEA
:1083300010FAF8D4DFED0B7AB4EEE70AF1EE10FA9A
:10834000CFDC9FED0E7AB4EEC70AF1EE10FA44BF0F
:1083500030EE270A37EE400AC7E700BFDB0F49407F
:10836000DB0FC940DB0FC93F9A7C2E36FAAF4FB9FD
:108370003587083CA4AA2ABEDB0F49C0DB0FC9BF62
:1083800010B5404CB4FBF2F4A14219D3DFED3E7AB4
:10839000F7EE005AB0EE677AB0EE676AF0EE676A01
:1083A0000023C0ED005AC0ED017A80ED027A80ED25
:1083B000036AC0ED046A836143610362C36110BD57
:1083C00007EE902AB8EE677ADFED307A27EE277A4B
:1083D000B7EE006AC6EE076A07EE901A9FED2C7A98
:1083E000F8EE677AB0EE405A67EE877AC7EEA64A93
:1083F000FDEEE47A17EE902A2032402A3FD8B0EE04
:10840000640AFFF757FFB0EE404ADFED227A34EE00
:10841000A70AFDEEC07A17EE902A2032402A29D80A
:10842000FFF748FFF8EE006A60EE266A012B1CD0C9
:10843000B7EE006A36EE406AF6EE004A66EE244A6F
:1084400035EE055AF7EE007A84EE057A77EE275A74
:1084500037EEC75A84EEA57AC6EE257A86EEA56A6F
:10846000C5EE256AF0EE475A9AE7B0EE666AF7EE77
:10847000004AE5E7DFED086A9FED030AD6E79FEDC6
:10848000024AC2E720A1070000000000BD37863580
:10849000DB0FC940DB0FC93F00000080DFED077A2A
:1084A00030EE270AFDEEC07A17EE903A2033402BCB
:1084B00000D8FFE69FED020A704700BFDB0FC93FFF
:1084C000000000002DE9F84FDDF82CB09DF82840A1
:1084D0008946002C1BF8011B0CBF4FF020084FF001
:1084E00030081C1E0546174608463ADB00295CD0BA
:1084F000002C55D04FF0000A5B4600E064B313F83F
:10850000016B013C002EF9D1BAF1000F2FD12646A4
:1085100044B14D454146284600D2B847013CF8D108
:108520000B9B18780146A0B14FF0FF344FF0000AC2
:1085300000E09B464D45284600D2B8475B4613F8FD
:10854000011B0029F5D10B9BF61A5E44BAF1000F0E
:1085500010D13046BDE8F88FBAF1000F1BD1564656
:10856000E0E7634229B31C464FF0010AC4E7002844
:10857000E0D10646002C04F1FF3AEADD54464D45B1
:108580004146284600D2B847013CF8D2013656444D
:108590003046BDE8F88F06460028DAD02646C9E7FF
:1085A0002646A2464FF0FF34C4E72646002CB0D141
:1085B000CFE76FEA040A0E46E0E700BF0FB430B51C
:1085C00083B006AB0A4C53F8042B0193D4E9DD01C8
:1085D00074F0E2FC0546206803685B699847002850
:1085E000F9D0284603B0BDE8304004B0704700BF62
:1085F000005F00200EB410B583B005AB044653F8FD
:10860000042B0749009301A8019474F0C5FC019B59
:1086100000221A7003B0BDE8104003B0704700BFDD
:10862000716B00080CB4F0B53C4CD4F87C33ADF55C
:10863000277D002B6DD094F8843399420BD9D4F860
:10864000882301238340134205D10DF5277DBDE822
:10865000F04002B07047324B324A1B68A2FB030263
:1086600092094FF47A7101FB123306A82E49FFF7E5
:10867000C1FF06AB03442D49AC9A01930646ADAB4E
:1086800001A8009374F088FC019B0A22591C0191F7
:108690001A70019B0022591C01911A70D4F87C5366
:1086A000ADB12B685B6A1BB128469847D4F87C5360
:1086B0009DF818100029C8D00DF119042B68284620
:1086C0001B68984714F8011B0029F7D1BDE7D4F8BF
:1086D0008073002FB9D0304426AB841CFD2206A93C
:1086E000ADF8102018462246CDF81250ADF81650BD
:1086F0007AF0BAFB02220346044402A93846CDE9C7
:10870000023439F021FC0DF5277DBDE8F04002B0C0
:108710007047D4F88033002B8DD196E7005F00209E
:10872000242A0020D34D62107CFB08089D680008B5
:10873000184A10B5D2F88C43033004EB9003B3F51C
:10874000007F18D802EB8101C2F88C3302F5647205
:1087500002EB8404D1F8902B20F003001044C3F501
:108760000073C1F8900B0C4A9B0004210020FFF716
:1087700059FF204610BD00210846084AFFF752FF66
:10878000074AD2F8B030002443F00073C2F8B0308A
:10879000204610BD005F002088FB0808ACFB0808DD
:1087A0000000001038B50568EB690446F3B198780D
:1087B00000B938BDB3F90A2007EE902AF8EEE77A3F
:1087C0000120C4ED057AB3F90C2007EE902AF8EEEB
:1087D000E77AF1EE677AC4ED047AB3F90E3007EE6A
:1087E000903AF8EEE77AC4ED067A38BD09211420F4
:1087F000FFF79EFF0346E861D9E700BF38B505687B
:10880000EB690446E3B1987800B938BDB3F90420A8
:1088100007EE902AF8EEE77A0120C4ED047AB3F966
:10882000062007EE902AF8EEE77AC4ED057AB3F950
:10883000083007EE903AF8EEE77AC4ED067A38BDD4
:1088400009211420FFF774FF0346E861DBE700BF4E
:1088500038B50568EB690446E3B1987800B938BDCE
:108860009A88D2BA07EE902AF8EEE77A0120C4ED92
:10887000047ADA88D2BA07EE902AF8EEE77AC4EDE5
:10888000057A1B89DBBA07EE903AF8EEE77AC4ED79
:10889000067A38BD09211420FFF74AFF0346E86134
:1088A000DBE700BF38B50468E3690D467BB1987813
:1088B00000B938BD5B89094ADBBA82FB0312DB17BA
:1088C000C3EB221303F26D132B80012038BD092165
:1088D0001420FFF72DFF0346E061E8E77978787808
:1088E0002DE9F04103EB4306964602EB460612F9EA
:1088F000067B86B00346754692F80080A3EB080419
:10890000A3EB070C002CB8BF6442BCF1000FB8BF4A
:10891000CCF1000C6445B8BF154602F10602B8BFA1
:108920004FFA88F7B242E7D16A889EF80000B84251
:10893000144614D1BEF80200A1EB0008A1EB020C12
:10894000B8F1000FB8BFC8F10008BCF1000FB8BF04
:10895000CCF1000CE045BEBF7546024604460EF160
:10896000060E7645E1D16A7904922A79CDE9024270
:108970002878054ACDE9001003210120FFF752FEB7
:10898000284606B0BDE8F081BCFB08084B1EDBB2F0
:10899000062B9CBF214A02EB430330B598BF1D8ACA
:1089A0001F4BA3F1580488BF4FF48075002808BFFF
:1089B0001C46A44620893CF8082B87B04FFA82FE5B
:1089C00090B1A5EB0E022B1A002AB8BF5242002B21
:1089D000B8BF5B429A42C4BF64464FFA80FE3CF87F
:1089E000080F0028EDD122880E4B0F4893F818CCC1
:1089F000A3790593A38804930C4BBCF1000F18BF17
:108A00000346A078CDE90015CDE902200321084AEC
:108A10000120FFF707FE204607B030BD10540808BC
:108A2000B0150020005F00202C0F090898FA0808F4
:108A3000F8FB080803685A1C02601878704700BFEA
:108A400003681A46591C016012F8021B026058782C
:108A500041EA0020704700BF10B402681346511C61
:108A6000016013F8021B0360D31C547803609378F1
:108A70001B0443EA0423141D0460D0785DF8044B02
:108A80000B4343EA0060704712B370B50446864654
:108A900004E0981B17D114EB0C0C15D01EF8013B09
:108AA000A3F14100192811F8010BA0F1410598BF6D
:108AB0002033192DA2EB0E0C00F12006E9D91B1A68
:108AC00004D10028E7D170BD604670BD184670BD66
:108AD0001046704710B402888378174C02F00301E7
:108AE00001EB4101013B03EB810304EB4303C1783C
:108AF0001B8CA2F5FA62920840F2B55404FB0233D3
:108B00004A1E1344017942798479008903EB4303B7
:108B100001EBC301C1EB0111084B02EB8102C2EB77
:108B20000212234403EB820300214FF47A72C3FB49
:108B300002015DF8044B70471054080880436D38FB
:108B4000F8B516461F460446394630464FF47A7249
:108B5000002375F087FA3B4D3B4B054483FB0560D2
:108B60002844E917C1EB601183FB01030B44374E26
:108B7000C817C0EB631086FB003CC317344EC3EB31
:108B8000AC0386FB03764FEAE37ECEEBE61EC1EB39
:108B90000116A5EB860CC0EB0015A1EB85016171F8
:108BA00003EB4301A0EBC10040F2B55101FB1E33C2
:108BB000B3F5896F84F806C020714FEA8E0635DA66
:108BC00040F2DA218B4237DCB3F5B77FB4BF4FF008
:108BD000000E4FF0010E1F490EEB4E0001EBC001DD
:108BE0007546C88E4FEA4E071B4907EB0E0C01EB8A
:108BF000CC0C0CF1160C0B2101E03CF8020D984254
:108C000011DD0139F9D11349774401EBC701088C13
:108C10000121013306F5FA6E1B1A7544A170E37049
:108C200022812580F8BD0131C9B2F2E7032540F267
:108C30009650AE460627D7E7022540F22940AE46B9
:108C40000427D1E780BC92C789888888ABAAAA2A62
:108C500073B06D16105408083054080830B52F4C06
:108C600086460D460FCC8DB0EC46ACE80F000FCC1D
:108C7000ACE80F0094E80F001EF0030F8CE80F0023
:108C80000FD1274B274A03FB0EF3B2EBB30F43D3AD
:108C9000254AB2EB331F34BF01220022C2F11D026C
:108CA00000E01C220EF1FF33002B019240F26D1206
:108CB000194602FB0EF2B8BF0EF1020102EBA1024F
:108CC0001A491B4C81FB0301DB17A3EB6110024423
:108CD000C3EBE1131A44253284FB02311144D3174C
:108CE000C3EBA103C3EBC303D31AADF10402EE46F9
:108CF00002EB85015EF8040FC21884FB023C944429
:108D0000D317C3EBAC03C3EBC3037145A2EB03035F
:108D1000F0D1C01A0DB030BD1D22C3E79054080831
:108D2000295C8FC2285C8F020AD7A3001F85EB51F4
:108D3000932449920D4B10B5D3F8204CD3F8243C22
:108D400054EA030209D1014640F201130020C1F8A0
:108D5000023088710880088110BD054A1268121916
:108D600043F10003FFF7ECFE012010BD005F00207F
:108D7000242A002030B5144DD5F8201CD5F8243C09
:108D800051EA030283B0044609D1002040F20113E6
:108D90002080C4F80230A071208103B030BD0B4A9E
:108DA0001268521843F10003FFF7CAFEB5F8283CD9
:108DB000ADF8063020460DF10602214670F084F829
:108DC000012003B030BD00BF005F0020242A002036
:108DD00088422DE9F0414FF001043DD301FB04F43A
:108DE000B0FBF4FC8C45F9D23CB3002616E0BCF194
:108DF000090F274698462C4623DD002A0CBF4FF06A
:108E0000570E4FF0370EF444B94288F800C003F112
:108E1000010306F1010610D8B0FBF5FCB4FBF1F537
:108E200004FB1C00002EE2D1BCF1000FDFDCA142EC
:108E30000AD90CF1300C03F801CB00221A70BDE8FE
:108E4000F0814FF0300EDEE7B0FBF5FC2C4605FB61
:108E50001C00B5FBF1F5E7E78446C6E72DE9F041D4
:108E6000044694421546084609D2B4FBF2F6154B67
:108E700005FB16441B5D00F8013BBDE8F081B4FB27
:108E8000F2F69642B6FBF2F70CD20E4B05FB1767D3
:108E900005FB1644DA5D00F8012B1B5D00F8013B71
:108EA000BDE8F081BA42B7FBF2F807D9054B05FBE4
:108EB000187813F8082000F8012BE7E74046FFF781
:108EC000CDFFF3E744FC0808B5EEC00ADFED347AC5
:108ED000F1EE10FACCBF30EE270A30EE670ADFED74
:108EE000317A20EE270A30B5FDEEC07A87B017EE52
:108EF000904A054684EAE470002303A9A0EBE470DD
:108F0000CDE90033029370F053F9002CB4BF2D2348
:108F1000202303A88DF8003074F08AFA012829D0A4
:108F2000022833D003281DD003A968467BF076FFC2
:108F3000684674F07DFAC41EE4B2224669462846AB
:108F400079F092FF00232B55284674F071FA2E23F6
:108F50002B5401300DEB040128447BF0D4FF28464C
:108F600007B030BD302303A968468DF801307BF08F
:108F700055FFDDE743F23002302303A96846ADF820
:108F800001208DF803307BF049FFD1E743F2300335
:108F900003A96846ADF801307BF040FFC8E700BF89
:108FA0006F12033A00007A440278202A034600F147
:108FB0000100F9D0092AF7D02D2A29D02B2A03BF86
:108FC0005A78B7EE000A0346B7EE000AA2F1300164
:108FD000C8B20928DFED4C7A10D8F2EE046A07EE29
:108FE000101AB8EEC77A13F8012FA7EEA67AA2F1ED
:108FF0003001C8B20928F0EE477AF0D92E2A49D0BC
:10900000197801F0DF01452907D020EE270A7047C3
:109010005A78BFEE000A0346D8E710B459782D29D4
:1090200062D02B2954D0A1F13002092A03F10103A7
:1090300055D80024002202EB820201EB420213F811
:10904000011FA1F130000928A2F13002F3D9B2F5D5
:109050009A7F134628BF4FF49A73072A50D9DFED41
:109060002B6A1A46B7EE007A083A072A27EE267AC4
:10907000FAD803F007032BB1F2EE046A013B27EEA6
:10908000267AFBD16CB3C7EE877A5DF8044B20EEED
:10909000270A70475978A1F13002D0B2092803F1AC
:1090A0000103AED8F2EE046AF0EE665A07EE102A1B
:1090B000B8EEC77A13F8011F87EE266AA1F13002D5
:1090C000D0B2092866EEA56A77EE867AEED998E7DF
:1090D0009978A1F13002092A03F10203A9D9B7EE68
:1090E000007A67EE877AD0E79978A1F13002092AF1
:1090F00003F1020388BFB7EE007AC4D8012499E7D0
:10910000B7EE007AB7E700BF0000000020BCBE4CFD
:109110000378202B024600F10100F9D0092BF7D08B
:109120002D2B08BF5378A3F13001CBB206BF024606
:109130004FF0FF3C4FF0010C092B4FF0000000D91D
:10914000704712F8013F00EB800001EB4000A3F1F3
:109150003001CBB2092BF4D90CFB00F0704700BFF3
:1091600070B5344D2B787E2B01D0002070BD0822C5
:109170004FF4FC4341F2210019B200294FEA4303A6
:10918000B6BF80EA41019BB28BB2013AF4D1B5F887
:10919000011069B32848294CA042E6D20638461887
:1091A000A642E2D241F2210C0529DED9864214D032
:1091B000013806F1FF3E10F8012F082183EA02234F
:1091C0001AB2002A4FEA4303B6BF8CEA42029BB2AE
:1091D00093B20139F4D17045EDD1318849B1B21D56
:1091E000A242C2D27218A2423046BED21646DBE775
:1091F000134E741E41F22100A44614F8012F0821D9
:1092000083EA02231AB2002A4FEA4303B6BF80EA78
:1092100042029BB293B20139F4D16645ECD1728817
:10922000D01A084A331D5B1BB0FA80F04009A2F83F
:109230002C3C70BD00000E0807000E08000010084E
:1092400001000E08005F00202DE9F04F914B924A7B
:109250008BB00020D21ACDE90600CDE90800D11864
:1092600005928E4A0393049110690028C0F281810F
:109270008A4AF320D0600020089089480122884261
:109280008DF8242000F271817E2007928DF818005D
:109290004FF4FC42082041F2210514B2002C4FEAA1
:1092A0004202B6BF85EA440492B2A2B20138F4D1B8
:1092B0007C48ADF802207C4A90427CD2804641F244
:1092C0002105B8F80200B8F80020C0F30B07C2F37C
:1092D0000B04120BBE1D4FF000098DF8082002048C
:1092E000ADF80460ADF806408DF8099000F1C38038
:1092F00006338B4200F2398101AE0DF10A0B344680
:1093000001E0A34513D0079B14F8011B03F12802C9
:109310006A440133042B079302F8101CF1D106A90B
:1093200003A8F9F7BBFCA345CDE90790EBD1089B57
:10933000002BC0F21A81BDF8024016F8013B08224A
:1093400084EA032423B2002B4FEA4404B6BF85EA23
:109350004303A4B29CB2013AF4D1B345EDD1D8F89D
:1093600004603A46314603A8FEF73EF90028C0F2F1
:10937000FC80F019864213D0711E013811F8013FAC
:10938000082284EA032423B2002B4FEA4404B6BF28
:1093900085EA4303A4B29CB2013AF4D18142EDD1F3
:1093A000DDE90302ADF8024011463F4A08F1140816
:1093B0009045034685D302334FF000089942ADF83B
:1093C0000480C0F0D28001AD2E460DF106042F4678
:1093D00001E0BC4213D0079B17F8011B03F12802E0
:1093E0006A440133042B02F8101C0793F1D106A93B
:1093F00003A8F9F753FCBC42CDE90780EBD1089BE9
:10940000002BC0F2B280BDF8023041F2210016F804
:10941000012B83EA0223082219B200294FEA4303F1
:10942000B6BF80EA41019BB28BB2013AF4D1B4429B
:10943000EDD10399ADF80230049B0231994200F25C
:1094400094800DF10206144602E0B54200F08A80D5
:10945000079B16F8011B03F128026A440133042B11
:1094600002F8101C0793F0D106A903A8F9F716FC1F
:10947000CDE90740E9E7CB460BF1010B06335FFA74
:109480008BFB99428DF809B06FD301AE0DF10A0A3A
:1094900034460DE000000E0800001008003C0240B9
:1094A00001000E08C0790908747F0908A24515D08B
:1094B000079914F801CB01F128030DEB03000131EA
:1094C0000429079100F810CCF0D106A903A8F9F7F8
:1094D000E5FB0023A24508900793E9D1089A002AEA
:1094E00043DBBDF8024016F8012B082184EA022470
:1094F00022B2002A4FEA4404B6BF85EA4202A4B26F
:1095000094B20139F4D1B245EDD1D8F8041001EB91
:1095100009063A46314603A8FEF766F8002824DB20
:10952000F019864213D0711E013811F8013F08224C
:1095300084EA032423B2002B4FEA4404B6BF85EA31
:109540004303A4B29CB2013AF4D18142EDD1DDE9EA
:109550000302BBF1030FADF8024003461146B944C4
:109560008AD121E7089B002B09DA00200BB0BDE867
:10957000F08F1548506000F18830506078E6079809
:1095800040B912490A6942F000420A61B3FA83F015
:109590004009EBE7DDE9033203449342E5D806AB2B
:1095A000C0F10402002118447AF080FD06A903A846
:1095B000F9F774FB002803460890D6DB9DF82420B9
:1095C000002AE3D0DDE700BF23016745003C0240ED
:1095D00008B5FFF739FE40B9FFF736FE28B9FFF7A7
:1095E00033FE10B9052007F0CBFDFFF7B9FD0028C9
:1095F000F8D008BD70B545880B460446C5F30B0589
:109600002A46002118467AF051FD0A4A2169914202
:10961000034606D3084A914206D3BDE87040184677
:1096200008470029F9D170BD2A46BDE8704079F09D
:109630001BBC00BF747F09089384090810B5037927
:10964000012B84B08E460ED0022B02D0002004B035
:1096500010BD8368DB0758BF01F07F0104B0BDE88F
:109660001040FDF7EBBF144682688DF80F4002F002
:10967000010201920DF10F020092417C90F910005D
:109680007246FAF7C3FF04B010BD00BFF8B57822E8
:10969000074600210068FFF7D1FF052607F014FDFB
:1096A00004460D4607F010FD001B61EB0501B0F507
:1096B0007A7F71F10001F5D3013EEFD138682022A5
:1096C0000121FFF7BBFF052607F0FEFC04460D460F
:1096D00007F0FAFC001B61EB0501B0F57A7F71F130
:1096E0000001F5D3013EEFD1324638680221FFF781
:1096F000A5FF642607F0E8FC04460D4607F0E4FCED
:10970000001B61EB0501B0F57A7F71F10001F5D323
:10971000013EEFD10120F8BD70B52422044641215D
:109720000068FFF78BFF90B9052607F0CDFC0446D3
:109730000D4607F0C9FC001B61EB0501B0F57A7F0F
:1097400071F10001F5D3013EEFD1012070BD206819
:1097500020223021FFF772FF0028E5D02068062282
:109760003121FFF76BFF0028DED020680022342172
:10977000FFF764FFD8E700BFF8B5072207460A21C4
:109780000068FFF75BFF052607F09EFC04460D46C8
:1097900007F09AFC001B61EB0501B0F57A7F71F1CF
:1097A0000001F5D3013EEFD1386824224121FFF7B3
:1097B00045FF052607F088FC04460D4607F084FCAB
:1097C000001B61EB0501B0F57A7F71F10001F5D363
:1097D000013EEFD13868C0224221FFF72FFF052656
:1097E00007F072FC04460D4607F06EFC001B61EBAF
:1097F0000501B0F57A7F71F10001F5D3013EEFD19B
:109800000120F8BD10B50446002221210068FFF7B1
:1098100015FF2068FC222021FFF710FF206840225E
:109820002421FFF70BFF20680C222321FFF706FFFE
:10983000206800222221FFF701FF012010BD00BF98
:10984000F8B50122074610210068FFF7F7FE00B9BE
:10985000F8BD142607F038FC04460D4607F034FC2A
:10986000001B61EB0501B0F57A7F71F10001F5D3C2
:10987000013EEFD13868A022BDE8F8401121DDE6B5
:1098800010B5044600680379012B84B011D0022B77
:1098900002D0002004B010BD01220B21FDF7CEFE46
:1098A0000028F6D020681D22092104B0BDE8104030
:1098B000C4E6826890F910C0417C8DF80F3002F048
:1098C000010201920DF10F02009260460B22FAF79D
:1098D0009DFEE5E72DE9F041802207460B21006857
:1098E000FFF7ACFE1E26804607F0EEFB04460D4651
:1098F00007F0EAFB001B61EB0501B0F57A7F71F11F
:109900000001F5D3013EEFD1B8F1000F02D10020E4
:10991000BDE8F081386806222921FFF78FFE002874
:10992000F5D0386808220B21FFF788FE0028EED01A
:109930003868CF22BDE8F0410A217FE610B5044621
:1099400094220B210068FFF779FE20687122012123
:10995000FFF774FE206800220421FFF76FFE2068E5
:10996000C8220521FFF76AFE206800220621FFF7C2
:1099700065FE2068C8220721FFF760FE20680022EC
:109980000821FFF75BFE2068C8220921FFF756FE79
:10999000012010BD10B50446C06900B110BD0921F9
:1099A0001420FEF7C5FEE06110BD00BF10B5174CD6
:1099B00004EB8000406830B300EB400004EB800310
:1099C00093F931CCBCF1FF3F1ED093F8390CD0B1E4
:1099D00004EB0C0293F8380C92F884EC8C231421DD
:1099E00003FB0CFC00220CEB000304EB43030139E6
:1099F000B3F8883C704412FA83F2F4D1044BA3FB11
:109A00000230C0F30F1010BD002010BD005F002019
:109A1000CDCCCCCC70B5104B104CA3421AD205461D
:109A200002E00C33A34215D293F805C08C45F8D15F
:109A300093F804C0AC4501D0002DF2D1D879904202
:109A4000EFD1186890F804E0E645EAD106689E4236
:109A5000E7D170BD002070BD94840908A486090870
:109A60000379022B00D0704710B490F910201C4CE1
:109A70001C4883B00831694402EB8202009450F81C
:109A8000222011F8084C18498A4224D0A1F57841C7
:109A90008A4222D001F580618A4218D1118821F0D2
:109AA0004001090403EB8303090C118000EB8300E0
:109AB0001388C16823F0380331F824101B041B0CF1
:109AC0000B43138013889BB243F04003138003B011
:109AD0005DF8044B70470023E0E70123DEE700BF99
:109AE00000010203500C002000300140F8B504686A
:109AF000002107462046FFF7B3FFB6221421204677
:109B0000FFF79CFD642607F0DFFA04460D4607F0D8
:109B1000DBFA001B61EB0501B0F57A7F71F1000102
:109B2000F5D3013EEFD1812210213868FFF786FD81
:109B300007F0CAFA04460D4607F0C6FA001B61EBAF
:109B40000501B0F57A7F71F10001F5D3802215216E
:109B50003868FFF773FD07F0B7FA04460D4607F0C3
:109B6000B3FA001B61EB0501B0F57A7F71F10001DA
:109B7000F5D338680321BDE8F84071E7F8B504680B
:109B8000002107462046FFF76BFFB6227E212046C4
:109B9000FFF754FD642607F097FA04460D4607F0D8
:109BA00093FA001B61EB0501B0F57A7F71F10001BA
:109BB000F5D3013EEFD1324638687C21FFF73EFDF8
:109BC000642607F081FA04460D4607F07DFA001B73
:109BD00061EB0501B0F57A7F71F10001F5D3013E2B
:109BE000EFD1386804227D21FFF728FD642607F0B5
:109BF0006BFA04460D4607F067FA001B61EB05019E
:109C0000B0F57A7F71F10001F5D3013EEFD18C22DE
:109C100040213868FFF712FD07F056FA04460D465A
:109C200007F052FA001B61EB0501B0F57A7F71F184
:109C30000001F5D3022241213868FFF7FFFC07F04D
:109C400043FA04460D4607F03FFA001B61EB05019D
:109C5000B0F57A7F71F10001F5D338680221FFF782
:109C6000FFFE4FF40063BB81F8BD00BF2DE9F0415A
:109C7000076882B08046B6227E213846FFF7DEFCB8
:109C8000642607F021FA04460D4607F01DFA001B72
:109C900061EB0501B0F57A7F71F10001F5D3013E6A
:109CA000EFD102213846FFF7DBFE7B6913B11A685A
:109CB0009B88538307F008FA04460D4607F004FA20
:109CC000001B61EB0501B0F57A7F71F10001F5D35E
:109CD0007B6913B11A689B8813830A2607F0F4F98D
:109CE00004460D4607F0F0F9001B61EB0501B0F5E5
:109CF0007A7F71F10001F5D3013EEFD132467C212C
:109D00003846FFF79BFC07F0DFF904460D4607F0E5
:109D1000DBF9001B61EB0501B0F57A7F71F1000101
:109D2000F5D3002259213846FFF788FC07F0CCF91B
:109D300004460D4607F0C8F9001B61EB0501B0F5BC
:109D40007A7F71F10001F5D397F91030BA688E4926
:109D500003EB83035E20920751F823408DF8070040
:109D600040F1E48001230DF107020021204673F049
:109D700081F84FF4A473854A2046002173F07AF8E5
:109D8000BB689B0740F1E6800A2607F09DF9044670
:109D90000D4607F099F9001B61EB0501B0F57A7FDC
:109DA00071F10001F5D3013EEFD10122592138466E
:109DB000FFF744FC07F088F904460D4607F084F9E4
:109DC000001B61EB0501B0F57A7F71F10001F5D35D
:109DD0008C2240213846FFF731FC07F075F9044624
:109DE0000D4607F071F9001B61EB0501B0F57A7FB4
:109DF00071F10001F5D3032241213846FFF71EFC23
:109E000007F062F904460D4607F05EF9001B61EBAE
:109E10000501B0F57A7F71F10001F5D35C4CD8F8FB
:109E2000382098F83500B4FBF2F2032391B2594A76
:109E3000FEF756FD4388B4FBF3F4C8F840400279BE
:109E4000422142F0C0023846FFF7F8FB07F03CF928
:109E500004460D4607F038F9001B61EB0501B0F52B
:109E60007A7F71F10001F5D3082243213846FFF7CC
:109E7000E5FB07F029F904460D4607F025F9001B1C
:109E800061EB0501B0F57A7F71F10001F5D3042291
:109E900058213846FFF7D2FB07F016F904460D4665
:109EA00007F012F9001B61EB0501B0F57A7F71F143
:109EB0000001F5D30A2253213846FFF7BFFB07F014
:109EC00003F904460D4607F0FFF8001B61EB05019E
:109ED000B0F57A7F71F10001F5D300227C2138467C
:109EE000FFF7ACFB07F0F0F804460D4607F0ECF87E
:109EF000001B61EB0501B0F57A7F71F10001F5D32C
:109F000006227D213846FFF799FB07F0DDF804466D
:109F10000D4607F0D9F8001B61EB0501B0F57A7F1B
:109F200071F10001F5D302B0BDE8F0817B6913B196
:109F30001A689B885383184B1849D3F81421184B7F
:109F40004868D200A3FB023292094B681B1A9A425E
:109F5000FBD207E7104B1149D3F81421104B486886
:109F60004FF4FA7404FB02F2A3FB023292094B682D
:109F70001B1A9A42FBD27B69002B3FF405AF1A688B
:109F80009B88138300E700BF500C0020C0540808D2
:109F900040420F0008560808005F0020001000E053
:109FA000D34D62102DE9F041836B07685A4A5B4D2F
:109FB000B5FBF3F10446062389B290F83500FEF7AD
:109FC0008FFC00214388B5FBF3F5804625643846B5
:109FD000FFF746FD80226B213846FFF72FFB6426F2
:109FE00007F072F804460D4607F06EF8001B61EBAF
:109FF0000501B0F57A7F71F10001F5D3013EEFD193
:10A00000032268213846FFF719FB642607F05CF845
:10A0100004460D4607F058F8001B61EB0501B0F54A
:10A020007A7F71F10001F5D3013EEFD101226B215E
:10A030003846FFF703FB0F2607F046F804460D46A7
:10A0400007F042F8001B61EB0501B0F57A7F71F172
:10A050000001F5D3013EEFD118221B213846FFF74E
:10A06000EDFA0F2607F030F804460D4607F02CF8FD
:10A07000001B61EB0501B0F57A7F71F10001F5D3AA
:10A08000013EEFD118221C213846FFF7D7FA0F26E0
:10A0900007F01AF804460D4607F016F8001B61EBAE
:10A0A0000501B0F57A7F71F10001F5D3013EEFD1E2
:10A0B00098F804201A213846FFF7C0FA0F2607F057
:10A0C00003F804460D4606F0FFFF001B61EB050197
:10A0D000B0F57A7F71F10001F5D3013EEFD198F828
:10A0E000052019213846FFF7A9FA642606F0ECFF8F
:10A0F00004460D4606F0E8FF001B61EB0501B0F5D4
:10A100007A7F71F10001F5D3013EEFD1384603218A
:10A11000BDE8F041A4E400BF1C56080840420F000F
:10A120002DE9F041836B0768654A664DB5FBF3F195
:10A130000446062389B290F83500FEF7D1FB0021D2
:10A140004388B5FBF3F5804625643846FFF788FC65
:10A1500080226B213846FFF771FA642606F0B4FFBF
:10A1600004460D4606F0B0FF001B61EB0501B0F59B
:10A170007A7F71F10001F5D3013EEFD1072268210A
:10A180003846FFF75BFA642606F09EFF04460D464C
:10A1900006F09AFF001B61EB0501B0F57A7F71F1C3
:10A1A0000001F5D3013EEFD132466B213846FFF76F
:10A1B00045FA642606F088FF04460D4606F084FF43
:10A1C000001B61EB0501B0F57A7F71F10001F5D359
:10A1D000013EEFD101226B213846FFF72FFA0F26FF
:10A1E00006F072FF04460D4606F06EFF001B61EBA1
:10A1F0000501B0F57A7F71F10001F5D3013EEFD191
:10A2000018221B213846FFF719FA0F2606F05CFFCB
:10A2100004460D4606F058FF001B61EB0501B0F542
:10A220007A7F71F10001F5D3013EEFD118221C2194
:10A230003846FFF703FA0F2606F046FF04460D46A0
:10A2400006F042FF001B61EB0501B0F57A7F71F16A
:10A250000001F5D3013EEFD198F804201A213846C9
:10A26000FFF7ECF90F2606F02FFF04460D4606F027
:10A270002BFF001B61EB0501B0F57A7F71F1000146
:10A28000F5D3013EEFD198F8052019213846FFF7A4
:10A29000D5F9642606F018FF04460D4606F014FFB3
:10A2A000001B61EB0501B0F57A7F71F10001F5D378
:10A2B000013EEFD138460321BDE8F041FFF7D0BBA6
:10A2C0001C56080840420F002AE700BFF0B504689A
:10A2D00083B0074600212046FFF7C2FB0C22252150
:10A2E0002046FFF7ABF90A2226213868FFF7A6F9C6
:10A2F000002263213868FFF7A1F9386881222721FD
:10A30000FFF79CF9142606F0DFFE04460D4606F022
:10A31000DBFE001B61EB0501B0F57A7F71F10001F6
:10A32000F5D3013EEFD10C2225213868FFF786F9DD
:10A330000A2226213868FFF781F90F226321386845
:10A34000FFF77CF9386881222721FFF777F90A2681
:10A3500006F0BAFE04460D4606F0B6FE001B61EBA1
:10A360000501B0F57A7F71F10001F5D3013EEFD11F
:10A37000032301AA102138466EF0E0F90A2606F000
:10A38000A3FE04460D4606F09FFE001B61EB05018F
:10A39000B0F57A7F71F10001F5D3013EEFD19DF860
:10A3A00004009DF805109DF806202C4B803080316C
:10A3B0008032A3F8D00FA3F8D21FA3F8D42F252101
:10A3C0000C223868FFF73AF90A2226213868FFF78D
:10A3D00035F9324663213868FFF730F93868812251
:10A3E0002721FFF72BF90A2606F06EFE04460D46DC
:10A3F00006F06AFE001B61EB0501B0F57A7F71F192
:10A400000001F5D3013EEFD10DF10302012302213A
:10A4100038466EF093F901230DF103020921384605
:10A420006EF08CF938680C222521FFF707F938689F
:10A430000A222621FFF702F9386812226321FFF76A
:10A44000FDF8812238682721FFF7F8F838680321E2
:10A45000FFF706FB012003B0F0BD00BF005F002046
:10A460002DE9F04105461F4695F91030244803EBCD
:10A470008303164650F82380AB689A070ED54046F2
:10A4800072F048FD3B4632460021404672F0F2FC35
:10A49000AB689B0719D50120BDE8F0816B6913B14A
:10A4A0001A689B885383174B174AD3F814314FEA25
:10A4B000C30E164BA2FB0E2E5A684FEA9E1E5C6816
:10A4C000A4EB020CE645FAD2D9E70E4B0F49D3F8BC
:10A4D00014210D4B4FF4FA7000FB02F2A3FB023281
:10A4E000486892094B681B1A9A42FBD26B69002B91
:10A4F000D1D01A689B8813830120BDE8F08100BF8A
:10A50000500C0020005F0020D34D6210001000E0CE
:10A5100030B50579012D83B08E460DD0022D02D0C5
:10A52000002003B030BD8468E40758BF41F08001CB
:10A5300003B0BDE8304093E714468268009402F00F
:10A540000102417C90F9100001927246FAF75EF820
:10A5500003B030BD2DE9F04105461F4695F9103096
:10A56000244803EB8303164650F82380AB689A0710
:10A570000ED5404672F0CEFC3B46002231464046A6
:10A5800072F078FCAB689B0719D50120BDE8F0811B
:10A590006B6913B11A689B885383174B174AD3F81A
:10A5A00014314FEAC30E164BA2FB0E2E5A684FEA27
:10A5B0009E1E5C68A4EB020CE645FAD2D9E70E4B6E
:10A5C0000F49D3F814210D4B4FF4FA7000FB02F23F
:10A5D000A3FB0232486892094B681B1A9A42FBD2CD
:10A5E0006B69002BD1D01A689B8813830120BDE8CA
:10A5F000F08100BF500C0020005F0020D34D62109E
:10A60000001000E030B50579012D83B08E460DD0E5
:10A61000022D02D0002003B030BD8468E40758BF8B
:10A6200041F0800103B0BDE8304093E714468268F2
:10A63000009402F00102417C90F9100001927246F0
:10A64000F9F7B0FF03B030BD2DE9F043836B076825
:10A65000804A814CB4FBF3F185B08046062389B271
:10A6600090F83500FEF73CF900214388B4FBF3F481
:10A670008146C8F840403846FFF7F2F980226B2146
:10A680003846FEF7DBFF962606F01EFD04460D4613
:10A6900006F01AFD001B61EB0501B0F57A7F71F140
:10A6A0000001F5D3013EEFD1032268213846FEF7C1
:10A6B000C5FF962606F008FD04460D4606F004FD8B
:10A6C000001B61EB0501B0F57A7F71F10001F5D354
:10A6D000013EEFD103226B213846FEF7AFFF06F0B3
:10A6E000F3FC04460D4606F0EFFC001B61EB050190
:10A6F0000F2871F10001F6D310226A213846FEF7C7
:10A700009DFF06F0E1FC04460D4606F0DDFC001B53
:10A7100061EB05010F2871F10001F6D300226C21D5
:10A720003846FEF78BFF06F0CFFC04460D4606F0D8
:10A73000CBFC001B61EB05010F2871F10001F6D382
:10A7400099F8052019213846FEF778FF06F0BCFC81
:10A7500004460D4606F0B8FC001B61EB05010F280E
:10A7600071F10001F6D318221B213846FEF766FF6F
:10A7700006F0AAFC04460D4606F0A6FC001B61EBA1
:10A7800005010F2871F10001F6D318221C2138466B
:10A79000FEF754FF06F098FC04460D4606F094FCC4
:10A7A000001B61EB05010F2871F10001F6D399F848
:10A7B00004201A213846FEF741FF06F085FC0546C5
:10A7C0000C4606F081FC8C4208BF8542F9D003217B
:10A7D0003846FFF745F9D8F800000623432102AABE
:10A7E000FFF710FF28B3BDF80810BDF80A30BDF818
:10A7F0000C20C9BA07EE901ADBBAD2BAF8EEE76AB3
:10A8000007EE102A07EE903AB8EEC77AF8EEE77A2C
:10A81000C8ED076AC8ED087A88ED097AFDEEE77A97
:10A82000CDED017A9DF90430013305D005B0BDE8C6
:10A83000F083D8ED087AF1E7D8ED077AFDEEE77AF4
:10A84000CDED017A9DF904300133EFD1062006F0F9
:10A8500097FC00BF1C56080840420F0008B500686E
:10A860000379022B0BBF114A114A07230623042147
:10A87000FFF7C8FE0F4B93F8DB1F93F8DACF93F87E
:10A88000DE2F090441EA0C2193F8D9CF41EA0C01EB
:10A8900093F8DDCFC3F88810120442EA0C2293F833
:10A8A000DCCF42EA0C0201201A6608BDD86E0020F7
:10A8B000D96E0020005F002010B5044600680379BF
:10A8C00082B0022B0CBF4321032106236A46FFF707
:10A8D00099FE68B1BDF80010BDF80220BDF8043043
:10A8E00049BA52BA5BBAE1866287238702B010BDCB
:10A8F000C4F83600608702B010BD00BF2DE9F047F4
:10A90000164F97F8E13F824689466BB9DAF80000A6
:10A9100097F8E23F00244A46492187F8E14FFFF7C4
:10A9200071FE0120BDE8F08706F0CEFBD7F8E83FC6
:10A93000C51AC5F5FA55002DE8DD06F0C5FB4FEA4E
:10A94000E57804460E4606F0BFFB001B61EB0601EE
:10A95000A84271EB0801F6D3D8E700BF005F0020E2
:10A960002DE9F041624C0546D4F8F00FC5F83600E9
:10A9700094F8E03FB4F8F42F6A87012B82B076D0C8
:10A98000022B0FD0002B69D10122022128466EF044
:10A990003DFD012394F8F66F84F8E03F304602B0A5
:10A9A000BDE8F08194F8E13F05F1360804F57F67D2
:10A9B000002B6ED169462846FFF7A0FF9DF80630B0
:10A9C000064600284AD01B0748D4B4F8D02FBDF85B
:10A9D000003013FB02F3474A93427DDBB3F5000FCF
:10A9E0006FDA002BB8BFFF331B125B421BB2B4F807
:10A9F000D22FEB86BDF8023013FB02F33D4A93429F
:10AA00006EDBB3F5000F6FDA002BB8BFFF3343F3F3
:10AA10000F23B4F8D42F2B87BDF8043013FB02F3B7
:10AA2000344A93425ADBB3F5000F5BDA002BB8BF10
:10AA3000FF331B125B421BB2D5F83600C4F8F00F8F
:10AA40006B87B8F80430BB8000220123304684F8BD
:10AA5000E02F84F8F63F02B0BDE8F08100263046D2
:10AA600084F8E06F84F8F66F02B0BDE8F08194F8E6
:10AA7000E13F94F8F66FD3B969462846FFF73EFFE9
:10AA80009DF8003008B19A071DD1002384F8E03FFB
:10AA900084E706F019FBD4F8E83FC01AB0F5FA5F76
:10AAA00088DA94F8F66F304602B0BDE8F08106F01F
:10AAB0000BFBD4F8E83FC01AB0F5FA5FFFF66EAFB3
:10AAC000DAE70D4B93E70722032128466EF09EFC40
:10AAD000022384F8E03F61E7084B88E7074BABE7C8
:10AAE000064B96E7044BA7E747F6FF7391E700BFD5
:10AAF000005F002001FF7FFF0180FFFF0080FFFF5C
:10AB000010B5044600680179012984B02AD00229D1
:10AB100002D0002004B010BD836813F0010F02AA18
:10AB20004FF0060308BF8221FFF714FD0028F0D084
:10AB3000BDF9083006EE903ABDF90A3007EE103A3A
:10AB4000BDF90C3007EE903AF8EEE66AB8EEC77A37
:10AB5000F8EEE77AC4ED076A84ED087AC4ED097A65
:10AB600004B010BD8368417C90F9100003F001032C
:10AB7000019302AB009302220623F9F713FDD5E7F8
:10AB800030B5044600680379012B85B014D0022B40
:10AB90000FD1826802AD12F0010F18BF03212A46BF
:10ABA00008BF8321FFF7D6FC18B19DF90930002BAF
:10ABB00010DB002005B030BD8368417C90F91000A7
:10ABC00003F0010302AD0193009502230322F9F77C
:10ABD000E9FCE9E7206807232A461221FFF712FD66
:10ABE0000028E6D09DF90A209DF809309DF90C1047
:10ABF00043EA022313EB430248BF03329DF80B30B4
:10AC0000921043EA012307EE902A13EB4302F8EE79
:10AC1000E77A48BF03329DF90E109DF80D30C4ED60
:10AC2000047A921007EE902A43EA012313EB4303C0
:10AC3000F8EEE77A48BF03339B10C4ED057A07EEC0
:10AC4000903AF8EEE77AC4ED067AB3E770B5066895
:10AC5000F46982B00546002C3FD03379012B04F112
:10AC600004022DD0022B26D1B36813F0010F4FF050
:10AC70000C03304614BF19468C21FFF76BFCA07003
:10AC8000D8B1B4F9043007EE903AF8EEE77AC5EDA2
:10AC9000077AB4F9063007EE903AF8EEE77AC5ED98
:10ACA000087AB4F9083007EE903AF8EEE77AC5ED85
:10ACB000097A02B070BD0023A370002002B070BDFD
:10ACC000B368717C96F91000009203F001030193C0
:10ACD0000C231A46F9F766FCD1E709211420FDF789
:10ACE00027FDF06104462E68B7E700BF70B506681F
:10ACF000F46982B00546002C3FD03379012B04F172
:10AD000003022DD0022B26D1B36813F0010F304679
:10AD10004FF00D0314BF0C218C21FFF71BFCA0701A
:10AD2000D8B1B4F90A3007EE903AF8EEE77AC5EDFB
:10AD3000077AB4F90C3007EE903AF8EEE77AC5EDF1
:10AD4000087AB4F90E3007EE903AF8EEE77AC5EDDE
:10AD5000097A02B070BD0023A370002002B070BD5C
:10AD6000B368717C96F91000009203F0010301931F
:10AD70000C220D23F9F716FCD1E709211420FDF769
:10AD8000D7FCF06104462E68B7E700BF10B5006835
:10AD90000379012B84B00C461AD0022B02D000207C
:10ADA00004B010BD836813F0010F03AA4FF0030332
:10ADB00014BF2221A221FFF7CDFB0028EFD0BDF95F
:10ADC0000D3003EB83031B12E633238004B010BD68
:10ADD0008368417C90F9100003F00103019303ABF9
:10ADE000009322220323F9F7DDFBE6E710B50446C2
:10ADF00000680379012B84B02DD0022B01D00020F4
:10AE000027E0836813F0010F02AA4FF0060314BF76
:10AE10001F219F21FFF79EFB0028F0D0BDF80810EE
:10AE2000BDF80A20BDF80C30C9BA07EE901AD2BAA4
:10AE3000F8EEE76A07EE902ADBBAB8EEE77A07EE9B
:10AE4000903AF8EEE77AC4ED046A84ED057AC4ED31
:10AE5000067A04B010BD8368417C90F9100003F0BD
:10AE60000103019302AB00931F220623F9F79AFB1B
:10AE7000D2E700BF10B5044600680379012B84B007
:10AE80002DD0022B01D0002027E0836813F0010FA2
:10AE900002AA4FF0060314BF2521A521FFF75AFB94
:10AEA0000028F0D0BDF80810BDF80A20BDF80C301D
:10AEB000C9BA07EE901AD2BAF8EEE76A07EE902AFE
:10AEC000DBBAB8EEE77A07EE903AF8EEE77AC4ED2F
:10AED000076A84ED087AC4ED097A04B010BD83686E
:10AEE000417C90F9100003F00103019302AB009341
:10AEF00025220623F9F756FBD2E700BF10B50068FC
:10AF00000379012B84B00C4625D0022B01D0002000
:10AF10001FE0826812F0010F18BF1D2103AA08BFAD
:10AF20009D21FFF717FB0028F1D0BDF80C309FEDF5
:10AF3000116ADFED116ADBBA07EE903AB8EEE77AF4
:10AF4000C7EE067A77EEA67AFDEEE77A17EE903A2C
:10AF5000238004B010BD8368417C90F9100003F099
:10AF60000103019303AB00931D220223F9F71AFB9F
:10AF7000D9E700BFCFF7534100007A4370B50668A8
:10AF8000F46982B00546002C3FD03379012B04F1DF
:10AF900004022DD0022B26D1B36813F0010F3046E6
:10AFA0004FF00E0314BF3B21BB21FFF7D3FAA07073
:10AFB000D8B1A389DBBA07EE903AF8EEE77AC5ED8F
:10AFC000077AE389DBBA07EE903AF8EEE77AC5ED47
:10AFD000087A238ADBBA07EE903AF8EEE77AC5EDF5
:10AFE000097A02B070BD0023A370002002B070BDCA
:10AFF000B368717C96F91000009203F0010301938D
:10B000003B220E23F9F7CEFAD1E709211420FDF7F0
:10B010008FFB0446F061B8E700B500680379012BA7
:10B0200085B011D0022B01D000200AE003AAF6213E
:10B03000FFF790FA0028F7D0BDF80C30094A5BBA48
:10B04000938205B05DF804FB8368417C90F91000A1
:10B0500003AA03F00103CDE900230223F622F9F746
:10B06000A1FAE7E7005F002000B500680379012B33
:10B0700085B01ED0022B01D0002017E0032303AAC5
:10B08000F621FFF767FA0028F6D09DF80D309DF8FD
:10B090000CC00F499DF80E201B0243EA0C431343DA
:10B0A000B1F93420C2F10802D3408B6305B05DF8DA
:10B0B00004FB8368417C90F9100003AA03F00103AC
:10B0C000CDE900230323F622F9F76CFADBE700BF92
:10B0D000005F002000B500680379012B85B033D0F4
:10B0E000022B0AD01F49D1F8F83FD1F8FC2FCA63D0
:10B0F0000020CB6505B05DF804FB062302AAF7210A
:10B10000FFF728FA0028EDD09DF809309DF808C017
:10B110009DF80C209DF80A109DF80BE01B0143EAF6
:10B120000C3312019DF80DC043EA111342EA0E32AE
:10B130000C4942EA1C12C1F8F83FC1F8FC2FCA635F
:10B14000CB6505B05DF804FB8368417C90F9100085
:10B1500002AA03F00103CDE900230623F722F9F741
:10B1600021FACFE7005F002000B500680379012BCA
:10B1700085B01ED0022B10D09DF80D309DF80C002C
:10B180009DF80E10124A1B0243EA00430B430120B4
:10B19000C2F8B03005B05DF804FB836813F0010F0E
:10B1A00003AA4FF0030314BF00218021FFF7D2F957
:10B1B000E2E78368417C90F9100003AA03F00103E1
:10B1C000CDE9002303230022F9F7ECF9D4E700BF0F
:10B1D000005F002000B500680379012B85B01ED008
:10B1E000022B10D09DF80D309DF80C009DF80E102C
:10B1F000124A1B0243EA00430B430120C2F8C43049
:10B2000005B05DF804FB836813F0010F03AA4FF04B
:10B21000030314BF00218021FFF79CF9E2E7836854
:10B22000417C90F9100003AA03F00103CDE900234B
:10B2300003230022F9F7B6F9D4E700BF005F00202E
:10B2400010B500680379012B84B029D0022B01D0FE
:10B25000002023E0836813F0010F4FF0030303AADB
:10B2600014BF19468321FFF775F90028F0D09DF827
:10B270000C309DF90C109DF80D209DF80EC01B049C
:10B28000002943EA0223A8BF00210C4AB8BF4FF0AF
:10B290007F4143EA0C030B43C2F8F83004B010BD01
:10B2A0008268417C90F9100002F0010203AC032394
:10B2B000CDE900421A46F9F775F9D6E7005F00209C
:10B2C00000B500680379012B85B02AD0022B01D08C
:10B2D000002023E0836813F0010F03AA4FF003035B
:10B2E00014BF00218021FFF735F90028F0D09DF828
:10B2F0000C309DF90C109DF80D209DF80EC01B041C
:10B30000002943EA0223A8BF00210D4AB8BF4FF02D
:10B310007F4143EA0C030B43C2F8F43005B05DF8FB
:10B3200004FB8368417C90F9100003AA03F0010339
:10B33000CDE9002303230022F9F734F9D5E700BF54
:10B34000005F002010B5044600680379012B84B02B
:10B3500043D0022B07D0002213461046C4F83620F3
:10B36000638704B010BD836813F0010F02AA4FF089
:10B37000060314BF11219121FFF7ECF80028EAD051
:10B38000BDF90820BDF90A3006EE902A5B42BDF9EE
:10B390000C2007EE103AF8EEE66AB7EE086A07EE00
:10B3A000902A66EE866AB8EEC77AFDEEE66A27EE68
:10B3B000067AF8EEE77A16EE903A67EE867ABDEEF8
:10B3C000C77AFDEEE77AE38617EE103A238717EE89
:10B3D000903A1BB2638704B010BD8368417C90F93A
:10B3E000100003F00103019302AB00931122062326
:10B3F000F9F7D8F8C2E700BF10B50446002300688B
:10B40000C4F8363063870379012B84B022D0022B35
:10B4100001D000201CE0836813F0010F02AA4FF056
:10B42000060314BF03218321FFF794F80028F0D00E
:10B43000BDF90A30BDF80810BDF80C205B4201EBE5
:10B44000410103EB430302EB4202E186238762875B
:10B4500004B010BD8368417C90F9100003F0010333
:10B46000019302AB009303220623F9F79BF8DDE773
:10B4700010B504464FF0000C0068C4F836C0A4F8BC
:10B480003AC00379012B84B018D0022B01D00020E0
:10B4900012E0836813F0010F02AA4FF0060314BFF5
:10B4A00061468021FFF756F80028F0D0029ABDF8D7
:10B4B0000C30C4F83620638704B010BD836890F95F
:10B4C00010E0417C03F00103019302AB009362465C
:10B4D00006237046F9F766F8E6E700BF10B584B0BA
:10B4E0000023044600680293CDF80B300279012A4C
:10B4F0001ED0022A19D1836813F0010F02AA4FF05F
:10B50000070314BF4E21CE21FFF724F8BDF8091020
:10B51000BDF80B20BDF80D30C9BAD2BADBBA012094
:10B52000E1862287638704B010BD1A461946F6E704
:10B53000836890F910C0417C02AA03F001030092D5
:10B5400001934E2207236046F9F72CF8DEE700BF8F
:10B5500070B50446234894F9103003EB8303154675
:10B5600050F82360A3689A070DD5304671F0D2FCDD
:10B57000012300222946304671F07CFCA3689B071A
:10B5800017D5012070BD636913B11A689B88538376
:10B59000154B164AD3F8143150684FEAC30C144BBC
:10B5A000A3FB0C3C4FEA9C1C53681B1A9C45FBD226
:10B5B000DBE70D4B0D49D3F814210D4B4FF4FA7016
:10B5C00000FB02F2A3FB0232486892094B681B1A87
:10B5D0009A42FBD26369002BD3D01A689B881383ED
:10B5E000012070BD500C0020005F0020001000E022
:10B5F000D34D621010B50379012B82B08E460DD069
:10B60000022B02D0002002B010BD8368DB0758BFB8
:10B6100041F0800102B0BDE8104099E7144682680D
:10B62000009402F00102417C90F9100001927246F0
:10B63000F8F7B8FF02B010BD70B505682B79012B83
:10B6400084B004460E4616D0022B02D0002004B06F
:10B6500070BDAB68E122DB074CBF11466121284673
:10B66000FBF7ECFF0028F1D020683246FF2104B040
:10B67000BDE87040BEE7AA68697C95F9100002F049
:10B6800001020DF10F0501920095E1228DF80F20C6
:10B69000F8F7BCFFE6E700BF70B505682B79012B12
:10B6A00084B004460E4617D0022B02D0002004B00E
:10B6B00070BDAB68DB074FF0C3024CBFE1216121D5
:10B6C0002846FBF7BBFF0028F0D020683246FF2158
:10B6D00004B0BDE870408DE7AA6895F91000697C58
:10B6E00002F0010201920DF10F020092C3228DF8C7
:10B6F0000F20E122F8F78AFFE5E700BF70B5056883
:10B700002B79012B84B004460E461CD0022B02D0AC
:10B71000002004B070BDAB68DB074FF0F0024CBFF7
:10B72000E12161212846FBF789FF0028F0D022465D
:10B73000FF2152F8040BFFF75DFF0028E8D02379C2
:10B74000337004B070BDAA6895F91000697C02F0EE
:10B75000010201920DF10F020092F0228DF80F20EC
:10B76000E122F8F753FFE0E7F0B5046883B0002169
:10B7700007462046FEF774F915227E212046FDF784
:10B780005DFF642605F0A0FC04460D4605F09CFC18
:10B79000001B61EB0501B0F57A7F71F10001F5D373
:10B7A000013EEFD1386811227E21FDF747FF0526C3
:10B7B00005F08AFC04460D4605F086FC001B61EB93
:10B7C0000501B0F57A7F71F10001F5D3013EEFD1AB
:10B7D00038680DF107020321FFF70CFF9DF80730D1
:10B7E00003F03C03142B40F09B800C22402138686E
:10B7F000FDF724FF05F068FC04460D4605F064FCE7
:10B80000001B61EB0501B0F57A7F71F10001F5D302
:10B81000BB6B454C454AB4FBF3F197F8350009235F
:10B8200089B2FDF75DF8034642215A88B4FBF2F471
:10B830003C641A793868FDF701FF05F045FC0446C1
:10B840000D4605F041FC001B61EB0501B0F57A7F68
:10B8500071F10001F5D3082241213868FDF7EEFEB1
:10B8600005F032FC04460D4605F02EFC001B61EB92
:10B870000501B0F57A7F71F10001F5D30022432173
:10B880003868FDF7DBFE05F01FFC04460D4605F0A9
:10B890001BFC001B61EB0501B0F57A7F71F1000123
:10B8A000F5D3102251213868FDF7C8FE05F00CFCD5
:10B8B00004460D4605F008FC001B61EB0501B0F5E0
:10B8C0007A7F71F10001F5D30A2253213868FDF720
:10B8D000B5FE05F0F9FB04460D4605F0F5FB001B2F
:10B8E00061EB0501B0F57A7F71F10001F5D380229B
:10B8F00056213868FDF7A2FE05F0E6FB04460D462A
:10B9000005F0E2FB001B61EB0501B0F57A7F71F1F8
:10B910000001F5D338680321FEF7A2F803B0F0BDAB
:10B92000062005F02DFC00BF40420F0040560808DD
:10B930002DE9F043836B0768A04AA14CB4FBF3F1F7
:10B9400083B08046052389B290F83500FCF7C8FF24
:10B9500000214388B4FBF3F48146C8F840403846E0
:10B96000FEF77EF8002276213846FDF767FE0F22AB
:10B970004E213846FDF762FE0F2605F0A5FB044672
:10B980000D4605F0A1FB001B61EB0501B0F57A7FC8
:10B9900071F10001F5D3013EEFD199F805204F2157
:10B9A00002F00F023846FDF749FE0F2605F08CFB2A
:10B9B00004460D4605F088FB001B61EB0501B0F560
:10B9C0007A7F71F10001F5D3013EEFD199F805209E
:10B9D000502102F00F023846FDF730FE0F2605F029
:10B9E00073FB04460D4605F06FFB001B61EB050180
:10B9F000B0F57A7F71F10001F5D3013EEFD1FF225E
:10BA000052213846FDF71AFE0F2605F05DFB04466D
:10BA10000D4605F059FB001B61EB0501B0F57A7F7F
:10BA200071F10001F5D3013EEFD198F835100729E7
:10BA300041D0644D95F8180CFCF7A8FF044601228C
:10BA400076213846FDF7FAFDA2780C213846FDF73D
:10BA5000F5FD22790D213846FDF7F0FDA279A38886
:10BA6000120142EA1322D2B20E213846FDF7E6FD5A
:10BA70004FF4807195F8180CFCF788FF04460222F9
:10BA800076213846FDF7DAFDA2785200032102F054
:10BA9000FE023846FDF7D2FD227904213846FDF733
:10BAA000CDFDA279A388120142EA13220521D2B268
:10BAB0003846FDF7C3FD002276213846FDF7BEFD6E
:10BAC000032214213846FDF7B9FD0F2605F0FCFAD4
:10BAD00004460D4605F0F8FA001B61EB0501B0F5D0
:10BAE0007A7F71F10001F5D3013EEFD13246632137
:10BAF0003846FDF7A3FD642605F0E6FA04460D4638
:10BB000005F0E2FA001B61EB0501B0F57A7F71F1F7
:10BB10000001F5D3013EEFD1082265213846FDF73B
:10BB20008DFD64210DF107023846FFF763FD9DF896
:10BB3000072022F0100242F06002642138468DF89E
:10BB40000720FDF77BFD0F2605F0BEFA04460D46E3
:10BB500005F0BAFA001B61EB0501B0F57A7F71F1CF
:10BB60000001F5D3013EEFD10DF106024D2138461B
:10BB7000FFF740FD9DF8062002F03F0242F0400230
:10BB80004D2138468DF80620FDF758FD0F2605F0AB
:10BB90009BFA04460D4605F097FA001B61EB050180
:10BBA000B0F57A7F71F10001F5D3013EEFD10321A9
:10BBB0003846FDF755FF03B0BDE8F0837856080816
:10BBC00040420F00005F0020F0B583B015460DF134
:10BBD00007021C4606460F46FFF70CFD9DF807209E
:10BBE00005EA0203A34201D103B0F0BD22EA050237
:10BBF00022433946304603B0BDE8F040FDF71EBD94
:10BC000010B582B004466A4600680821FFF7F2FCCE
:10BC10009DF80030DB0602D4002002B010BD206881
:10BC200006236A460021FEF7EDFC0028F4D09DF8BB
:10BC300001309DF800109DF802209FED4B6A1B0219
:10BC400003EB01439DF804101C029DF803401A44C5
:10BC50004FEA01219DF8053001EB044148BF02F194
:10BC60007F420B4407EE902A090248BF03F17F434D
:10BC7000B8EEE77A07EE903AF8EEE77AC7EE066A92
:10BC80003A4BB3F99820B3F99E10C7EE863A07EE07
:10BC9000102A374A93ED256A12F8F84CB3F99A2026
:10BCA000D3ED247AF8EEC65A06EE102AB3F99C209A
:10BCB00005EE102AB3F9A02004EE901A04EE102A23
:10BCC000B8EEC77A112CF8EEE77AB8EEC66AB8EE8D
:10BCD000C55AF8EEE44AB3F9A210B3F9A420B8EEBD
:10BCE000C44A27EE237A26EEA32A23D0A6EE845A4E
:10BCF000A6EEA46AE5EE265AE5EEA67A77EE877AF6
:10BD0000E6EE027AB3F98E2007EE102AB3F98C2002
:10BD1000C3ED2A7A06EE902AB8EEC77AF8EEE66A04
:10BD200027EE237AB6EE006AA6EE867A83ED2B7AAA
:10BD300002B010BD03EE102AF8EEC32A03EE101A6B
:10BD4000A6EEA24AB8EEC33AA4EE265AE6EE834A1D
:10BD5000E5EE265AA4EEA66AE5EEA67A77EE877A95
:10BD6000E6EE027ACEE700BF00007848005F0020D0
:10BD7000F86F0020F0B5002283B007460A21006862
:10BD8000FDF75CFC142605F09FF904460D4605F00E
:10BD90009BF9001B61EB0501B0F57A7F71F10001A1
:10BDA000F5D3013EEFD138680F220A21FDF746FC9A
:10BDB0000A2605F089F904460D4605F085F9001BB1
:10BDC00061EB0501B0F57A7F71F10001F5D3013E19
:10BDD000EFD13868032301AA1021FEF713FC0A26CD
:10BDE00005F072F904460D4605F06EF9001B61EB93
:10BDF0000501B0F57A7F71F10001F5D3013EEFD175
:10BE00009DF804209DF805009DF80610194B80321E
:10BE10008030803123F8F42C23F8F20C324623F8DA
:10BE2000F01C38680A21FDF709FC0A2605F04CF9D8
:10BE300004460D4605F048F9001B61EB0501B0F51D
:10BE40007A7F71F10001F5D3013EEFD10DF10302CC
:10BE500038680221FFF7CEFB0DF103023868092193
:10BE6000FFF7C8FB386811220A21FDF7E7FB012024
:10BE700003B0F0BDF86F0020F0B5002283B0074694
:10BE80000A210068FDF7DAFB142605F01DF90446C7
:10BE90000D4605F019F9001B61EB0501B0F57A7F3D
:10BEA00071F10001F5D3013EEFD138680F220A216C
:10BEB000FDF7C4FB0A2605F007F904460D4605F018
:10BEC00003F9001B61EB0501B0F57A7F71F1000108
:10BED000F5D3013EEFD13868032301AA1021FEF704
:10BEE00091FB0A2605F0F0F804460D4605F0ECF843
:10BEF000001B61EB0501B0F57A7F71F10001F5D30C
:10BF0000013EEFD1324638680A21FDF797FB0A2639
:10BF100005F0DAF804460D4605F0D6F8001B61EB93
:10BF20000501B0F57A7F71F10001F5D3013EEFD143
:10BF30000DF1030238680221FFF75CFB0DF10302EB
:10BF400038680921FFF756FB386801220A21FDF7FE
:10BF500075FB012003B0F0BD30B5002385B0044669
:10BF6000C0F8363043870DF1070200680221FFF761
:10BF700041FB18B19DF80730DB0703D400252846A4
:10BF800005B030BD062302AA03212068FEF73AFB64
:10BF900020680DF107020921FFF72CFB0546002858
:10BFA000ECD09DF8073013F00C0FE7D1BDF8082056
:10BFB000BDF80C30BDF80A102068C2EB8232C3EB2A
:10BFC00083339B0092008900E286218763870122E8
:10BFD0000A21FDF733FB284605B030BDF0B583B02C
:10BFE000002307468DF80230142605F06DF804464C
:10BFF0000D4605F069F8001B61EB0501B0F57A7F8D
:10C0000071F10001F5D3013EEFD131460DF102028D
:10C010003868FFF7EFFA0DF1020280213868FFF768
:10C02000E9FA4FF4F842ADF8042038688DF806605C
:10C03000032301AA6021FEF76BFA142605F044F8E9
:10C0400004460D4605F040F8001B61EB0501B0F514
:10C050007A7F71F10001F5D3013EEFD131460DF148
:10C06000030238688DF80360FFF7C4FA4CF26243AC
:10C07000ADF8043004238DF806303868032301AA94
:10C080006021FEF745FA142605F01EF804460D4619
:10C0900005F01AF8001B61EB0501B0F57A7F71F12C
:10C0A0000001F5D3013EEFD131460DF103023868AE
:10C0B0008DF80360FFF79EFA4FF4E853ADF80430B3
:10C0C00008238DF80630386801AA03236021FEF7A3
:10C0D0001FFA142604F0F8FF04460D4604F0F4FF9E
:10C0E000001B61EB0501B0F57A7F71F10001F5D31A
:10C0F000013EEFD10DF10302314638688DF803603F
:10C10000FFF778FA38680DF102021E21FFF772FA84
:10C11000012003B0F0BD00BFF0B5044683B00D466A
:10C120001746061D20680379012B1AD0022B02D076
:10C13000002003B0F0BD8368DB0732464FF0FF01FB
:10C140005CBF3246FF21FFF703FA0028F0D015B19B
:10C150002379DB07E6D4002FEBD023793B7003B0C3
:10C16000F0BD8268417C90F9100002F00102CDE937
:10C170000062FF22F8F716FAE7E700BF30B5044681
:10C18000051D20680379012B83B017D0022B02D044
:10C19000002003B030BD8368DB072A464FF0FF0163
:10C1A0005CBF2A46FF21FFF7D3F90028F0D023799E
:10C1B000DB07EED520680379012BE7D18268417C4B
:10C1C00090F9100002F00102CDE90052FF22F8F7C9
:10C1D000E9F9EAE730B50246044652F8040B037960
:10C1E000012B83B00ED0022B01D0002008E0FF21EC
:10C1F000FFF7AEF90028F8D02079C04300F0010025
:10C2000003B030BD8568417C90F91000009205F0C4
:10C2100001050195FF22F8F7C5F9EBE730B5B42227
:10C2200083B00446FF210068FDF708FA10B900202A
:10C2300003B030BD20680379012B04F1040514D04C
:10C24000022BF4D18368DB072A464FF0FF015CBF65
:10C250002A46FF21FFF77CF90028E8D02379DB0785
:10C26000E6D520680379012BEAD18268417C90F9F8
:10C27000100002F00102CDE90052FF22F8F792F916
:10C28000EAE700BF30B50A4683B00446A52100683E
:10C29000FDF7D4F910B9002003B030BD2068037950
:10C2A000012B04F1040514D0022BF4D18368DB07C1
:10C2B0002A464FF0FF015CBF2A46FF21FFF748F9ED
:10C2C0000028E8D02379DB07E6D520680379012B25
:10C2D000EAD18268417C90F9100002F00102CDE9B8
:10C2E0000052FF22F8F75EF9EAE700BF70B582B0AE
:10C2F000CDE900230446FFF791FF10B9002002B0FA
:10C3000070BD20685522A521FDF798F90028F5D0C9
:10C31000251D20682A46FF21FFF76CF90028EDD083
:10C320002379DB07F5D40DF1FF350DF1070615F87C
:10C33000011F2046FFF7A6FF0028DFD0B542F6D147
:10C34000DDE700BF002A35D0F0B5044683B00E46C5
:10C350008F18051D16F8012B2068A521FDF76EF931
:10C3600090B9002003B0F0BD8268417C90F91000C4
:10C3700002F00102CDE90052FF22F8F713F900287C
:10C38000EFD02379DB0710D520680379012BEBD0A0
:10C39000022BE6D18368DB072A464FF0FF015CBF22
:10C3A0002A46FF21FFF7D4F8E9E7B742D2D10120AE
:10C3B00003B0F0BD0120704770B5962282B00446EC
:10C3C0000E460068FF21FDF739F910B9002002B0D0
:10C3D00070BD251D20680379012B1FD0022BF5D1DC
:10C3E0008368DB072A464FF0FF015CBF2A46FF2126
:10C3F000FFF7AEF80028E9D02379DB07EAD4E12281
:10C4000020681146FDF71AF90028DFD0206832466F
:10C41000FF2102B0BDE87040FFF7ECB88268417CB4
:10C4200090F9100002F00102CDE90052FF22F8F766
:10C43000B9F8DFE7002A43D0F0B5044683B00E46D2
:10C440008F18051D20689622FF21FDF7F7F890B997
:10C45000002003B0F0BD8268417C90F9100002F02A
:10C460000102CDE90052FF22F8F79CF80028EFD036
:10C470002379DB0710D520680379012BEBD0022B41
:10C48000E6D18368DB072A464FF0FF015CBF2A46EE
:10C49000FF21FFF75DF8E9E7E12220681146FDF78B
:10C4A000CDF80028D4D020683246FF21FFF7A2F84B
:10C4B0000028CDD00136B742C4D1012003B0F0BD71
:10C4C0000120704770B505460B460446164655F8E0
:10C4D000040B82B087211A46FDF7B0F82068037973
:10C4E000012B1AD0022B02D0002002B070BD83684D
:10C4F000DB072A464FF0FF015CBF2A46FF21FFF70A
:10C5000027F80028F0D02379DA07E7D4002EECD002
:10C51000C3F34013337002B070BD8268417C90F960
:10C52000100002F00102CDE90052FF22F8F73AF8BC
:10C53000E7E700BF70B5782182B004461646006870
:10C540000022FDF77BF810B9002002B070BD251D58
:10C5500020680379012B14D0022BF5D18368DB0707
:10C560002A464FF0FF015CBF2A46FF21FEF7F0FF8D
:10C570000028E9D02379DA07EAD45B09337002B0E6
:10C5800070BD8268417C90F9100002F00102CDE993
:10C590000052FF22F8F706F8EAE700BF30B5CC22D8
:10C5A00083B00446A5210068FDF748F810B90020C3
:10C5B00003B030BD20680379012B04F1040514D0C9
:10C5C000022BF4D18368DB072A464FF0FF015CBFE2
:10C5D0002A46FF21FEF7BCFF0028E8D02379DB07BD
:10C5E000E6D520680379012BEAD18268417C90F975
:10C5F000100002F00102CDE90052FF22F7F7D2FF4E
:10C60000EAE700BF30B5B42283B00446FF210068DA
:10C61000FDF714F810B9002003B030BD251D2068C7
:10C620000379012B22D0022BF5D18368DB072A4640
:10C630004FF0FF015CBF2A46FF21FEF789FF00286B
:10C64000E9D02379DA07EAD4CC212046FFF71AFE95
:10C650000028E0D002E02379DB07DDD520682A46F8
:10C66000FF21FEF7C7FF0028F5D1D4E78268417C9F
:10C6700090F9100002F00102CDE90052FF22F7F715
:10C6800091FFDCE72DE9F04F8BB0CDE9072304469D
:10C69000002004908A460390251D049B079A20469B
:10C6A000DE0002EBC30BFFF7B9FD20B935E02379BB
:10C6B00013F0010207D020682A46FF21FEF79AFFF7
:10C6C0000028F4D129E005929A07099040F1D8801A
:10C6D000F0212046FFF7D6FDF8B1079BDDF8148066
:10C6E000083E3344012606933746BAF1000F54D072
:10C6F000082F52D807F1FF394AFA09F909F0010960
:10C7000020684FEAC9127821FCF798FF28B1206809
:10C710000379012B50D0022B06D00020089B049AED
:10C720001A700BB0BDE8F08F8368DB072A464FF024
:10C73000FF015CBF2A46FF21FEF70AFF0028ECD06C
:10C74000237913F00102E2D1C3F3801CD9099B06BF
:10C7500046D5BCF1000F60D1BAF1000F5AD0082FB6
:10C7600058D8894540F08880B9F1000F48D01BF8AF
:10C77000083033430BF808307600013716F0FF0617
:10C78000FFB2B2D108F101085FFA88F8B8F1080FDA
:10C7900043D00126BAF1000FAAD1049BC3B1039B79
:10C7A000BB4215D9069B13F808301E4214BF4FF048
:10C7B00001094FF00009A3E78268417C90F910005D
:10C7C00002F00102CDE90052FF22F7F7EBFEB5E7D8
:10C7D000039BA3EB0709B9FA89F94FEA59198FE7C7
:10C7E000BAF1000F13D0082F11D8894596D1B9F1AD
:10C7F000000FBCD1059BBCF1000F08BF3B46059361
:10C800001BF8083023EA06030BF80830B4E70029C8
:10C81000ADD1EFE70029AAD1F2E7402F06D8089B57
:10C82000049A1B7893423FF638AF77E79BF807707E
:10C830000BF1FF360BF1060B16F801CF082182EA47
:10C840000C0343F30003013923F0730383EA52021C
:10C8500011F0FF01D2B24FEA5C0CF0D1B345EBD13D
:10C860009742DCD1049B0133DBB20493059B002B80
:10C870003FF454AF0393D2E7DDF8248040464DE700
:10C88000804640464AE700BF30B504460068037959
:10C89000012B85B062D0022B03D00025284605B0BD
:10C8A00030BD826802AD12F0010F18BF19462A464A
:10C8B00008BF8221FEF74CFE0028EED09DF808301C
:10C8C000DA07EAD52A46206807230321FDF79AFEF6
:10C8D00005460028E1D0206811220A21FCF7AEFEAF
:10C8E0009DF80E301B07D8D42A49BDF8083031F81E
:10C8F000F42C13FB02F3284A93423FDBB3F5000FFD
:10C900003ADA002BB8BFFF331B125B421BB2BDF8F3
:10C910000A20E38631F8F23C12FB03F31E4A9342ED
:10C9200030DBB3F5000F31DA002BB8BFFF3343F330
:10C930000F22BDF80C3031F8F01C2287164A13FB89
:10C9400001F393421CDBB3F5000F1DDA002BB8BFD7
:10C95000FF331B125B421BB263879FE7826890F92B
:10C9600010C0417C02F0010202AD019200956046C8
:10C970000222F7F717FE9FE7084BC8E7084BC6E708
:10C98000074BE9E7064AD4E7044BE5E747F6FF72B1
:10C99000CFE700BFF86F002001FF7FFF0180FFFF9E
:10C9A0000080FFFF10B5044686B0006800238DF8B4
:10C9B0000F300379012B31D0022B02D0002006B0BA
:10C9C00010BD8368D9070DF10F024CBF2721A721A5
:10C9D000FEF7BEFD0028F1D09DF80F301B07EDD506
:10C9E0002068062304AA2821FDF70CFE28B3BDF910
:10C9F0001030BDF91220002BB8BF03339B10E38623
:10CA0000BDF91430002AB8BF0332002BB8BF03337E
:10CA100092109B102287638706B010BD826890F940
:10CA200010C0417C02F0010201920DF10F02009250
:10CA300060462722F7F7B6FDCCE7C4F836006087DA
:10CA40000020BCE730B504464FF0000C0068C4F885
:10CA500036C0A4F83AC00379012B87B02AD0022B44
:10CA600002D0002007B030BD8368D9070DF10F0256
:10CA70004CBF61468021FEF76BFD0028F1D09DF888
:10CA80000F301B07EDD52068062304AA0121FDF70E
:10CA9000B9FD0028E5D0BDF81430BDF81010BDF880
:10CAA00012205BBA49BA52BA5B42E1862287638799
:10CAB00007B030BD8568417C90F9100005F0010594
:10CAC00001950DF10F0562460095F7F76BFDD4E770
:10CAD00010B5044600230068C4F836306387037934
:10CAE000012B86B023D0022B02D0002006B010BD4F
:10CAF0008368D9070DF10F024CBF06218621FEF78E
:10CB000027FD0028F1D09DF80F305B07EDD5206898
:10CB1000062304AA0021FDF775FD0028E5D0049A3C
:10CB2000BDF81430C4F83620638706B010BD8268A3
:10CB300090F910C0417C02F0010201920DF10F0248
:10CB4000009260460622F7F72DFDDAE710B504469D
:10CB500000230068C4F8363063870379012B86B060
:10CB600029D0022B02D0002006B010BD8368D9075F
:10CB70000DF10F024CBF09218921FEF7E9FC0028C5
:10CB8000F1D09DF80F30DB07EDD52068062304AA0D
:10CB90000121FDF737FD0028E5D0BDF81210BDF8E2
:10CBA0001020BDF81430494252425B42E186228790
:10CBB000638706B010BD826890F910C0417C02F016
:10CBC000010201920DF10F02009260460922F7F76F
:10CBD000E9FCD4E710B5044600230068C4F83630F9
:10CBE00063870379012B86B012D0022B0DD18368A5
:10CBF000DB070DF10B024CBF3421B421FEF7A8FC7A
:10CC000018B19DF90B30002B11DB002006B010BDD0
:10CC1000826890F910C0417C02F0010201920DF18E
:10CC20000B02009260463422F7F7BCFCE8E720686C
:10CC3000092303AA2421FDF7E5FC0028E5D09DF88F
:10CC400010209DF80F109DF81330120442EA016283
:10CC5000C2F30F429DF8121022871B049DF80D208D
:10CC600043EA01639DF80C10120442EA0162C2F328
:10CC70000F42C3F30F43E286638706B010BD00BFC7
:10CC800010B50368DA6B82B0044612B1904740B128
:10CC900023685B6B1BB1214601A8984718B9FF2395
:10CCA000E38202B010BDBDF80630013B9BB2F7E74E
:10CCB000F0B5044683B018460D4616461F4670F080
:10CCC000B7FB2844D4F800C0A073E67320460024C4
:10CCD0000094DCF814403B4632462946A04703B096
:10CCE000F0BD00BF38B58B68016004460D4698471B
:10CCF00000230B4A226123752B6B13B12046984702
:10CD00002075084B13F8EC3C1BB1237D23F0010385
:10CD100023750023E3822046BDE83840B0E700BF1A
:10CD20000001FF00F86F002010B5154B53F8E84CD8
:10CD300084B084B12379012B10D0022B0BD1A168D0
:10CD400011F00101024618BF8021204604B0BDE861
:10CD50001040FAF773BC002004B010BDA268617CDB
:10CD60008DF80F0002F0010294F910000DF10F048C
:10CD7000CDE900428022F7F749FC04B010BD00BFA6
:10CD8000F86F0020F0B5294B53F8E85C85B09DB1F1
:10CD9000B02280212846FCF751FC40228021284601
:10CDA000FCF74CFC002280212846FCF747FC1022AF
:10CDB00080212846FCF742FC4FF480642DB9013CE9
:10CDC000A4B2002CFBD105B0F0BD00270DF10F0679
:10CDD0002B79012B08D0022B04F1FF3217D094B22B
:10CDE000002CF0D0012BF6D1AA6895F91000697CCF
:10CDF0008DF80F7002F00102013CCDE90062A4B28F
:10CE00004022F7F703FC002CE2D105B0F0BDAA6880
:10CE1000013C12F0010218BF002240212846A4B2B2
:10CE2000FAF70CFC002CD3D105B0F0BDF86F002050
:10CE30000B4B10B553F8E84C8CB15038C2B280217E
:10CE40002046FCF7FBFB002280212046FCF7F6FB86
:10CE500020461022BDE810408021FCF7EFBB10BD3A
:10CE6000F86F0020F0B5264B264C53F8E85C2038CC
:10CE700000EB8000661D85B00444064425B90134EA
:10CE8000A642FCD105B0F0BD0DF10F072B79227839
:10CE9000012B1BD0022B0AD00134A642F7D100226D
:10CEA0004021284605B0BDE8F040FCF7C7BBAB68A1
:10CEB000DB074FF04001284619D50134FAF7BEFBD5
:10CEC000A642E3D1002DEAD105B0F0BD8DF80F20C8
:10CED000AA6895F91000697C02F00102CDE90072A0
:10CEE00001344022F7F792FBB442CFD1D7E70134A7
:10CEF000FAF7A4FBB442C9D1002DE5D0CFE700BFBB
:10CF0000F86F002098560808F0B5754B53F8E85CA8
:10CF100085B0002D00F09680D42280212846FCF7B1
:10CF20008DFB802211462846FCF788FBA822802131
:10CF30002846FCF783FB3F2280212846FCF77EFB36
:10CF4000D32280212846FCF779FB00228021284645
:10CF5000FCF774FB402280212846FCF76FFB8D22F2
:10CF600080212846FCF76AFB142280212846FCF722
:10CF700065FBA12280212846FCF760FBC8228021A6
:10CF80002846FCF75BFBDA2280212846FCF756FB9B
:10CF9000122280212846FCF751FB8122802128465D
:10CFA000FCF74CFBCF2280212846FCF747FBD92217
:10CFB00080212846FCF742FBF12280212846FCF71D
:10CFC0003DFBDB2280212846FCF738FB40228021F4
:10CFD0002846FCF733FBA42280212846FCF72EFBD1
:10CFE000A62280212846FCF729FBAF228021284673
:10CFF000FCF724FBA62280212846FCF71FFBAE226B
:10D0000080212846FCF71AFB202280212846FCF7C5
:10D0100015FB002280212846FCF710FBB02280215E
:10D020002846FCF70BFB402280212846FCF706FB34
:10D03000002280212846FCF701FB1022802128468F
:10D04000FCF7FCFA4FF4806435B9013CA4B2002C23
:10D05000FBD1012005B0F0BD00270DF10F062B79A3
:10D06000012B2AD0022B04F1FF3214D094B2002CF1
:10D07000F6D1812280212846FCF7E0FAC8228021DF
:10D080002846FCF7DBFAAF2280212846FCF7D6FAC7
:10D09000012005B0F0BDAA68013C12F0010218BFE2
:10D0A000002240212846A4B2FAF7C8FA002CD6D1B3
:10D0B000002DDED1012005B0F0BDAA6895F9100061
:10D0C000697C8DF80F7002F00102013CCDE900622D
:10D0D000A4B24022F7F79AFA002CC0D1C9E700BFEA
:10D0E000F86F0020FAF75CBDFAF75ABDFAF758BDA1
:10D0F000FAF756BDFAF754BDFAF752BD0120704752
:10D10000034620B1026812B1D26902B1104793ED13
:10D11000017A084BB8EEC77A53ED386AF6EE007A1A
:10D12000E7EE267AFDEEE77A17EE900A00F30B00A1
:10D13000704700BFF86F0020034620B1026812B1AB
:10D14000126A02B1104793ED027A084BB8EEC77A23
:10D1500053ED376AF6EE007AE7EE267AFDEEE77ACF
:10D1600017EE900A00F30B00704700BFF86F002025
:10D17000034628B102681AB1516A09B19369184788
:10D1800093ED037A074BB8EEC77A53ED366AF6EEA5
:10D19000007AE7EE267AFDEEE77A17EE900A00F3C2
:10D1A0000B007047F86F002010B5044630B10368DB
:10D1B00023B1DB6813B1BDE81040184703F084FFCA
:10D1C000D4E904239042994134BF0120002010BDCE
:10D1D000F8B170B506680F4B06F13F4202F57E02CA
:10D1E00003EB92230C4682B0054693F82C056BF0B6
:10D1F000BDFFC4F34112C4F30013A9883046CDE942
:10D200000032C4F3810304F003026FF0F3FB02B0B9
:10D2100070BD704710540808B0B3F0B507681B4BD9
:10D22000144607F13F4202F57E0203EB92230546C6
:10D2300083B093F82C050E466BF098FFA988B1FADD
:10D2400081F3C3F11F03C3F3CC0207EB820203F0A7
:10D250000703156A4FF00F0C9B009C400CFA03F378
:10D2600025EA03031362136A1C431462C6F3001316
:10D270007209CDE900323846C6F3810306F0030295
:10D280006FF0B8FB03B0F0BD704700BF1054080842
:10D2900010B50409013C032C19D80F4A00F00F0304
:10D2A00032F8140040FA03F212F0010211D0012208
:10D2B00002FA03F3013B184077F0B4FE074B084A2B
:10D2C0001B5D184400EB400002EB800010BD002005
:10D2D00010BD104610BD00BF0854080804540808CB
:10D2E0002C2B00202DE9F04F542204460021C34886
:10D2F00091B076F0DBFEC24A611EE01C144611F8C4
:10D30000013F5D1E052D88BF0023814244F8043B88
:10D31000F5D102F11003114651F8040B012800F079
:10D3200058819942F8D1114651F8040B022800F0B7
:10D3300046819942F8D1114651F8040B032800F0B8
:10D3400052819942F8D152F8041B042900F02D8132
:10D350009A42F8D10520F9F749FC0620DFF89C92A3
:10D36000DFF8BC82F9F742FC4C464FF01A0A00265F
:10D3700008F2345B277B57B3384694F90D50FFF71A
:10D3800087FF28B105238371002380F807A003726B
:10D390001321FFF71DFF00231BF83310B9422FD0D4
:10D3A0000133102BF8D10021964B216105EB450587
:10D3B00003EBC5050122D5F8D43923751344C5F80C
:10D3C000D4390723A375627585F8D02916440AF16C
:10D3D000010A5FFA8AFABAF1200F04F10C04C9D1EC
:10D3E0005EB1894D894F00262B7C73B90136032E1F
:10D3F00005F1180507F58C77F6D111B0BDE8F08F6F
:10D4000008EBC303D3F83815CEE768796BF0AEFEAE
:10D4100028796BF0ABFED5F808A05046F6F754FA21
:10D42000D5F814802C680397142303FB08F30593A5
:10D430000023CDE90C33CDE90E3304930693EB685A
:10D44000019304F14C034FF4806202934FF40063A4
:10D45000CDE907234FF400514FF48073CDE9091350
:10D4600050464FF4003301A90B936BF053FEDAF8EA
:10D4700000206749674B42F00102CAF800204A6861
:10D48000134043F440334B606368B8F1010F23F05D
:10D490004073D4BF0022012223F4807343EA0223A5
:10D4A0006360A2685C4B134043F00203A360E36A2D
:10D4B00008F1FF385FFA88F823F4700343EA085351
:10D4C000E36209F148014B4601204FFA86FC02E075
:10D4D0000C338B4231D05A7D002AF9D093F90D20BC
:10D4E0006245F5D11A7C93F816A0092A36D802EBCA
:10D4F000420BD4F810800AFA0BFE4FF0070A0AFA22
:10D500000BFA28EA0A084EEA080EC4F810E00628CA
:10D5100037D800F1FF3ED4F834800EEB8E0E4FF07A
:10D520001F0A02FA0EF20AFA0EFE28EA0E0E42EA6C
:10D530000E0262630130C0B2CAE7A36843F400730D
:10D54000A360A36843F48073A360A36843F001035E
:10D55000A360A36843F08043A36047E7A2F10A0EEB
:10D56000D4F80C800EEB4E0E4FF0070B0AFA0EFAB1
:10D570000BFA0EFE28EA0E0E4AEA0E0EC4F80CE074
:10D58000C5E70C284ED8A0F1070ED4F830800EEB7A
:10D590008E0E4FF01F0A02FA0EF20AFA0EFE28EA69
:10D5A0000E0E42EA0E022263C4E71C4B93F8842C51
:10D5B0003021013283F8601C83F8842CCAE61749B5
:10D5C00091F8840C3524013081F8484C81F8840CA2
:10D5D000B1E6124991F8840C3424013081F83C4CB6
:10D5E00081F8840C9FE60D4991F8840C20240130C9
:10D5F00081F8544C81F8840CA5E600BF306B002004
:10D60000045F0020500C002010160020886B0020C2
:10D6100000230140E030FCFFFDF7FFC0005F002069
:10D6200010540808A0F10D0ED4F82C800EEB8E0ECD
:10D630004FF01F0A02FA0EF20AFA0EFE28EA0E0E48
:10D6400042EA0E02E26275E710B503681A79022A0F
:10D65000044603D000232371236010BD987AFFF79E
:10D6600017FE0028F6D040F61A610022C18002722F
:10D670002021FFF7ADFD00232371236010BD00BF03
:10D680002DE9F04FB04EB14CA64285B056D21D46A2
:10D6900002E00C36A64251D273798B42F9D133792C
:10D6A000834201D00028F4D1F3799342F1D1346858
:10D6B000002C43D000236360A360E36023616361B7
:10D6C000A361E36126603379237196F806B0C4F84C
:10D6D00008B0317AE160012B32D0022B2ED1F07AE2
:10D6E000FFF7D6FD96F90970A061B07A2774FFF7AD
:10D6F000CFFD06466061F0B1DFF8708207EB87016D
:10D70000BB0058F82190019308EB8101B9F1000F9B
:10D7100011D0887CE8B10E220023F2713372B5710A
:10D7200009213046FFF754FD3368B2881A8320463A
:10D7300005B0BDE8F08F2046FFF786FF0024F6E72E
:10D74000F07AFFF7A5FD727AB37A6374A061227450
:10D75000EDE791F808A050466BF008FD4FEA5A102B
:10D7600001210AF01F0A023801FA0AF1032808D839
:10D77000DFE800F0AA9EA402754B586920EA010177
:10D780005961BB00D91908EB810107F1010A4879F9
:10D79000FFF77EFD5FFA8AFA014620B180F808A003
:10D7A00040F60A30C880BB00D81908EB800002910F
:10D7B000C079FFF76DFD02990190034620B180F812
:10D7C00008A040F60A50D880BB00D81908EB8000AA
:10D7D00002918079FFF75CFD0299034620B180F841
:10D7E00008A040F60A40D880BA00D01908EB8000A3
:10D7F0001BF0040290F809A0CDE902230846524626
:10D8000068D04A21FFF708FD019852462A21FFF708
:10D8100003FD039B524618460A21FFF7FDFCBB009F
:10D82000DA1908EB820292F804B0BBF1000F61D163
:10D83000484A914571D0484A914563D0474A91453D
:10D8400000F0A180464A914500F09280454A9145FA
:10D850006ED0454A914500F0A180029BB9F80010B6
:10D86000002B01F441510CBF032200220A4342F471
:10D870004572A9F80020B9F81C2022F400621204B5
:10D88000120CA9F81C200722A9F81020B9F80020D2
:10D8900092B242F04002A9F80020BBF1000F20D163
:10D8A000BB003B4408EB8308012388F8123032E7C1
:10D8B000274B186A20EA0101196262E7244B1869B4
:10D8C00020EA010119615CE7214B586A20EA010155
:10D8D000596256E70A21FFF79FFC019852460A2138
:10D8E00095E75846FFF7D4FC0028D9D00268838812
:10D8F0001383D5E75846FFF7CBFC52460921FFF7C3
:10D900008BFC95E702F50032116A41F48041116207
:10D91000116A21F4804111629FE702F58432516A55
:10D9200041F480515162516A21F48051516294E76F
:10D9300002F56842516A41F480115162516A21F442
:10D940008011516289E700BF94840908A486090800
:10D95000003802400030014000380040003C0040E8
:10D96000003401400050014000540140500C0020A0
:10D9700002F58232516A41F400515162516A21F438
:10D980000051516269E702F5FE32116A41F400412B
:10D990001162116A21F4004111625EE702F56442EE
:10D9A000516A41F400115162516A21F4001151622F
:10D9B00053E700BF014B1B685B681847586F002096
:10D9C000024B1B6808309B68184700BF586F002047
:10D9D00001207047012070470120704701207047E7
:10D9E0000120704731B10C4BD3ED017AF8EEE77AA4
:10D9F000C1ED007A72B1084BDFED086A9B68A3F5B0
:10DA0000D543333B07EE903AF8EEE77A87EEA67AF5
:10DA100082ED007A704700BF586F00200000C842B6
:10DA2000012070470120704710B4414C002322466A
:10DA300092F90410012902F10C022DD00133052BBB
:10DA4000F6D12246002392F90410032902F10C02B8
:10DA500034D00133052BF6D1002394F90420052A94
:10DA600004F10C043FD00133052BF6D1314B1B6878
:10DA7000D9034ED5304B016803F1F00402E01433B2
:10DA8000A34246D01A689142F9D1DA68D201F6D59C
:10DA900001205DF8044B7047284A03EB430302EB77
:10DAA0008303DB68EBB1264A037992F83DC09C45BD
:10DAB000EED092F83C209A42C3D1E9E71F4A03EB2B
:10DAC000430302EB8303DB68002BC6D01D4A0379B6
:10DAD00092F83D109942DBD092F83C209A42BBD19B
:10DAE000D6E72246AFE7154A03EB430302EB830375
:10DAF000DB68002BBAD0144A037992F83D109942A2
:10DB0000C6D092F83C209A42C2D00A4B1B68D90377
:10DB1000B0D40379203BDBB2152B06D80B495DF856
:10DB2000044BD94001F0010070470020B1E700BF6D
:10DB3000646F0020B400001058160020586F0020B9
:10DB40002403002070050020BC07002001003100E4
:10DB50000C4B10B5844603F1F00E002002E01433A4
:10DB60009E450ED01A686245F9D1DA688A4218BF1C
:10DB7000D96000F1010403F1140318BFE0B29E451F
:10DB8000F0D110BD58160020704700BF044B40F282
:10DB9000FF7203EBC0039142A8BF11469980704702
:10DBA000A4600020112806D8044B03EB8003DB6C33
:10DBB0000BB19B6819602EF033BA00BF586F00207C
:10DBC000112806D8034B03EB8003DB6C0BB19B6879
:10DBD00019607047586F00200D4A92F8F03083B1F9
:10DBE0000C4B93F8941061B193F8951061B1D2F891
:10DBF000F4000022FA2883F89520A8BF4FF0FF30E8
:10DC000070476FF0010070476FF00200704700BF6F
:10DC100058160020586F00202DE9F041104C04F1F7
:10DC2000980884F899101746002502234246FF21E0
:10DC3000064684F89850FCF76BFC68B142463046C3
:10DC40000223FF21FCF7DEFC30B1B4F898305BBA58
:10DC500028463B80BDE8F0816FF00C00FAE700BF7A
:10DC6000586F00200C4B93F898218AB193F89921B2
:10DC70005AB10A49D1F8F8000022B0F5967F83F82E
:10DC80009921A8BF4FF0FF3070476FF00200704736
:10DC90006FF00100704700BF586F00205816002039
:10DCA000024BD3F89C315B68184700BF586F0020C7
:10DCB000024BD3F89C319B68184700BF586F002077
:10DCC000024BD3F89C31DB68184700BF586F002027
:10DCD000014BD3F8FC00704758160020054B93F811
:10DCE000A0311BB1044BD3F8000170476FF0010065
:10DCF000704700BF586F00205816002070B5324C96
:10DD000005460323006804F5D2720021FCF77AFC73
:10DD100058B96FF00103C4F8A8312C4AD4F8AC31DB
:10DD2000116832338B4245D370BDB4F8A43194F8F6
:10DD3000A6015BBA9BB207EE903AF8EEE77AF2EEF4
:10DD4000046A87EEA67A94F8A4310821BDEEC77A5A
:10DD500084ED6A7A4FFA83FCBCF1000F4FEA4C0263
:10DD6000A8BF5B0082F00702B4BFD3B2DBB20139B7
:10DD7000F0D194F8A521082153405AB2002AB8BF27
:10DD800052004FEA4303B6BF82F00702DBB2D3B2C0
:10DD90000139F2D19842C0D1D4F8A8312BB1D4F8CE
:10DDA000A8214FF6FF739A42B7D14FF0FF33C4F862
:10DDB000A831B2E7C4F8AC112868054ABDE8704044
:10DDC00001233121FCF7A4BB586F0020242A002036
:10DDD00008710020014BD3F8A8017047586F00204C
:10DDE000437A5A1C0344D2B242729972037A934224
:10DDF00000D97047002AFCD010B5044604F10A018E
:10DE0000D0E9003098470023637210BDF0B54B4D48
:10DE100095F8943083B03BB195F8B061012E04467B
:10DE200039D0022E57D00EB103B0F0BD01228021AF
:10DE30000068FBF703FC20680122FF21FBF7FEFBD3
:10DE4000324631462068FBF7F9FB95F8B12120688E
:10DE50009121FBF7F3FB314620680122FBF7EEFB33
:10DE600032462068FF21FBF7E9FB3246206880211B
:10DE7000FBF7E4FB314620680122FBF7DFFB304B68
:10DE800030491A6881F8F0000123C5F8B42185F8FB
:10DE9000B03103B0F0BD01AA00682A4F0021FDF7A0
:10DEA000A9FB9DF8043087F8F000DA073DD5D5F8D6
:10DEB000B831002BB8D0224AD5F8B411126892B20A
:10DEC000521A9342B0D24FF0FF320023C7F8F42029
:10DED00085F8B031A8E700681A4F01AA1321FDF7B1
:10DEE00089FB9DF8043087F8F0005B07DFD02068DD
:10DEF000334601AA1E21FCF785FBBDF804302068DB
:10DF000001220B215CBAFBF799FB0F4B87F8F0005D
:10DF1000A4B2A3FB0434E40801220023C7F8F440B0
:10DF200085F8952085F8B0317EE7054A022312680E
:10DF3000C5F8B42185F8B03176E700BF586F0020EE
:10DF4000242A002058160020CDCCCCCC30B503209C
:10DF500083B00D461446FBF729FD01909DB107EEF5
:10DF6000900A9FED0B7AF8EE677AF0EE006A67EEA2
:10DF7000877AB8EE047AA7EEA67ADFED067A67EE26
:10DF8000277AC5ED007A0CB1034B236003B030BD96
:10DF90006740533A00007A443313904300B5006859
:10DFA0000379012B85B00DD0022B07D1012303AAE1
:10DFB000FF21FCF7CFFA05B05DF804FB002005B0A7
:10DFC0005DF804FB8268417C90F9100002F00102C8
:10DFD000019203AA0092FF22F6F7E4FA05B05DF879
:10DFE00004FB00BF30B5044600680379012B85B0FF
:10DFF0002DD0022B0ED0224B6FF00102C3F8FC2073
:10E000002049214AD1F8BC3115683233AB422CD3B8
:10E0100005B030BD826812F0010F18BF512103AA6C
:10E0200008BFD121FCF796FA0028E4D0BDF80C30E7
:10E03000134A5BBA9BB2C2F8FC30D2F8FC30B3F59D
:10E04000C87FDDDD4FF0FF33C2F8FC30D8E78368CE
:10E05000417C90F9100003F00103019303AB00939E
:10E0600051220223F6F79EFADEE701F5E072C1F8CD
:10E07000BC51206800235121FCF74AFA05B030BD9D
:10E0800058160020586F0020242A002000B5006890
:10E090000379012B85B02DD0022B24D1826812F098
:10E0A000010F18BF002103AA08BF8021FCF752FA14
:10E0B0001B4B83F8A00198B1BDF80C305BBA9BB242
:10E0C000B3F5FA6F24D2174A1749A2FB0323DB08E2
:10E0D00007EE903AF8EEE77AFDEEE77AC1ED407A86
:10E0E00005B05DF804FB0E4B002283F8A02105B0BB
:10E0F0005DF804FB8368417C90F9100003AA03F0EB
:10E100000103CDE9002302230022F6F74BFACFE703
:10E11000054B4FF0FF32C3F8002105B05DF804FB5A
:10E12000586F0020CDCCCCCC5816002010B500681C
:10E130000379012B84B00C461FD0022B02D00020A3
:10E1400004B010BD826812F0010F18BF002103AAAD
:10E1500008BF8021FCF7FEF90028F0D05CB19DF8E3
:10E160000D309DF90C20DB0903EB830302EB8202E7
:10E1700003EB4203238004B010BD8368417C90F917
:10E18000100003F00103019303AB0093002202236C
:10E19000F6F708FAE0E700BF70B50668F56982B0E7
:10E1A0000446002D59D000232B7004230DEB0302ED
:10E1B0003046FF21FCF726FA10B9002002B070BDEE
:10E1C000206804236A46FF21FCF71CFA0028F4D0DB
:10E1D0009DF804309B09023B012BEED9BDF80430B9
:10E1E000BDF80620BDF80010BDF802605BBA43F62A
:10E1F000FF74C3F30D03A342DFD0002BDDD052BA6E
:10E20000C2F34A1240F2FF7C6245D6D0002AD4D035
:10E2100049BAC1F30D01A142CFD00029CDD076BAC1
:10E22000C6F34A166645C8D0002EC6D05C1A002C2C
:10E23000B8BF6442FF2CC0DC941B002CB8BF644202
:10E24000FF2CBADC0B445B1032445210C5F8053089
:10E250000123C5F801202B70B0E709211420FAF73B
:10E2600067FAF061054626689DE700BF70B506684D
:10E27000F0690D461446A0B3D0F80130CDB1D0F806
:10E2800005209FED1B7ADFED1B5ADFED1B6A07EEC1
:10E29000902AF8EE677AB7EE006A77EEC77A77EEE3
:10E2A000A77A87EEA57A77EE467A67EEE67AC5ED2D
:10E2B000007AACB107EE903A9FED107ADFED106A6C
:10E2C0009FED106AF8EEE77A67EE877A87EEA67A16
:10E2D000DFED0D6A77EE467A77EEA67AC4ED007A26
:10E2E00070BD09211420FAF723FAF061C4E700BFDA
:10E2F0009AC9CC449AC94C460E76D745000048438B
:10E3000000E0FF44000048423393884370B506683C
:10E31000F46982B0F4B10023237004230DEB0302EF
:10E32000FF213046FCF76EF910B39DF804309B09CD
:10E3300019D1BDF80420BDF8063052BA5BBA92B2CA
:10E34000C3F34A1301212170C4F80520C4F8013039
:10E3500002B070BD054609211420FAF7E9F9F06111
:10E3600004462E68D7E7044A04210320FAF75AF935
:10E37000002002B070BD00BF50FD080870B50668EF
:10E38000F06982B00D461446002848D0D0F8053018
:10E39000DFED266A9FED267A07EE903AF8EE677A6F
:10E3A000D0F8013077EEE67AF3EE096A67EE877A05
:10E3B000B2EE047A67EEA67AF4EEC77AF1EE10FABE
:10E3C00020DCBAEE047AF4EEC77AF1EE10FA19D432
:10E3D0002DB19FED187A67EE877AC5ED007A7CB192
:10E3E00007EE903A9FED146ADFED146AB8EE677A93
:10E3F000DFED137AE7EE067A77EEA67AC4ED007ABF
:10E4000002B070BD17EE900A6FF07EF90D4ACDE9AB
:10E41000000104210320FAF705F902B070BD0921BB
:10E420001420FAF785F9F061B0E700BF000000465C
:10E43000000080380AD778430319C83D33938843D6
:10E44000000048C274FD0808F0B52DED028B4E4E59
:10E4500016F83C3C022B83B00D46144619D0DFED74
:10E460004B7A7DB19FED4A7A9FED4A6ADFED4A6AA9
:10E4700067EEA77A67EE877A87EE867A77EE267A56
:10E48000C5ED007A0CB1454B236003B0BDEC028BA7
:10E49000F0BD434B96F820105B6803F0020239BBD5
:10E4A0005B0525D42AB3B6F9463007EE903AB6F9A3
:10E4B0004430F8EEE77A06EE903A27EEA77AF8EEC7
:10E4C000E66AB6F94830A6EEA67A07EE903AF8EE7C
:10E4D000E77AA7EEA77AB5EEC07AF1EE10FABEDBC6
:10E4E000F1EEC77AF4EE677AF1EE10FAB9D7B6E733
:10E4F0001AB9336ED3ED337AB3E72A4F0DF1060024
:10E500002CF068FBBDF80630D7F8AC259FED266AE5
:10E51000DFED266A9FED267A9B1A07EE903AF8EE19
:10E52000E77AB0EE408A67EE867AA7EEA67AFDEE2D
:10E53000C77AB0EE470A17EE903A2033402B1FD827
:10E54000F9F7B8FE1B4B97F8D211D6ED0B7AA3F171
:10E550002C021846443B002918BF134693ED057A58
:10E56000D0ED006A77EE877AE8EE406A27EEA77A68
:10E57000A6EEA67AB5EEC07AF1EE10FAB0DA6EE742
:10E580009FED020ADEE700BF50800020000000007F
:10E59000CDCC9C3F00409C4682E6C5473313904358
:10E5A000B4000010586F00200AD7233C35FA8E3C87
:10E5B000DB0FC93F1875002010B50B4B82B053F824
:10E5C000304001916CB107EE901A94ED047A94ED0D
:10E5D000030AF8EEE77AA7EE870A70F0C9FCA36891
:10E5E000186002B010BD00BFA46000202DE9F0410A
:10E5F000DFF8BC802C4E2D4D41F0010284B000218B
:10E600000446FBF71BF8D8F80070C6F8B47119E09F
:10E61000022B3FD1A368DB070DF10F024FF013016E
:10E6200020465EBF0DF10F0293212046FCF790FFBC
:10E630009DF80F3085F8F00013F0070319D1D6F8D4
:10E64000B8214ABB2379012BE2D1A268617C94F9FD
:10E65000100002F0010201920DF10F02009213224C
:10E66000F5F7A0FF9DF80F3085F8F00013F00703D1
:10E67000E5D001220B212046FAF7E0FF00221146E7
:10E680002046FAF7DBFF012385F8F000184604B0B6
:10E69000BDE8F0810020CBE7D8F8001089B2C91B93
:10E6A0008A42CFD2F2E700BF586F002058160020F0
:10E6B000242A002010B5164C84F89910017984F8AA
:10E6C0009A2001294FF0000282B084F8982010D0DF
:10E6D000022903D06FF00C0002B010BD032304F137
:10E6E0009802FF21FBF7BCFE0028F3D0002002B007
:10E6F00010BD8268417C90F91000983402F001024C
:10E70000CDE900420323FF22F5F780FFECE700BFCD
:10E71000586F002000680379012B0BD0022B00D02A
:10E72000704783680E4A13F0010315D0002351216E
:10E73000FBF796BE00B58368094A417C90F910004A
:10E7400083B003F00103CDE9002300235122F5F744
:10E750005DFF03B05DF804FBD121FBF781BE00BF74
:10E760001871002000680379012B0CD0022B00D017
:10E77000704783680E4A13F0010F4FF0010313D066
:10E780000021FBF76DBE00B58268417C90F9100056
:10E7900083B002F001020192054A00920022F5F7CF
:10E7A00035FF03B05DF804FB8021FBF759BE00BFC5
:10E7B0000871002030B5194D95F8983183B00BB928
:10E7C00003B030BD04460DF1050100686CF022F97C
:10E7D0009DF805307BB92068114A01214FF40644A9
:10E7E00085F89A100323FF21A5F8984003B0BDE8EF
:10E7F0003040FBF78DBE0DF1060296212068FFF731
:10E800000BFA084ABDF806300749A2FB0323DB08D0
:10E810000122C1F8F83085F89921DCE7586F002013
:10E82000F06F0020CDCCCCCC58160020F8B50446B3
:10E830000F46164600252046202176F0FEFA0446B3
:10E84000C8B10378202B03D114F8013F202BFBD053
:10E850002046FAF75DFCB0F5617F10DB40F634032B
:10E86000984211DD30231A46C5B17B7033780133ED
:10E8700033702046F8BD002DFBD10125DBE70023D6
:10E880001A46002DF1D109E0074AA0F56173A2FBF9
:10E890000323DA08C3F3C703002DE6D13A703378B7
:10E8A00001333370E9E700BF1F85EB51074B53F885
:10E8B000203021B14BB11A689B8853837047002BDD
:10E8C000FCD01A689B88138370477047F853080878
:10E8D0002DE9F04F604BD3F8649091B0B9F1000F7F
:10E8E00004D05E4A03214846F4F700FB0021484665
:10E8F000F4F774FBD9F80430594DD3F800801F6940
:10E900000022560105EB4210A959794011F47C54BC
:10E9100002F1010208D0102AF3D10023C9F80C300B
:10E92000002011B0BDE8F08F027FC9F80C00002A6A
:10E93000F6D1B8F84420DFF840A16FEA42426FEA0E
:10E94000524292B2A8F84420B8F8002092B242F0A5
:10E950008002A8F8002093F805B09B791AF80B10F4
:10E96000B8F820205B074CBF042301238B409BB2E7
:10E9700092B222EA0302A8F82020B8F820203949F0
:10E9800092B21343A8F82030B8F8003042689BB226
:10E9900043F00103A8F80030334B9A42334A136B1B
:10E9A0000CBF43F4001343F48003136306F1180211
:10E9B0004FF0070C354421F802C04B462C49032286
:10E9C000F4F770FDAD682846F4F77EFF2B6823F05E
:10E9D00001032B602846F4F777FF0023CDE90C33C1
:10E9E000CDE90E3306930A93BBF1030F05D8DFE898
:10E9F0000BF0302D022A08F13C04FFB20AEB870A23
:10EA000040F62B4205921B48DAF8043001934FF48C
:10EA100080614FF48042079109924FF48051402267
:10EA2000CDE9030208914FF40033284601A90B9366
:10EA300002946AF06FFB2B68012043F010032B60F7
:10EA400011B0BDE8F08F08F14004D6E708F13804B2
:10EA5000D3E708F13404D0E750800020009F240061
:10EA6000080A00200C0A0020006002400038024022
:10EA7000A10200088CDD0020DC59080838B5104DD3
:10EA80006C6E24B10F4A64212046F4F72FFA00215E
:10EA90002046F4F7A3FA6368012285F868201A6813
:10EAA000B2F844306FEA43436FEA53439BB2A2F893
:10EAB000443013889BB243F00103138038BD00BF7C
:10EAC00050800020009F24001D4AF8B5536E73B19A
:10EAD0005D6892F868206C7906464AB1032C2CD800
:10EAE000DFE804F0222528022B6840331E60F8BDC1
:10EAF000DF681449D7F808C031F814E0DCF80010DA
:10EB0000286821F00101CCF80010818989B221EA3E
:10EB10000E0181811A7403889BB243F001030380C4
:10EB20003A77FFF7ABFFD9E72B683433DEE72B6882
:10EB30003833DBE72B683C33D8E700231B60FFDE6C
:10EB4000508000200853080810B5224C636E83B132
:10EB500094F868206AB194F86C20032A0AD0022A3B
:10EB600010D0002384F86830FFF7B2FE08B984F8AB
:10EB70006D0010BD5A685379032B27D8DFE803F0E6
:10EB800023201D185A685379032B1FD8DFE803F0A0
:10EB90000D0A07021368403300221A6010BD136883
:10EBA0003C33F9E713683833F6E713683433F3E797
:10EBB0001368403364221A6010BD13683C33F9E7D0
:10EBC00013683833F6E713683433F3E700231B6028
:10EBD000FFDE00BF508000202DE9F04FDFF810A3CA
:10EBE000C0499AF871809AF870709AF872E083B010
:10EBF0004FF0000C0AF174000AF51D7BCDF804C03B
:10EC00000122CDF800808378C578C3F1FF039BB261
:10EC10002C46002B00F03281B0F80080B24EC3F1D8
:10EC2000FF03A6FB089605FB03F376091B12052ECE
:10EC300000F26381DFE816F01001F400DC00C2008E
:10EC4000A8000600A84EA6FB08E46409C4EB04145F
:10EC5000A8EB8404A4B2EF1AC4F13C0407FB04F44B
:10EC6000A6FB0464DEB206EB54145FFA84FE2F4662
:10EC70001C462B4601250096F14601951E0246EAE8
:10EC80000446172446EA09060CEB0408A8EB040323
:10EC900002FA04F59BB2354203F12A030CBF0125A9
:10ECA0000225013C41F82350631CEFD104300CF1E4
:10ECB000180C58451FFA8CFCA5D14FF44063AAF8F4
:10ECC00074328023AAF87632019BDDF800802BB1E4
:10ECD0008AF872E08AF871808AF870709AF86D305C
:10ECE000002B4ED0DAF86430002B4AD0EFF31181BC
:10ECF000102282F31288D8685D688468226822F046
:10ED0000010222602C68794A6D7932F81550A28987
:10ED100092B222EA0502A281026944681F2A40F2E7
:10ED2000B580203A202000FA02F2E260CAB282F3F3
:10ED30001188DA68DAF86400926840F62B41516075
:10ED400011680124214311601C7403681A7DA242DA
:10ED500004BF02221A7593F82C100CBF4FF40072F6
:10ED60000022012900F0AB8093F84410012900F043
:10ED7000928093F85C10012900F0AE80002A40F0E8
:10ED8000B98003B0BDE8F08F574FEE1AA946A7FB34
:10ED900008546409C4EB0414A8EB8404A4B204FB73
:10EDA00006F6A7FB0647DCB204EB5717FFB20125B6
:10EDB0000094CE461C4601953B465FE74A4EEF1A4B
:10EDC000A946A6FB08546409C4EB0414A8EB840408
:10EDD000A4B2C4F13C0407FB04F4A6FB0464DFB254
:10EDE00007EB5414E4B201250094CE46019545E7A3
:10EDF0003D4F0095EE1AA7FB08E56D09C5EB05151B
:10EE0000A8EB8505ADB205FB06FEA7FB0E7EDFB2C3
:10EE100007EB5E1E5FFA8EFE0125F14601952DE798
:10EE2000314E0095A5EB030EA6FB08756D09C5EBE9
:10EE30000515A8EB8507BFB2C7F13C070EFB07F726
:10EE4000A6FB07675FFA83FE0EEB5717FFB29946E2
:10EE5000012301933B4611E7EC1A234E08FB04F40F
:10EE60005FFA83FEA6FB04640EEB5414E4B29946E9
:10EE70002F462B46012500940195FFE6AE46A94694
:10EE80002B4600952F4601250195F7E6202000FA34
:10EE900002F2A2604AE7022183F8441093F85C1062
:10EEA000012942F4006217D043681B6800215962AF
:10EEB000998989B20A439A8103B0BDE8F08F022193
:10EEC00083F82C1093F84410012942F48062E2D0B8
:10EED00093F85C100129E7D1022183F85C1042F419
:10EEE0008052E1E78CDD0020898888880853080873
:10EEF000508000204FF40072D6E7009C3B46F1465C
:10EF0000BCE600BF2DE9F04FA04FA7B000210A26B4
:10EF10000C4607F51E754FF0050B01968BE0BAF114
:10EF2000000F19D143F04003BEF18C0F87F87C36F7
:10EF300000F2E48004F1010C98340DEB040A0CF1AA
:10EF400098040DEB040C74464FF0040E0AF88CEC98
:10EF50000CF88C3C04F1020EBEF18C0F42F0020C56
:10EF600000F2CC8004F198036B4403F88BCC04F1DD
:10EF7000040CBCF18C0F03F88CBC00F2BF800EF1C6
:10EF800098060DEB060E4FF0060A0EF88CAC04EB5B
:10EF90000A0E4FEA8909BEF18C0F5FFA89F603F871
:10EFA000890C00F2AB8004F19C0CEC444FF0070993
:10EFB0000CF88C9C04F1080CBCF18C0F03F8876CE6
:10EFC00000F29C800EF198060DEB060E0EF88CBC3C
:10EFD00003F8852C04F10A028C2A00F28F8004F1D8
:10EFE000A0060DEB060C0CF88CAC03F8830C04F1B6
:10EFF0000C008C2800F2828004F1A20204F1A30329
:10F000006A446B4402F88C9C044603F88C8C4809D3
:10F0100001F01F0C55F82030012202FA0CF223EA0D
:10F02000020345F82030019B013B01936ED0013172
:10F03000B1F5F07F6AD23C222846F8F7D1FD011ED7
:10F040005FDB07EB410297F87C36B2F8B4C21CF0E4
:10F05000040FC1F30722C8B25FFA8CF94FEA1C28EB
:10F0600003F0400A04F1020E7FF459AFBAF1000F29
:10F0700003D103F0380CCC4519D003F0870343EAE1
:10F080000903BEF18C0F87F87C3637D804F1010CE8
:10F090000CF1980698346C440DEB060C4FF0040903
:10F0A00004F88C9C74460CF88C3C0EF1020EBEF1F8
:10F0B0008C0F23D804F198030DEB030C231D8C2B2C
:10F0C0000CF88B2C0CF88CBC18D80EF198020DEBB8
:10F0D000020E06220EF88C2C0CF8890CA0188C2835
:10F0E0000CD804F19C0304F19D026B446A4407248C
:10F0F00003F88C4C044602F88C8C88E76FF00044CF
:10F1000085E7204614B927B0BDE8F08FD7F87456CC
:10F110001F4995F91030AA6803EB8303920751F851
:10F12000230020D5234603AA00216DF0A3FEAB687F
:10F130009B0701D50120E6E7164B17491A68174BC4
:10F140004FF4FA7000FB02F2A3FB02324868920906
:10F150004B681B1A9A42FBD26B69002BEAD01A68E3
:10F160009B881383E6E76B6913B11A689B88538306
:10F17000084B09491A68094B4E68D200A3FB0232BA
:10F1800092094B689B1B9A42FBD2CBE75080002030
:10F19000500C002014600020001000E0D34D6210DD
:10F1A000F0B5284CD4F8740683B010B194F87A36D0
:10F1B0000BB103B0F0BD01230DF10702842184F8E7
:10F1C0007A36FCF717FA94F87C26D4F874060421F2
:10F1D0000A43FAF733FAD4F874060DF107028421D2
:10F1E000FCF708FA9DF8073013F00406F3D1164D2A
:10F1F00084F87C363C223146284674F057FF32466C
:10F20000124E05F13A0005F2FA374FF0010E30F8D0
:10F21000023F334002F01F019BB24FEA521C0EFA2C
:10F2200001F1013223B155F82C300B4345F82C3055
:10F23000B842ECD1FFF766FE0028FBD184F87A06CD
:10F2400003B0F0BD50800020C882002004DFFFFF23
:10F2500070B5404DD5F8744682B08CB395F87836C9
:10F26000012B41D0022B2DD1082294F910303A49BC
:10F2700085F87B2603EB830300208DF8040051F80A
:10F280002300A3688DF8052040F20442ADF8062063
:10F290009A0742D504230DEB030200216DF0EAFD2D
:10F2A000A3689B0722D52D483C22FF2174F0FEFE67
:10F2B00095F8793623B9FFF773FF012385F879367E
:10F2C00002B070BD0DF10302A0212046FCF792F9B7
:10F2D0009DF8033003F00503012B37D0002B2FD10D
:10F2E000D5F874460822C0E74822BEE71C4B1D49EA
:10F2F0001A681D4B48684FF4FA7606FB02F2A3FB2E
:10F30000023292094B681B1A9A42FBD26369002BA6
:10F31000C9D01A689B881383C5E7636913B11A685B
:10F320009B8853830E4B0F491A680F4B4E68D200CF
:10F33000A3FB023292094B689B1B9A42FBD2A9E7BE
:10F340000A4A126840F2DC539A42B9D9D5F8744699
:10F3500048228AE750800020500C0020C8820020FC
:10F3600014600020001000E0D34D6210242A002019
:10F370002DE9F041334D95F87A3682B003B1FEE7BE
:10F38000012285F87A2695F87B26044602F0F702DA
:10F39000D5F8740685F87B260E461946FAF74EF91D
:10F3A000E2B207460921D5F87406FAF747F9B4F531
:10F3B000807F3FD0D5F87406DFF88C80502208217A
:10F3C000FAF73CF9D5F874060DF10702A021FCF715
:10F3D00011F948B9D8F8D830B8F8DC2059690A4290
:10F3E00014BF5A831A83EDE79DF8074014F02004F8
:10F3F000F0D1E2B20A21D5F87406FAF71FF93219F2
:10F40000D5F87406C0210134FCF7F4F8362CF0D19D
:10F4100057B995F87B26D5F8740602F0F7023946FD
:10F4200085F87B26FAF70AF9002385F87A3602B0C8
:10F43000BDE8F081D5F8740640220A21FAF7FEF8FB
:10F44000B8E700BF508000202C2B00202DE9F04FA2
:10F450005F4D95F87A76C3B007B1FEE795F87B2645
:10F46000044602F0F7020123D5F8740685F87B26DE
:10F470000E46394685F87A36FAF7E0F8FF2C4FF059
:10F4800009038DF8054088BFA40801AA8CBF04F0C9
:10F49000C008B84602204FF0000C4FF00A0B0DF1E7
:10F4A000050A4FF00B09137014E0B1F5827F02F8E2
:10F4B00000B00AF8003016F80C3017D80CF1010C27
:10F4C000BCF1360F02F8079004F1060402F80E3082
:10F4D000084614D0871C48EA0C03B7F5827F00F178
:10F4E00004010446DBB200F1030EDED90CF1010C7D
:10F4F0006FF00041BCF1360F364C0846EAD1B4F546
:10F50000827F61D8082353540DF10503A0211954BB
:10F51000831CD5F87446304894F9101001EB810132
:10F5200050F82100A168890722D500216DF0A2FCC6
:10F53000A3689B0731D5294CD5F874060DF1030259
:10F54000A021FCF757F848B9D4F8D830B4F8DC203B
:10F5500059690A4214BF5A831A83EDE79DF80330B4
:10F5600013F02003F0D185F87A3643B0BDE8F08F70
:10F57000616911B10E68898871831949194F0E6844
:10F580001949D7F804C0F600A1FB0616B609796838
:10F59000A1EB0C018E42FAD2C7E7114B11491A6850
:10F5A000114B48684FF4FA7606FB02F2A3FB0232D5
:10F5B00092094B681B1A9A42FBD26369002BBAD09E
:10F5C0001A689B881383B6E76FF00043A1E700BF7A
:10F5D0005080002001000080500C00202C2B0020C7
:10F5E00014600020001000E0D34D6210002ABCBF60
:10F5F00080185242002B30B503EB010503DA0C46AC
:10F600005B42294625460028B7BF121A84181446C3
:10F610000020A4F11D0C0029BCBF2B460021BCF129
:10F62000000FC4BFA2EB0C021418A5F10F02002AB0
:10F63000C4BF9B1A5D1884421EDBC1F1010C0F4A46
:10F64000AC44C1EB0113CCEB0C1C00EB43030134C5
:10F650004FEA4C0C02EB43024FF0200E8D42A8BF44
:10F66000002304DB22F813E01E339C45FAD101305D
:10F67000A04202F10202F1D130BD00BF048300209C
:10F680001B4B1C48196C1C4A10B441F080510124DA
:10F69000196404625321FF24CA20546250625162EB
:10F6A0005B6FDB0085B013D40023144902930291F1
:10F6B000029A134804320292029A13600393039150
:10F6C000039B0393039B186005B05DF8044B7047E0
:10F6D0000A4B002201920193019B0193019A084B6E
:10F6E00012689A42E0D105B05DF8044B704700BF44
:10F6F0000038024000000E42002800405028004020
:10F7000076614E6970B50546BDF8106001600C4623
:10F7100019B119462046F3F7E9FB31462046F3F7C5
:10F720005DFC61680B68B3F844206FEA42426FEAFF
:10F73000524292B2A3F844201A8892B242F00102D7
:10F740001A804A79032A17D8DFE802F0110C070261
:10F7500040330022AB601A6070BD3C330022AB60C6
:10F760001A6070BD38330022AB601A6070BD34334C
:10F770000022AB601A6070BD0023AB601B60FFDE2F
:10F780002DE9F04F85B00646BDF838B09DF83CA095
:10F79000894617469846F3F759FB002857D02D4C59
:10F7A00094F880360A2B4DD803EB430204EB421247
:10F7B00002900020C2F8840682F888065A1CD2B251
:10F7C00084F8802603EB43033079039204F28464C7
:10F7D00004EB4314FDF75CFD0299054618B3039A48
:10F7E000027280F806900220E87143463A46CDF84E
:10F7F00000B02046FFF786FFBAF1000F0AD11121B1
:10F800002846FDF7E5FC2B68AA885A83204605B0F8
:10F81000BDE8F08F2846327A0221FDF7FDFC204634
:10F8200005B0BDE8F08FCDF800B043463A4620461B
:10F83000FFF768FFBAF1000FECD111215046FDF738
:10F84000C7FCE3E7044A00210420F8F7EBFE00249C
:10F85000DCE700BF5080002098FD080830B5036841
:10F86000284D294C2DED028BAB42246883B0F0EE7D
:10F87000408AB0EE608A10D005F58065AB420CD0AE
:10F8800005F57055AB4208D005F58065AB4204D054
:10F8900005F58065AB4218BF6408B4FBF1F303F5CE
:10F8A0007F43FF331B0CB4FBF3F40023B4FBF1F5EF
:10F8B000019200932246ABB20221FFF761FFE0B153
:10F8C000B5EE408A07EE904AF1EE10FAF8EE677A4C
:10F8D0000ABF07EE105A28EE278AB8EE478A9FED36
:10F8E0000B7AC8EE076A0123037127EE667AC0ED32
:10F8F000046AA8EEA77A80ED037A03B0BDEC028B10
:10F9000030BD00BF00000140D400002000007A4458
:10F910002DE9F04F2DED028BAA4BAB4E1B78AB4D72
:10F92000DFF8CCA2B5B000270293B046B146BB4683
:10F93000D9F80040002355F83320944203D0013316
:10F940000E2BF8D1FF23534493F8A43A022B00F076
:10F95000BB80032B00F0AF80012B09D1D9F80C300C
:10F9600023F0807323F0080343F00403C9F80C303C
:10F970004846FEF759F848B90BEB8B0308EB8303B5
:10F98000D96801F00C03042B00F0A9800BF1010BE6
:10F99000BBF10C0F09F11409CAD18D4DDDF80880B7
:10F9A000A5F1F00408E02068E260FEF7D1F84844D1
:10F9B000C7B21434A5421FD02046FEF735F8002800
:10F9C000F7D1E368590703F00C02F2D5042AF0D00E
:10F9D00023F0080242F00402781C474511465FFA02
:10F9E00080F923F00403DED32068E3601946143461
:10F9F000FEF7AEF8A542DFD10025764FDFF8F4918F
:10FA00002C46A846AB463046FEF70EF8002840F0DC
:10FA1000A880F06842076AD5029B57F80C2C434532
:10FA200000F2A680030764D4002D57F80C3C40F385
:10FA3000BD8028A900229C4602E0AA4200F0B580C1
:10FA400051F8043F1B689C4502F10102F5D1C20147
:10FA500064D40BF1010BBBF10C0F06F1140607F196
:10FA60001407D0D1574B93F800E0BEF10C0F00F310
:10FA70001082594B594A1B791370032B40F2BC80FA
:10FA80001A1F022A00F27982052B00F06782062BEA
:10FA90000CBF4FF47A564FF47A6651495148002210
:10FAA0004A600027504AB2FBF6F200260A60C0E91D
:10FAB00000674E4AA1E0D9F80C3023F00C0343F064
:10FAC0008073C9F80C3053E7D9F80C3023F08073F9
:10FAD00023F0040343F00803C9F80C3048E720463C
:10FAE000FEF736F80137FFB20744FFB24EE70207D0
:10FAF000ADD5002C57F80C3C4BDD1DA900229C46CF
:10FB000001E0A24244D051F8043F1B689C4502F139
:10FB10000102F6D1410787D4C2019AD5002C57F8CB
:10FB20000C3C0ADD1DA9002251F8040F0068834235
:10FB300002F101028DD0A242F6D1002D0ADD28A9E2
:10FB4000002251F8040F0068834202F1010280D0C4
:10FB5000AA42F6D14FF080711846F160FDF7F8FF28
:10FB600077E75B464A4601210420F8F75BFD70E722
:10FB700020F00801F1601046FDF7EAFFF06808F197
:10FB8000010803075FFA88F8B3D44107C4D54BE7EF
:10FB90006346184634AB03EB85020821F16042F856
:10FBA0002C6C0135FDF7D4FF53E76346184634ABA0
:10FBB00003EB84020421F16042F8586C0134FDF734
:10FBC000C7FF46E7AC000010581600207453080821
:10FBD000481700206416002068620020586000204A
:10FBE000606000206860002040420F008DDB00084C
:10FBF00050800020D4FD0808B84ACAF8B42AB84A90
:10FC000012F81330002B00F0B281A64500F3B78143
:10FC1000BEF1000F00F0A6809FEDB28ADFF820B39E
:10FC2000DFF8148304951DAC4FF000097746AE4B06
:10FC3000DBF800201B7854F8046FC2F30072062B27
:10FC400000F23C81DFE803F0B5ABA17904040400C5
:10FC5000052B00F07781A549A548062B18BF014662
:10FC60000025019200950A46142302213046FFF731
:10FC700087FD0290002800F021819E4B31681A78A0
:10FC8000002A00F01281CDF80C8003E00135954286
:10FC900000F00D812B0158F803309942F6D1EAB2F9
:10FCA000082A00F00B810298934B016805910D68BA
:10FCB0004E6807954FF4907101FB0231039BC165BB
:10FCC00003EB02130691996013016A6E089335687D
:10FCD000002A00F05881B5F8443088486FEA434361
:10FCE0006FEA53439BB2A5F844302B889BB243F094
:10FCF00080032B80737909931946B379405C298C72
:10FD00005B074CBF0423012383409BB289B221EAE5
:10FD100003012984298C89B20B432B842B889BB245
:10FD200043F001032B80002A00F05B81029A01233B
:10FD30001371734B43F839200EE0DFED720A724BFA
:10FD4000B0EE600A59883046FFF788FD6C4B43F8E7
:10FD50003900002800F0A28109F101094F457FF424
:10FD600066AF049D694C94F8C03263BB684A0221B7
:10FD70000420F8F757FC9AF8B20AB0FA80F040096C
:10FD800035B0BDEC028BBDE8F08FDFED620A9FED70
:10FD9000620A30464FF4FA61FFF760FDD6E7DFED07
:10FDA0005F0A3046B0EE600A4FF47A71FFF756FDF5
:10FDB000CCE79FED4C0AF0EE480A30464FF4C8718C
:10FDC000FFF74CFDC2E794F8C19294F8C23209F1F2
:10FDD0000109A9EB0309B9F1120F0BDD122302216E
:10FDE00000934F4A8AF8B21A4B4600210420F8F7D4
:10FDF00019FCC0E794F8CC32012B00F0B480022B40
:10FE000040F0A2806AF010FB464BC4F8D03294F860
:10FE1000CC32002B00F0A580022B40F09980122DEF
:10FE20002B46B8BF12239BB24B45C0F2D080A945E8
:10FE3000A8BFA946B9F1000F9DDD3B4FDFF800B127
:10FE4000DFF8E88028AE002504E001354D4547F88D
:10FE5000040B90D0DBF80030B4F8C412C3F3007286
:10FE6000B4F8C63201920091B8FBF3F32F4A56F86A
:10FE7000040F9BB20321FFF783FC0028E5D1052482
:10FE800001462B4A8AF8B24A2B460420F8F7CAFBEF
:10FE900071E7284ACDF800B001218AF8B21A7346FA
:10FEA00000210420F8F7BEFB5CE7234B039313010A
:10FEB0000398C1500F49531C0B70F1E6104A049D82
:10FEC000002342F8393005218AF8B21A1B4A4B4602
:10FED00000210420F8F7A6FB44E700BFB9E50008BD
:10FEE000105408086F12833A58600020001BB700B6
:10FEF000C0C62D00A0600020088B0020DC59080837
:10FF0000A4600020000000006862002048910020EA
:10FF10009CFE0808ACC5A737ACC5A7366F120339DD
:10FF2000B8FE0808A5DB0008A46F002040420F00BF
:10FF300058FF0808ECFD08080461002074FE08085A
:10FF4000B400001056498BE6564AC4F8D02243B19B
:10FF5000554A02210420F8F765FB0CE74FF4FA56E6
:10FF60009BE52B465FE76AF05FFA504B4DE7504A3E
:10FF700002210420F8F756FBF4E64E4A3DE64E4ACD
:10FF80000094032189E7D6F810C04C490992134622
:10FF90004FEA431E01EB431051F80E208CEA020E8B
:10FFA0001EF47C5F03F1010309D0102BF0D1059AF8
:10FFB0000023D360424B029A43F83920CCE6059BDC
:10FFC000099AD860037F002B3FF485AEF2E7042046
:10FFD00000953C4A8AF8B20A4B460021F8F722FB0A
:10FFE000C9E6059B3849DB680A931A46374B5268C5
:10FFF0000A989A42364A136B0CBF43F4001343F439
:020000040801F1
:1000000080031363072383830322059BF3F74AFAD4
:100010000A9880680B90F3F757FC069A337C0F928E
:100020002C4A0B98069002EB83034FF480465B68E2
:100030000D93036823F0010303600023CDE9183317
:10004000CDE91A3312931693122311934FF4806360
:1000500013934FF48053CDE9143640234C3510935D
:100060000DA94FF400330E95179369F053F80698D5
:10007000089D039A03680A992A44079D43F01003D8
:1000800003606966144B099933F81130A5F868309C
:1000900093815060059A0123137447E6049D12E78B
:1000A000808D5B00C1DB0008E4FE080821C0030866
:1000B00018FE080889DB000838FE0808080A002036
:1000C000A460002020FF0808A10200080060024090
:1000D00000380240DC5908080853080810B5104CD5
:1000E000D4E90423A16882B002FB03F38B428DF8AC
:1000F000070012D06368E0680DF10701184472F040
:10010000B3FE63682269A16813446269B3FBF1F02E
:10011000013201FB10336360626102B010BD00BFA9
:100120007860002010B50379012B84B00C4627D0ED
:10013000022B23D18368DB070DF10F024CBF012195
:100140008121FBF705FA9DF80F300022C3F300115F
:1001500061F30702C3F3800161F30F220F49C3F378
:10016000C00C6CF3174281F8F000C3F3801161F307
:100170001F62DB092260237104B010BD0020E2E79A
:1001800082680DF10F0102F00102CDE900121A465A
:10019000417C90F91000F4F705FAD4E758160020D6
:1001A0002DE9F04182B014460E4601AA50210546C1
:1001B000FBF720FA9DF80430DFF8F080394F013367
:1001C0005B00DBB24621238001AA2846FBF712FA26
:1001D00023789DF8042008FB03F303F5FA73A7FBCB
:1001E000031301329909DB0902FB0133A280A7FB4B
:1001F00003239B0901AAE360512102232846FAF751
:1002000001FA2378BDF8040008FB03F340BA03F5B4
:10021000FA73A7FB0323C2B2C0F307208240013266
:1002200092B29809DB0902FB0033A7FB03739B0919
:100230007021E280238201AA2846FBF7DBF99DF8B2
:10024000043001335B00DBB201AA63807121022319
:100250002846FAF7D7F9BDF80430134AF17882F846
:10026000F0005BBADAB2C3F307239A40013292B2CC
:10027000228119B1E388D21A92B222810B48A37865
:10028000084900FB03F303F5FA73A1FB0303980984
:10029000DB0902FB0033A1FB03139B09638202B05D
:1002A000BDE8F081D34D621058160020002F3A00AF
:1002B0002DE9F047DFF89882DFF89892A34F8CB0D1
:1002C000054600264FF4FA7307AA89210068C8F88A
:1002D000B83188F89460FBF78DF99DF81C202868E8
:1002E00042F001028921F9F7A9F9324688212868EC
:1002F000F9F7A4F9012280212868F9F79FF9012272
:10030000FF212868F9F79AF9324631462868F9F74B
:1003100095F907AA91212868FBF76CF99DF81C3024
:10032000286888F8B13131460122F9F787F9324659
:10033000FF212868F9F782F9324680212868F9F709
:100340007DF907AA60212868FBF754F99DF81C2065
:10035000286842F012026021F9F770F94FF4005357
:10036000ADF81C3007AA022344212868FAF7D0F818
:10037000FF2201212868F9F761F92C680122802108
:100380002046F9F75BF90122FF212046F9F756F9DB
:10039000324631462046F9F751F90622FF21204620
:1003A000F9F74CF907AA83212046FBF723F99DF8BA
:1003B0001C20832142F004022046F9F73FF907226E
:1003C000FF212046F9F73AF9012281212046F9F769
:1003D00035F9012280212046F9F730F96B2294216A
:1003E0002046F9F72BF9324683212046F9F726F902
:1003F000D9F80060C8F8B4612379012B00F0988027
:10040000022B0FD000209DF81C3087F8F000DBB9DC
:10041000D9F800309BB29B1BB3F5FA7FECD90CB036
:10042000BDE8F087A368DB0707AA4FF083012046E9
:100430005EBF07AA83212046FBF78AF89DF81C308F
:1004400087F8F000002BE3D0012283212046F9F742
:10045000F5F807AA92212046FBF7CCF8002281216B
:1004600020469DF81CA0F9F7E9F80622FF21204656
:10047000F9F7E4F807AA83212046FBF7BBF89DF8BB
:100480001C20832102F0FB022046F9F7D7F8012255
:10049000FF212046F9F7D2F8012200212046F9F782
:1004A000CDF80022FF212046F9F7C8F820460022A7
:1004B0008021F9F7C3F80623B02105AA2868FAF7C6
:1004C000A1F80122FF212868F9F7B8F800224F218E
:1004D0002868F9F7B3F82C224E212868F9F7AEF80E
:1004E0000022FF212868F9F7A9F84FEADA162868F0
:1004F000B422B621F9F7A2F80024002E18BF0C266A
:100500000AF07F0AA1464FF0010EC4F3C403303352
:100510006B44E2B213F81C0C04F0070C0EFA0CF159
:10052000964220EA010117D903F81C1C0134ECE7BC
:10053000A268617C94F9100002F00102019207AAFE
:1005400000928322F4F72EF85DE700BF58160020D2
:10055000586F0020242A0020D14540FA0CF200F008
:100560001283D30744BF09F101095FFA89F9013405
:10057000302CCAD1062305AAB0212868F9F7C8FF94
:100580000122FF212868F9F759F80022114628684E
:10059000F9F754F80022FF212868F9F74FF80022F4
:1005A00009212868F9F74AF8002210212868F9F78C
:1005B00045F8002211212868F9F740F8012224218A
:1005C0002868F9F73BF8FF2225212868F9F736F863
:1005D000002275212868F9F731F80122FF212868E7
:1005E000F9F72CF82C224E212868F9F727F8002279
:1005F00048212868F9F722F8214620222868F9F7CF
:100600001DF80022FF212868F9F718F82146092271
:100610002868F9F713F8002254212868F9F70EF832
:10062000042231212868F9F709F8032232212868C9
:10063000F9F704F8832240212868F8F7FFFF252204
:1006400046212868F8F7FAFF002260212868F8F7A9
:10065000F5FF002227212868F8F7F0FF0622502135
:100660002868F8F7EBFF002251212868F8F7E6FF29
:10067000962252212868F8F7E1FF082256212868BF
:10068000F8F7DCFF224657212868F8F7D7FF002249
:1006900061212868F8F7D2FF002262212868F8F764
:1006A000CDFF002264212868F8F7C8FF00226521E9
:1006B0002868F8F7C3FFA02266212868F8F7BEFF74
:1006C0000122FF212868F8F7B9FF32222221286889
:1006D000F8F7B4FF142247212868F8F7AFFFFF228C
:1006E00049212868F8F7AAFF00224A212868F8F76C
:1006F000A5FF0022FF212868F8F7A0FF0A227A212F
:100700002868F8F79BFF00227B212868F8F796FFFE
:10071000212278212868F8F791FF0122FF2128681B
:10072000F8F78CFF342223212868F8F787FF00228E
:1007300042212868F8F782FFFF2244212868F8F751
:100740007DFF262245212868F8F778FF05224621FB
:100750002868F8F773FF402211462868F8F76EFF03
:1007600006220E212868F8F769FF1A22202128683E
:10077000F8F764FF402243212868F8F75FFF002262
:10078000FF212868F8F75AFF032234212868F8F778
:1007900055FF442235212868F8F750FF0122FF2138
:1007A0002868F8F74BFF042231212868F8F746FF44
:1007B00009224B212868F8F741FF05224C212868BF
:1007C000F8F73CFF04224D212868F8F737FF002294
:1007D000FF212868F8F732FF002244212868F8F743
:1007E0002DFF202245212868F8F728FF08224721FD
:1007F0002868F8F723FF282248212868F8F71EFF09
:10080000002267212868F8F719FF04227021286860
:10081000F8F714FF012271212868F8F70FFFFE2274
:1008200072212868F8F70AFF002276212868F8F775
:1008300005FF002277212868F8F700FF0122FF2139
:100840002868F8F7FBFE01220D212868F8F7F6FE6C
:100850000022FF212868F8F7F1FE01228021286894
:10086000F8F7ECFEF82201212868F8F7E7FE0122EC
:10087000FF212868F8F7E2FE01228E212868F8F7A8
:10088000DDFE012200212868F8F7D8FE0022FF21B2
:100890002868F8F7D3FE002280212868F8F7CEFEFA
:1008A00004220A212868F8F7C9FE2C6807AA8421C7
:1008B0002046FAF79FFE9DF81C20204602F0EF022A
:1008C0008421F8F7BBFE01220B212868F8F7B6FE59
:1008D0002C6803A92046FFF725FC07AA03A9204698
:1008E000FFF75EFC9DF80C30002B00F05D810A9C48
:1008F00004F684549DF80E30002B00F04B810A9BC7
:1009000003F2B22304EB43049DF80F3023B1BDF88A
:100910002C3003F525731C449DF8103023B1BDF82D
:100920002E3003F226231C44A44E2868C6F8D44275
:10093000E8220121F8F782FE286821466AF0A0F833
:10094000012211462868F8F779FE402187F8F00067
:100950002868FDF74BFE00283FF461AD01212868AF
:100960000222F8F76BFE002187F8F0002868FDF7F7
:100970003DFE00283FF453ADE82201212868F8F736
:100980005DFE4FF4005307AAADF81C30442102234A
:100990002868F9F7BDFD2C6803A92046FFF7C2FBC4
:1009A00007AA03A92046FFF7FBFB50225721204648
:1009B000F8F744FE082256212046F8F73FFE0822A9
:1009C00050212046F8F73AFEBDF82C204FF47A71FA
:1009D00048F20E6301FB0233794A934240F2EB8006
:1009E000784AA2FB0332120C013AFF2A4FF00003AF
:1009F00006DD52080133FF2A9BB2FAD81B029BB2D4
:100A00001343C3F30722DBB28DF808208DF80930B9
:100A100002AA022351212046F9F77AFD0A9A4FF4DF
:100A20007A7148F20E6301FB0233674A934200F287
:100A3000C080644AA2FB0332120C013AD2B24621B2
:100A40002046F8F7FBFD2046D6F8D4126AF018F8D5
:100A500002AA01212046FAF7CDFD02229DF8089056
:100A600001212046F8F7EAFD00212046FDF7BEFDF2
:100A70004A4620460121F8F7E1FD2C6803A92046EB
:100A8000FFF750FB07AA03A92046FFF789FB48227E
:100A900011462046F8F7D2FD082247212046F8F7F4
:100AA000CDFD032232212046F8F7C8FD0722302170
:100AB0002046F8F7C3FD0122FF212046F8F7BEFDCE
:100AC000202230212046F8F7B9FD0022FF212046E0
:100AD000F8F7B4FD062270212046F8F7AFFDBDF807
:100AE0002E103A4A4FF47A7046F6440300FB013365
:100AF000A2FB03239DF80F201B0B1AB1BDF8222087
:100B000013449BB2002B52D05A1EFF2A4FF0000311
:100B100006DD52080133FF2A9BB2FAD81B029BB2B2
:100B20001343C3F30722DBB28DF808208DF8093098
:100B300002AA022371212046F9F7EAFCD6F8D41262
:100B4000204669F09DFF02AA01212046FAF752FDD6
:100B50009DF80850022201212046F8F76FFD002180
:100B60002046FDF743FD2A4601212046F8F766FDA1
:100B70006422012387F8F000C8F8B82188F894307F
:100B80000CB0BDE8F0870EFA0CFC20EA0C0003F86C
:100B90001C0CECE49DF80D30002B3FF4B5AE0A9B25
:100BA00003F525731C44AFE640F63634A2E61A4638
:100BB000BAE7FF2243E700231A4625E748910020C1
:100BC0001B0C0100950370F41B280D014963A4134D
:100BD00010B5164C84F89910017952BAA4F89A20ED
:100BE00001294FF0000282B084F8982010D0022929
:100BF00003D06FF00C0002B010BD042304F1980282
:100C0000FF21F9F72DFC0028F3D0002002B010BD21
:100C10008268417C90F91000983402F00102CDE91D
:100C200000420423FF22F3F7F1FCECE7586F0020A9
:100C30002DE9F04F9D4F9E4D06683C464FF0000851
:100C400085B0834685F898815B37C4F12D0905F19D
:100C5000980A13E0022B0FD1B26812F0010F4FF087
:100C6000030352464FF0FF01304601BF03235246B3
:100C7000FF213046F9F7F4FBA7421AD0337985F803
:100C8000988009EB0401012B14F8012F85F89910C5
:100C900085F89A20DED1B368717C96F9100003F0D4
:100CA0000103CDE900A3FF220323F3F7AFFCA74222
:100CB000E4D14FF40743A5F89830402385F89A30E3
:100CC00052460323FF213046F9F722FC00238DF81A
:100CD0000E300DF10E01304669F09CFE9DF80E308D
:100CE000002BF6D04FF40643A5F898300123714A43
:100CF00085F89A30FF2103233046F9F709FC4FF4B9
:100D000007436C4AA5F8983000240323FF2130469E
:100D100085F89A40F9F7FCFB4FF40063A5F898308A
:100D20000923644A85F89A30FF2103233046F9F7F6
:100D3000EFFB4FF43063A5F898305E4A85F89A408F
:100D400030460323FF21F9F7E3FB002800F0AC80D5
:100D5000DBF800400DF10E025E212046FCF75CFF3F
:100D6000BDF80E30B3F5D77F00F08C806AD8512BD8
:100D700000F0848078D81D2B7ED10F2608BB0A2274
:100D80004B212046FDF796FC0F2260212046FDF7FF
:100D900091FC0D2263212046FDF78CFCB8226921CD
:100DA0002046FDF787FC40F60D7278212046FFF7BC
:100DB0000FFF40F60E627A212046FFF709FF002858
:100DC0006DD0DBF80000212169F07AFDDBF80040EE
:100DD0000DF10E02DE212046FCF71EFFBDF80E309D
:100DE0009FED357AC3F3090303EB8303DB0007EEC2
:100DF000903AF8EEE77A4FF4D84267EE877AA5F892
:100E00009820FCEEE77A524617EE903A1BBAC5F8E6
:100E10009A30FF2106232046F9F77AFB4FF4074169
:100E20004023DBF80000A5F8981085F89A30524668
:100E30000323FF21F9F76CFBB0B385F8980105B0E7
:100E4000BDE8F08F40F2E132934219D01CD840F255
:100E5000D922934214D040F2E122934202D0B3F55A
:100E6000E67FAED1642689E7AD2B0BD0D62B01D01F
:100E7000602BA6D1212681E71E2BA2D114267DE767
:100E8000C8267BE7322679E740F28F42934203D0AF
:100E900040F29152934294D14FF4FA766EE7314684
:100EA000204669F00DFD8CE70020C6E7FF590808D1
:100EB000586F0020F06F00209A99893F03682DE950
:100EC000F0411F6A1FB13B46BDE8F0411847002AB8
:100ED000164611DD04460D460E4400E023689B686B
:100EE000204698470028F9D0236815F8011B1B6895
:100EF00020469847B542F1D1BDE8F081DEE700BF5A
:100F0000204A214B116893F8E222C90603D5B3F8B1
:100F1000E412490715D4F2B993F80023D3F8FC3250
:100F200052B143B120B11A689B88138370473BB319
:100F30001A689B885383704780F00100002BF1D121
:100F4000F9E7B2B993F80023D3F8FC32002AEED1C6
:100F5000002BE8D17047D3F8F422002AEBD058B127
:100F60009268B3F8F812094BB3FBF1F35B1013600E
:100F70007047D3F8F42222B1936800221A607047B8
:100F800070477047B00000104891002040420F00A9
:100F9000BFF34F8F0549064BCA6802F4E062134362
:100FA000CB60BFF34F8F00BFFDE700BF00ED00E057
:100FB0000400FA0508B572B600224FF0FF31930025
:100FC00003F1604303F561430132082AC3F880103E
:100FD000C3F88011F3D1FFF7DBFF00BF012108B593
:100FE0000846F3F747FBFFF7E5FF00BF00B583B006
:100FF0000D49002200920091009B04330093009B56
:101000001B68012B02D003B05DF804FB0192019133
:10101000019B064904330193019B1A600B6883F31B
:1010200008884B689847FEE7502800400000FF1FE3
:1010300010B4EFF31183102282F31288094C0A488E
:1010400022684FF0E021013222608A69C0F804234F
:101050000022C0F808230A69DBB283F311885DF827
:10106000044B7047242A00204891002030B4EFF34D
:101070001182102383F312884FF0E023D2B29969D2
:10108000186910F4803F0D481EBF0121C0F80813F5
:1010900099690B4B1D68D0F8083382F31188094811
:1010A00004684FF47A7202FB04F02B44401A0021CA
:1010B000B0FBF4F030BCE3FB020170474891002024
:1010C000242A002014600020124B5B68C3F308033D
:1010D000FBB9EFF31183E3B930B40F4A0F4C4FF073
:1010E000E02C1368DCF8180011688B42F9D1D4F8B1
:1010F00004138842F5D80A4A15684FF47A7404FB41
:1011000005F20021101AB0FBF5F0E3FB040130BC3E
:101110007047ABE700ED00E0242A00204891002052
:101120001460002090B170B5461EFFF7CDFF044655
:101130000D46FFF7C9FF001B61EB0501B0F57A7F93
:1011400071F10001F5D3013EEFD270BD704700BFD1
:1011500070B5006801220921F8F770FA6426FFF7DC
:10116000B3FF04460D46FFF7AFFF001B61EB05011F
:10117000B0F57A7F71F10001F5D3013EEFD170BD7A
:101180002DE9804883B0431C0193DFF83C810A239A
:101190000093D8F89C10D8F8D830B8F8A000B8F868
:1011A000DC20DDF804B048834FF0320A1A834FF098
:1011B0000509D8F89C30B8F8A02059690A4214BF34
:1011C0005A831A83D8F8D830B8F8DC2059690A4213
:1011D00014BF5A831A830120FFF792FE56465746E2
:1011E000FFF772FF04460D46FFF76EFF001B61EB31
:1011F0000501B0F57A7F71F10001F5D3013FEFD120
:10120000D8F89C30B8F8A02059690A4214BF5A8314
:101210001A83D8F8D830B8F8DC2059690A4214BFCC
:101220005A831A830020FFF76BFEFFF74DFF044639
:101230000D46FFF749FF001B61EB0501B0F57A7F12
:1012400071F10001F5D3013EEFD1B9F1000F1CD0CF
:10125000B9F10109ADD14FF4FA76FFF735FF044635
:101260000D46FFF731FF001B61EB0501B0F57A7FFA
:1012700071F10001F5D3013EEFD14FF0FA0ABBF155
:10128000000F07D04FF0000993E70BF1FF3BBBF1D4
:10129000000FF7D14FF47A76FFF716FF04460D469C
:1012A000FFF712FF001B61EB0501B0F57A7F71F1CA
:1012B0000001F5D3013EEFD1009B013B00937FF489
:1012C00068AFFFF78BFE00BF2C2B002018B103681E
:1012D0005B6903B11847704718B103681B6A03B113
:1012E00018470020704700BF38B50B4D0C4620B1A1
:1012F0000368DB6A0BB1984760B90020C4E90000BD
:10130000C4E90200C4E906552D223023206122756C
:1013100084F8203038BD00BFF05C09080178F9B1CD
:10132000F8B5104F0546002602E015F8011FB1B1CF
:10133000D7F80C43637A5A1C2344D2B26272997272
:10134000237A9342F1D804F10A01002AEDD0D4E9BE
:1013500000309847667215F8011F0029E8D1F8BDE2
:10136000704700BF4891002070B5124C05460E46EC
:101370001148FFF7D3FF2A461049D4F80C0333462F
:101380006BF00AFED4F80C536A7A32B12B686868A5
:1013900005F10A01984700236B7294F810333BB1B2
:1013A00094F812330122134484F8112384F8123381
:1013B00070BD00BF4891002080FF0808E1DD0008F3
:1013C00080B51948194DFFF7A9FF1948FFF7A6FF87
:1013D000D5F80C43627A32B12146606851F80A3B75
:1013E000984700236372D5F814733B6838465B69ED
:1013F0009847B0B90A26FFF767FE04460D46FFF787
:1014000063FE001B61EB0503B0F57A7F73F1000307
:10141000F5D3013EEFD13B6838465B699847002819
:10142000E8D001200DF0AAFE8CFF080848910020AA
:10143000A8FF0808154B93F81823012A00D070471D
:1014400010B593F81D23062A84B00DD00A2A06D1C0
:1014500035F012FB0E4804B0BDE810405EE70D48C1
:1014600004B0BDE8104059E7D3F838434CB10A4AFC
:1014700007CA01AB03C301A91A7020460922FFF76E
:101480001DFD064804B0BDE8104047E74891002024
:10149000C4FF0808B4FF0808FCFF0808E0FF0808BC
:1014A00080B52F482F4FFFF739FF2F48FFF736FF42
:1014B000B7F83C63002E43D1D7F80C43627A32B1BF
:1014C0002146606851F80A3B984700236372274B16
:1014D00000251D7087F84053C7F8805324F0ACFFF7
:1014E0002348FFF71BFFD7F80C43627A2AB1214645
:1014F000606851F80A3B98476572D7F814733B68E7
:1015000038465B699847B0B90A26FFF7DDFD044607
:101510000D46FFF7D9FD001B61EB0503B0F57A7F9F
:1015200073F10003F5D3013EEFD13B6838465B69A8
:1015300098470028E8D000200DF020FE013EBBD0E7
:10154000FFF7C2FD04460D46FFF7BEFD001B61EB31
:101550000501B0F57A7F71F10001F5D3EEE700BF28
:10156000080009084891002078020908E85F002077
:10157000A8FF080870B50C48FFF7D0FE0B4BB3F876
:101580003C6316B970BD013EFCD0FFF79DFD0446DB
:101590000D46FFF799FD001B61EB0501B0F57A7F61
:1015A00071F10001F5D3EEE77802090848910020B7
:1015B00070B504460F48FFF7B1FE2046FFF7AEFEB8
:1015C0000D48FFF7ABFE0D4BB3F83C6316B970BD89
:1015D000013EFCD0FFF778FD04460D46FFF774FD91
:1015E000001B61EB0501B0F57A7F71F10001F5D3C5
:1015F000EEE700BF3400090878020908489100208E
:10160000800601D5002933D10CB470B5194C1A49A4
:10161000D4F80C0382B007AB069A01936BF0BCFCC4
:10162000D4F80C536A7A32B12B68686805F10A0164
:10163000984700236B721148FFF770FEB4F83C63C3
:101640003EB9012002B0BDE8704002B07047013ED3
:10165000F7D0FFF739FD04460D46FFF735FD001BB7
:1016600061EB0501B0F57A7F71F10001F5D3EEE78A
:101670000020704748910020E1DD00087802090849
:1016800010F0400031D00CB470B50C4682B029B1D6
:10169000002002B0BDE8704002B07047194ED6F885
:1016A0000C536B7A5A1C2B44D2B223216A72997262
:1016B0002B7A93421AD9069A134907AB284601930D
:1016C0006BF06AFCD6F80C43627A32B1D4E9003090
:1016D00004F10A01984700236372FFF74BFF0120D2
:1016E00002B0BDE8704002B070477047002AE2D0F7
:1016F000D5E9003005F10A0198476C72D6F80C5311
:10170000D9E700BF48910020E1DD00080FB410B513
:1017100082B004AB0C4C53F8042BD4F80C030B49E7
:1017200001936BF039FCD4F80C43627A32B1D4E9FE
:10173000003004F10A0198470023637202B0BDE84B
:10174000104004B0704700BF48910020E1DD000860
:101750002DE9F0413C4884B0FFF7E0FD3B4B1B6DA9
:101760005BB119689A880B691A4206D13848FFF7AD
:10177000D5FD04B0BDE8F041FCE6364C2368002BF3
:101780004AD09B699847002846D02368002B59D03F
:10179000DB69DFF8E88098470646407C3268337D95
:1017A000B1790290307C0190708A009052082A48EA
:1017B000B51DFFF7ABFF00270B3601E0B54216D091
:1017C000D8F80C4315F8011F637A5A1C2344D2B28F
:1017D00062729972237A9342F0D8002AEED0D4E94B
:1017E000003004F10A019847B5426772E8D11B4CFA
:1017F0001B48FFF793FD6378022B18D00ED804F531
:1018000080541848FFF78AFD94F8B431022B15D0A4
:10181000032BAED11448AAE71448A8E7032BA8D19C
:101820001348FFF77BFD04B0BDE8F041A2E6114884
:10183000FFF774FD04B0BDE8F0419BE60E48FFF7EA
:101840006DFD96E79B79FFDE3C000908CC2900205E
:1018500048000908782D002068000908D84C0020AD
:1018600098000908C0000908E400090858000908A0
:10187000A8000908B0000908C8000908489100201C
:101880000FB470B582B006AB174C53F8042B174950
:10189000D4F80C0301936BF07FFBD4F80C536A7AF5
:1018A00032B12B68686805F10A01984700236B7212
:1018B0000F48FFF733FDB4F83C6336B902B0BDE81A
:1018C000704004B07047013EF8D0FFF7FDFB0446BE
:1018D0000D46FFF7F9FB001B61EB0501B0F57A7FC0
:1018E00071F10001F5D3EEE748910020E1DD000839
:1018F0007802090870B508B10378EBB9FDF724F94F
:101900001348FFF70BFD1348FFF708FD124BB3F820
:101910003C6316B970BD013EFCD0FFF7D5FB044611
:101920000D46FFF7D1FB001B61EB0501B0F57A7F97
:1019300071F10001F5D3EEE7F7F7EAFB044680B258
:10194000FDF7C2F821460548BDE8704098E700BFA2
:101950000C0109087802090848910020F8000908DC
:101960002DE9F84F06466BF063FDDFF83C91044625
:10197000D9F88473F8B94148414DDFF82481FFF765
:10198000CDFC01263F49542304E055F8041F0134DF
:1019900071B10B7806FA04F2002BF6D03A42F4D07B
:1019A0004046FFF7B3FE55F8041F01340029F0D17B
:1019B000BDE8F84FDEE5024633493046F7F764F8F4
:1019C000002842D03378DFF8B8A02E4D2D2B03BF6E
:1019D000013604F1FF344FF0010B4FF0000B4FF0D4
:1019E000000804E05AF8045F08F10108C5B1224676
:1019F00029463046F7F748F80028F3D1012303FAC7
:101A000008F3BBF1000F32D027EA03031F48C9F8DF
:101A10008433FFF783FC29461D48BDE8F84F2FE7C4
:101A20001C48FFF77BFC1C48FFF778FCFFF7A2FD82
:101A300099F810333BB199F812330122134489F815
:101A4000112389F81233BDE8F88F14480C4C144D5B
:101A5000FFF764FC0B49542300E00B7828460BB1D8
:101A6000FFF754FE54F8041F0029F6D1A0E73B43CA
:101A70000C48C9F88433FFF751FCCCE7280109086A
:101A80005C5A080818010908380109085C010908AE
:101A9000343D090880FF08084C0109084001090885
:101AA0003401090868010908489100202DE9F84F20
:101AB00007466BF0BDFCDFF830910446D9F890631F
:101AC000C8B93D483D4F3E4DFFF728FC4FF0010897
:101AD0003C49234607E00134E4B207EB8402234685
:101AE000D2F80411D1B108FA03F33342F3D02846F7
:101AF000FFF70CFEEFE7024633493846F6F7C4FF1E
:101B000078B93248324C2E4DFFF708FC2D49284653
:101B1000FFF7FCFD54F8041F0029F8D1BDE8F84F89
:101B200028E53B78DFF8A8A0264D2D2B03BF013711
:101B300004F1FF344FF0010B4FF0000B4FF00008A1
:101B400004E05AF8045F08F10108C5B122462946AD
:101B50003846F6F799FF0028F3D1012303FA08F37A
:101B6000BBF1000F20D026EA03031A48C9F89033CE
:101B7000FFF7D4FB29461848BDE8F84F80E6174820
:101B8000FFF7CCFB1648FFF7C9FBFFF7F3FC99F80A
:101B900010333BB199F812330122134489F8112311
:101BA00089F81233BDE8F88F1E430E48C9F89063D8
:101BB000FFF7B4FBDEE700BF28010908DC5908087D
:101BC00034010908700109083801090840010908B1
:101BD000E05A08085C010908343D090880FF08083C
:101BE0004C01090868010908489100202DE9F84FC7
:101BF00080466BF01DFCDFF8A8A1DAF8D862D0B9F6
:101C00005B485C4CDFF89081FFF780FD04F590772E
